:020000040000FA
:10000000021F3F022003FFFFFFFFFF02200BFFFF45
:10001000FFFFFF022013FFFFFFFFFF02201BFFFF78
:10002000FFFFFF022023FFFFFFFFFF02202BFFFF48
:10003000FFFFFF022033FFFFFFFFFF02203BFFFF18
:10004000FFFFFF022043FFFFFFFFFF02204BFFFFE8
:10005000FFFFFF022053FFFFFFFFFF02205BFFFFB8
:10006000FFFFFF022063FFFFFFFFFF02206BFFFF88
:10007000FFFFFF022073FFFFFFFFFF02207BFFFF58
:10008000FFFFFF022083FFFFFFFFFF02208BFFFF28
:10009000FFFF70DFFFFF040000000002000000C847
:1000A000030002030369A5020269A532730000017F
:1000B00000000000000400FFFFFFFFFFFFFFFF0440
:1000C00003090424035400650078006100730020D4
:1000D0000049006E0073007400720075006D0065C9
:1000E000006E007400730024035400490020004394
:1000F000004300320035003300310020005500532A
:10010000004200200043004400430000035F005F02
:100110000030005800000000000000000000000057
:1001200000000000000000000000000000000000CF
:100130000000000000303132333435363738394171
:100140004243444546331C881C881C881C881C90EC
:100150001C74F8121BCD900391E06015900302749B
:10016000FEF0900304744DF0A37405F07A011207B9
:100170001C7F01021D6C74F8121BCD74FF121EB699
:100180007E00801F851882851983E064FE700690CA
:1001900003877401F0851882851983E0F890038441
:1001A000E068F07901AA18AB191210E9E9700302AE
:1001B0000287851882851983E064EF70027E07E06C
:1001C000C0E0900387E0FA900385E0F8EA28F8E4BD
:1001D0003400F9740228F582740339F583D0E0F015
:1001E000900387E0609E14600E14602B14603B1433
:1001F0006051146067809E900384E4F085188285C6
:100200001983E0900386F0C394809003874003E451
:1002100080827402020194851882851983E090031C
:1002200082F09003877403020194851882851983F4
:10023000E0900383F0900386E060199003877404D4
:10024000020194900385E004F0F8900386E0686072
:10025000030201959003877405020194900385E4DD
:10026000F0900387F0900384E0F885188285198365
:10027000E0686003020195900382E0644D60030230
:1002800001951203BF8002EEF97401121E370201BC
:100290007174F7121BCD74FB121EB6EAFEEBFF75EC
:1002A00008047509007808121ED07402121F377AEC
:1002B000907B0079041218EB7402121E3712070E9D
:1002C000121F88E0687003A3E069701285188285A8
:1002D0001983E0F47003A3E0F4600302039A74044A
:1002E000121F2F1207708A088B09A808A909740227
:1002F000121F88E8F0A3E9F07404121F88E0600878
:1003000079011201510203B3851882851983E068CF
:100310007003A3E0697076851882851983E0F47014
:1003200003A3E0F470197402121F887410F0A37410
:1003300020F08518828519837410F0A37420F0755D
:1003400008017509007808121ED07402121F377A4E
:10035000247B0812196F7402121E3775080478087E
:10036000121ED07402121F377A907B007904121883
:10037000EB7402121E3712070E121F88E06870031A
:10038000A3E069700479028006790480027903127F
:1003900001518E828F83741E80058E828F83E4F0DC
:1003A00012070E121F88E0687003A3E069700479D9
:1003B00001800279007405121E377F02021D6C74E1
:1003C000ED121BCD74F8121EB6900307E0FD9003EA
:1003D00006E0FCFAEDF8E4C8F9EA28FEE93408FF83
:1003E000751001750B00750A068E088F0974027866
:1003F00008121F1CC39508F8E49509F9740228F542
:100400000E740339F50F8E088F0974097808121FCE
:100410004EE508F511EE2410F508E43FF509EEF578
:100420000CEF5401F50D900383E014605914700330
:100430000204FB14700302057614601024FE70039E
:100440000206311470030206E10206F1750A03790F
:100450004E1213BD9003071207047402F0A37440F8
:100460001207027408120702F0A3F07418C394076D
:1004700004F510AA10A90B12071CA90A7408121E71
:10048000377F0C021D6C750A04794E1213BDEE45C0
:100490000D7005A9111219D5C3EE9425EF940850DB
:1004A0003CC3E5089424E50994084031E50E249600
:1004B000F8E50F3420F988828983E0701BA3AA82B3
:1004C000AB83E070139003887401F0888289837491
:1004D000A5F08A828B838004900388E4F07508106D
:1004E0007509007808121ED07C087D03EEFAEFFB38
:1004F00012196F7402121E37020473750A05E51192
:10050000C394794006750B0102047375124075138C
:10051000007812121ED07C097D037402780C121F21
:100520001CAA0CAB0DA9111218EB7402121E379005
:100530000307E0A3F0900306E0A3F0751043C3EEB9
:100540009425EF94084003020473C3E5089424E55E
:100550000994085003020473900388E070030204B6
:1005600073E50E2497F8E50F3420F988828983E437
:10057000F0A3F00204737508047509007808121ED0
:10058000D07402121F377A907B0079041218EB7432
:1005900002121E377402121F88E0F8A3E0F98518D2
:1005A00082851983E0687003A3E069851882851944
:1005B00083700BE0F47003A3E0F470578009E0F45B
:1005C0007003A3E0F4700D8518828519837410F010
:1005D000A37420F012070E121F88E8F0A3E9F0754B
:1005E00008017808121ED07402121F377A247B0883
:1005F00012196F7402121E377508047808121ED083
:100600007402121F377A907B0079041218EB74027F
:10061000121E3712070E121F88E0687003A3E069EC
:100620007006750A01020473750A02750B0702044D
:10063000739003D6E0600764026003020473EDFF69
:100640007A01790012071CE060030206D5800312CC
:10065000118512116CE970F77404121F881206F6E6
:100660007404121F887808121F6C85080C85090D08
:10067000850A0E850B0F9003C2780C121EF67404C7
:10068000121F88780C121F5DE5084509450A450BC5
:1006900070CE8EC2E5C554E04FF5C57404121F88B4
:1006A0001206F67404121F887808121F6C85080C55
:1006B00085090D850A0E850B0F9003C2780C121E5A
:1006C000F67404121F88780C121F5DE50845094571
:1006D0000A450B70CE7A01790012071C79080204D2
:1006E0007CEC900391F07003020473750A09020414
:1006F00073790602047CE4F0A37426F0A3E4F0A36B
:10070000F022F0A3E4F0A3F0A3F0A3F0A322851855
:1007100082851983E0F8A3E0F974022274F8121BB1
:10072000CDEAFE900305E0D2E7F0E9A3F0EE9003F6
:1007300003F08E0874042AFE7C028004E062080C38
:10074000ECFA3395E0FB74022AF58274033BF583DF
:10075000EEF8C3EA98EB9400A2D265D03340DDE511
:1007600008F074012AF97A027B0312112702017141
:1007700074E9121BCD7582007583FE121E198A164C
:100780008B177514007515008A828B83E4F0900333
:10079000D6E07006D2AAD2AF800464027005790058
:1007A000120151750C00750D20750E00750F00902B
:1007B00003D6E0600464027015121185120176E917
:1007C000F874096860030208AC7900120151E06412
:1007D000027007A29240030208877508007509029B
:1007E0007808121ED07402121F37850C08850D0977
:1007F000AA08E5095407FB850E0A850F0B740B78D0
:1008000008121E87A9081218EB7402121E377E0008
:100810007F009003CAC0828E10EFF5113395E0F58A
:1008200012F513850C08850D09850E0A850F0B78C6
:10083000087910121F099003C67808121EF67583F6
:1008400003D0827808121DFA501D851882851983FD
:10085000E5822EF582E5833FF583E0F9AA14AB1516
:100860001208DB8A148B150EEE70010FC3EF940291
:1008700040A09003CE780C121EF69003D2780C1292
:100880001DFA40030207AF7900AA14AB151208DB6A
:1008900079001208DB8B159003D6E07004C2AFC25A
:1008A000AAEA451570277AA57BA58021E870030286
:1008B00007CE74066870030207CE740768700302DF
:1008C00007CE8516828517837401F080BA75820081
:1008D000758302121E197F10021D6CC008C0097CAE
:1008E000088A088B09740F7808121F4EE508F8EA89
:1008F00025E0FAEB33FBE9A2E7500474014AFAE879
:10090000A2E0500874216AFA74106BFBE9C333F952
:100910001CEC70CDD009D00822C082C083120F33E6
:1009200060030209F0A3E0F8A3E060030209F0A36A
:10093000E064027002A3E060030209F09003B8E0F3
:100940002480600914604F14605C0209F0E86003C1
:100950000209F09003B2E060047801800278009010
:1009600003C0E8F0A3E4F09003B1E0600A9003C094
:10097000E04402F0A3E4F09003A6E0640460149065
:1009800003B374C0F0A37403F0A3E4F0A3740212E1
:100990000F95F0020E6E90039FE064047052900376
:1009A000C0E4F0A380D0E8547FFA90039FE0640491
:1009B000703EEAC394065038749F2AF582E43403EB
:1009C000F583E854806018A3A3A3A3A3A3A3E064C2
:1009D0000370047801800278009003C0E88094E5F9
:1009E00082240CF58250020583E0640370E980E301
:1009F0009003A67404809B74F8121BCDE9FE90034B
:100A0000BE120F366003020AD990039FE0640460AF
:100A10000B9003BC120F366003020AD99003B8E0B2
:100A2000541F6009146030146020020AD99003BA80
:100A3000E064017022EE9003B1F060047905800259
:100A400079067A00121BCB020ADF9003BCE0547FC8
:100A5000FA9003BAE060057900020AE1EAC394065D
:100A60005077EA90620EF0749F2AF8E43403F9900C
:100A700003BCE05480602EEE600474108002744069
:100A8000906211F0EE60047B0380027B00EB8882B1
:100A90008983A3A3A3A3A3A3A3F0EE600479088092
:100AA0002F7907802BEE60047B2080027B80EB9007
:100AB0006214F0EE60047B0380027B00E8240CF5F6
:100AC00082E439F583EBF0EE6004790A800279095B
:100AD000121BCB90620EE480059003A67404F0799B
:100AE000017F01021D6C79001209F7E97003121BE6
:100AF000BA2279011209F7E97003121BC922C082D8
:100B0000C0839003BC120F367015A3120F36700FFE
:100B10009003BA120CD95480FAE9FBEA4B600790B3
:100B200003A67404801AE8906200F090039F6009A5
:100B3000E06402700C74038007E0640370037402C5
:100B4000F0020E6E74F5121BCD9003BAE0FAA3E02A
:100B50001460081460101460398057121754120C76
:100B6000B6A37B8080417900121776120CB67B8089
:100B7000E92402F9E43AFA121E6DFC1919E0FAA30D
:100B8000E92403F9E43AFA121E6DF9ECA3F0A3E9A3
:100B9000801CEAF91217E49003B3EAF0A3EBF0A388
:100BA000E4120CC5A37B00121E6DA3F0A3E4F002B7
:100BB0000C709003B3E4F0A3F0A3F0750B00900465
:100BC0007DE0FAA3E0FB020C4E850B08750900746A
:100BD000037808121F1CEA2508F8EB3509F9900381
:100BE000BA120CCFE493C0E0EFFCD0E06C705DA3D0
:100BF000E4936E70579003BC120CCFA3A3E493C090
:100C0000E0EFFCD0E06C704488828983A3A3A3E466
:100C1000936E703888828983A3A3A3A3E493F50815
:100C2000740193F5099003B3E508F0A3E509F0A377
:100C30007480F088828983A3A3A3A3A3A3E493F879
:100C4000740193F99003B6E8F0A3E9F0050B900462
:100C50007F120CD9C39AF508E99BF509740378084B
:100C6000121F4EC3E50B9508E495095003020BC90A
:100C70009003B3E0FCA3E0FDA3E0FEEC4D4E900337
:100C8000A6700474048029E0640460259003BEE02B
:100C9000FAA3E0FB9003B6E0F8A3E0F9C3EA98EB0F
:100CA0009950089003B6EAF0A3EBF09003A6740104
:100CB000F07F04021D6C9003B3EAF0A3EBF0A37481
:100CC00080120CC522F09003B3E0F9A3E0FA22E011
:100CD000FEA3E0FF8882898322E0F8A3E0F9E822FE
:100CE00074EE121BCDEA2404F8E43BF98808890964
:100CF0008882F583E4936025900481120CD9FEE983
:100D0000FF8007EE2404FE50010F8E828F83E49350
:100D1000F8740193F9EA687002EB6970E6750B00EC
:100D2000803F9062147490F07410120E3570037549
:100D30000A408E828F83A3A3A3E493550E6006E539
:100D40000AD2E0F50AE50A906215F0EA906213F023
:100D5000EC240CF582E43DF583E4F090620EF0059E
:100D60000B850882850983E493F8E50BC39840035B
:100D7000020E307A0079051216E78A0C8B0DEA45CF
:100D80000D60DCEA2402F8E4350DF9881089118839
:100D900082F583E493540FF51290620EF0750A0009
:100DA0008A828B83A3A3A3A3E4932407F50EA3E471
:100DB000933400F50F7403780E121F4EAA0EA8127A
:100DC000749F28F8E43403F9E8FCE9FD750E017519
:100DD0000F00E512780E121F1CE50EF50EE50C242F
:100DE00003F8E4350DF9851082851183E493A2E7B9
:100DF0004003020D229062117448F07408120E35FF
:100E00007003750A408E828F83A3A3E493550E600E
:100E100006E50AD2E0F50AE50A906212F0EA90626D
:100E200010F08C828D83A3A3A3A3A3A3A3020D59C7
:100E30007F0B021D6CF088828983E4935403640164
:100E400022C082C083120F337010A3120F36700AB3
:100E5000A3E064017002A3E060079003A67404801D
:100E60000C9003B374A0F0A37403120F8BF0D08323
:100E7000D0822274F3121BCD90039FE064026014B1
:100E80009003BC120F36700CA3120F36700690033D
:100E9000BBE060099003A67404F0020F2E7A00797B
:100EA00001121BCB9003BAE0606F7A00F91217763B
:100EB0008A0A8B0BEA450B605890039F7404F090EC
:100EC00003BAE09003A0F0750800850A82850B83C1
:100ED000A3A3A3A3E493F8E508C398504AA8087411
:100EE000A128F8E43403F9E8FEE9FF8E828F83E459
:100EF000F07A0079041216E78A828B83A3A3A3E415
:100F000093F88E828F83E06870E7120CE00508800A
:100F1000B99003A67404F0800E9003A0F090039F94
:100F20007403F0F91216677A007902121BCB7F0660
:100F3000021D6C9003BAE0F8A3E0F9E8492274F6C8
:100F4000121BCD90039FE0640470199003B8E06415
:100F5000817011120F33700C9003BEE064017002B7
:100F6000A3E060079003A67404801A9003BCE024F9
:100F7000A1F508A3E03403F5099003B3E508F0A355
:100F8000E509120F8BF07F03021D6CF0A3E4F0A3C0
:100F900004120F9522F0A3E4F09003A6042274F744
:100FA000121BCD90039FE0640470649003B8E0646A
:100FB00001705C9003BE120F3670549003BAE0FBD0
:100FC0009003BCE0FA9003A0E0F91217AE8A088BF8
:100FD00009AE08AF09EE4F60369003BCE0FA790322
:100FE000121BCB9003BAE0C0E09003BCE024A1F850
:100FF000A3E03403F988828983D0E0F0EEFAEFFBB6
:10100000120CE09003BCE0FA7904121BCB8006902E
:1010100003A67404F07F02021D6CC082C0838003AB
:10102000121A31A2E840F9A823E854046009782391
:10103000E654FBF612140EA823E854106009782336
:10104000E654EFF612142FA823E8A2E05005782307
:1010500054FCF690620EE0FA7404F0906214E0A280
:10106000E05039A9A8C2AF906216E0F8A3E0E8FB0F
:10107000E9A2E792AF8017906228E0C0E090039366
:10108000E0F812111CD0E0F0900393E004F0EBFDC7
:1010900074FF2DFB0470E0906214E4F0EA90620E9D
:1010A000F0E0FC7404F0906211E0A2E040319003A3
:1010B00095E0F8900394E06860257A4090039412DC
:1010C000115FE0906228F0900394E004F008900330
:1010D00095E06860041AEA70E39062117401F0EC24
:1010E00090620EF0D083D0822274F8121BCDE9FEFC
:1010F0007900801212111CE08A828B83F090039297
:10110000E00412115409900392E0F8900393E06810
:101110006005E9C39E40DD7F01021D6C748528F5E2
:1011200082E43404F58322C082C083E9FC80188AFB
:10113000828B83E0C0E090039512115FD0E0121122
:1011400054900395E004F0ECF874FF28FC0470DF81
:1011500079018090F08A828B83A3AA82AB8322E0FC
:10116000F8748528F582E43405F58322C082C083B3
:10117000900395E0F8900394E068600479018002A0
:1011800079000210E402101A74FB121EB67E009061
:1011900006857808121F6C794A1213BD9006857473
:1011A00001F0A3F0A37469F0A374A5F09003D778BD
:1011B00008121EE170047E0180159003DB7808128E
:1011C0001EE16008E59D541864107003022000EED3
:1011D000F9121334C280D291EEA2E050030212E75A
:1011E000AA18AB19120291E970030212E7C29185A5
:1011F0001882851983E0C3943C500EE0F8743CC318
:1012000098F50895E0F5098006750800750900E471
:10121000F50AF50B9003DF780C121F6C7808790C37
:10122000121AD1790612015112101A120176E9F838
:101230007409687007790612015180277407686085
:1012400016A2935012E8600874066860030212E761
:10125000A292400F0212E7750800750900750A0096
:10126000750B0085080C85090D850A0E850B0F90FE
:1012700003C27808121EF6E50C450D450E450F70A9
:10128000A7D2807907120151800312101A12116C33
:10129000E970F77E007F007401121F88E4F0A374E8
:1012A00026F0A3E4F0A3F07401121F887808121F3F
:1012B0006C85080C85090D850A0E850B0F9003C2FD
:1012C000780C121EF67401121F88780C121F5DE54F
:1012D000084509450A450B70CEA29250FCA29350D6
:1012E000F81213B8022000D280D291794E1213BDA9
:1012F000750800750900750A00750B007905120163
:101300005112101A120176E9F874096860EE74013E
:101310006870EE12101A9003E37808121EF690031C
:10132000E77808121DFA50EB1213B802200074057A
:10133000121E372274F8121BCDE9FE53BEFBE59D49
:10134000A2E650FA0078F8790100E824FF18E934A1
:10135000FFF9E84970F375C6807480659E70FA43A2
:10136000BE049062707408F01213ADEE700853F46E
:10137000FEC29043FE017403F5D575D4899003969F
:10138000E4F0A374C2F0A37401F0A3E4F0A3F0A30B
:10139000F0A37408F01213D37AFF7BFF1219EC53F9
:1013A000F4FED29043FE011213AD021117D2804316
:1013B000FD01C29143FE0222D280C29122781075B3
:1013C000B60FE5B4A2E750FAE5BBC39940F118E8BF
:1013D00070ED2274F7121BCD7A0079011217768A0C
:1013E000828B83A3A3A3A3A3A3A3E493A2E6900366
:1013F000B2500474018001E4F09003B1E4F0906213
:101400000F7403F0E0A2E750FB7F02021D6CC08264
:10141000C08390039F7402F0A3E4F09003A6F079D8
:1014200003121667752100752200D083D0822274C2
:10143000F6121BCD90620EE0FEE4F0906211E0FF28
:10144000A2E4501D7480F09003A67407F0E52145D6
:10145000226009852182852283121F979003A6E4CA
:10146000F0EFA2E2500B906211E4F09003A6F0803E
:10147000679003A6E0F87402687046906216E0FF79
:101480009003B3121DACEFF97A207B6212168174BF
:1014900003121E37EFF89003B612164512164F2F9F
:1014A000121657A3E0F8A3E0F9E8496004744080FD
:1014B000027448906211F0E849600302163B02167C
:1014C000177406687009852182852283121F979000
:1014D00003A6E060030215C2EFA2E0400302163B40
:1014E0007508B8750903750A007808121ECC7908CA
:1014F0007A207B621216817403121E3775210075E3
:1015000022009003B8E054E0601D24E0700302154F
:101510009D24E0607224C0604824E070030215A896
:1015200024E0606E0215B3A3E014602624FE601D63
:1015300024FE600A24FC601F24FE60208075120ACD
:10154000FE9003A6E06404707278608070120AF264
:1015500080EF120AE680EA120E7380E5120F9E8079
:10156000E0A3E0600E24FA600F24FE601024FE6009
:1015700011804012091980C9120B4480C4120E4117
:1015800080BF120F3E80BA7521B675221B121BB6A2
:1015900080AF7521B875221B121BB880A47521512C
:1015A00075221B121B51809975218175221B121BFC
:1015B00081808E9003A67404F0808E7840E890625B
:1015C00011F09003A6E0F874016870617F02900347
:1015D000B6E0F8A3E0F9C3E89420E994005007E8E6
:1015E000F5087F0A80037508209003B3121DACA98B
:1015F000087A207B621216AC7403121E37AC0812F4
:10160000164F2C121657A808A3121645EF90621118
:10161000F0E8C394205024E5214522600985218209
:10162000852283121F979003A6E4F0800E7405684C
:101630007009852182852283121F97EE90620EF039
:101640007F03021D6CC3E098F0A3E09400F02290A9
:1016500003B31216D9E922F9E43AFA9003B3E9F098
:10166000A3EAF0A3EBF022C082C083E99003A7783D
:1016700005F0A3D8FC9003AC7805F0A3D8FC0214C5
:101680002A74F8121BCDEAFCEBFDE9F87408121F6E
:10169000881216D460118C828D83E0121EA0E9247A
:1016A0000109E43AFAD8EF7F01021D6C74F8121BAD
:1016B000CDEAFCEBFDE9F87408121F881216D4601D
:1016C00011121E6D8C828D83F0E9240109E43AFA2F
:1016D000D8EF80D31216D9E822E0F9A3E0FAA3E00C
:1016E000FB22D083D08222C082C083E9FCEAFD7A4B
:1016F000007B00800312173290039DE0F8A3E0F90D
:1017000090047BE0687003A3E069602490039EE08E
:10171000F5838882A3E493F8EC68700D90039DE054
:10172000FAA3E0FB1217328007ED6870C8ED60C5C0
:1017300080B090039DE0F8A3E0F5838882E493F8FD
:1017400090039DE028F8A3E03400F990039DE8F0B1
:10175000A3E9F022C082C0831217657A00790112D2
:1017600016E70216E2900479E0F8A3E0F990039DF1
:10177000E8F0A3E9F02274F7121BCDE9FFEAFE12AC
:1017800017657A0079021216E7EA4B601CEF6010C9
:101790008A828B83A3A3A3A3A3E4936F70E480093D
:1017A000EEF874FF28FE0470D97F02021D6C74F5F8
:1017B000121BCDEAFF8B087A001217767A027904A1
:1017C0001216E7EA4B60188A828B83A3A3E4936F17
:1017D00070EA8A828B83A3A3A3E493650870DD7FFC
:1017E00004021D6C74F7121BCD74F0121EB6E97A58
:1017F000007B00600C146010146014146018021850
:10180000D47AF37B030218D47AF77B030218D47AD4
:101810001B7B040218D490043FE060030218D090B0
:1018200003EB7408121F377408121DD9750808F5E8
:10183000097808121ED07402121F377AE87B0779E4
:101840007F1218EB7402121E377808121ED0740A29
:10185000121F377402121F2F121C907402121E37AF
:101860008B09EA450970197509007808121ED07CA9
:101870000C7D787402121F2F121D267402121E375F
:101880007C287D00EDF8851882851983E58228F58E
:1018900082E43583F583E0FFECF8743F28F8E43404
:1018A00004F9EF1218DC88828983F0EFC41218DC87
:1018B000C0E0E824FEF582E934FFF583D0E0F00DC6
:1018C00074FC2CFCEDC3940840BA90043F742AF0D9
:1018D0007A3F7B047410121E370217A9540FFA7452
:1018E000692AF582E43404F583E02274F6121BCDF4
:1018F000890A740F550AF508750900740B780812E7
:101900001F1CEA2400F8EB3480F9E82400E93509CB
:10191000F985C709A2AFE433F508C2AFE50AC4549C
:101920000FFAE5C754F84AF5C7740A121F88E0FA9F
:10193000A3E0FB801C88828983E08C828D83F08801
:10194000828983A3A882A9838C828D83A3AC82AD74
:1019500083EAFEEBFFEE24FF1AEF34FFFBEE4F703D
:10196000D48509C7E508A2E092AF7F03021D6C741D
:10197000F7121BCDED900389F0ECA3F0A37462F095
:10198000A37473F0A3E0541FF07409121F88E0F5EC
:1019900008A3E0F509E508333354FC90038EF07496
:1019A000067808121F4EE50890038DF090038F749F
:1019B00012F0A37442F075D1FE75D601EA906271FF
:1019C000F0EBA3F0906270E0D2E1F0E0A2E740FB20
:1019D0007F02021D6CC082C083E9C333906272F043
:1019E000906270E0D2E0F0D083D0822274F7121BB4
:1019F000CD7523007524007525008A268B27EA9073
:101A0000620BF08A088B0974047808121F4EE508EF
:101A1000906207F08A088B0974097808121F4EE556
:101A200008543E906209F0758B00C2E87F02021DE7
:101A30006C74F7121BCDE59DA2E650FA906206E0A9
:101A4000F9A2E25034AA26EA90620BF0F508852745
:101A50000974047808121F4EE508906207F08A089E
:101A600085270974097808121F4EE508543E9062D4
:101A700009F0906201E0D2E0F0E9782346F6906246
:101A800002E0F50875090074047808121F1C782319
:101A9000E50846F608E50946F6906204E0F50875A3
:101AA000090074097808121F1C7824E50946F6E934
:101AB000A2E050037525017406596003752500E501
:101AC0008BA2E55006758BDF752500121BCC021A20
:101AD00027080808EAC0E0EBC0E086F0E7A4FA189F
:101AE0000986F0E7A42AFA180986F0E7A42AFA186A
:101AF0000986F0E7A42AFA1986F0E7A4FBE5F02AA4
:101B0000FA190886F0E7A42BFBE5F03AFA190886E3
:101B1000F0E7A42BFBE5F03AFA18180986F0E7A4E1
:101B2000C5F02BFBE43AFA1908E7C5F0C6A426F67F
:101B3000E5F03BFBE43AFA1886F0E7A4F6E5F00896
:101B400026F6E43B08F6E43A08F6D0E0FBD0E0FAEB
:101B500022C082C0839003B9E0F8742268700890B4
:101B600003A6E0701A80117420689003A6700DE03F
:101B7000700D121BA89003A6740280027404F080FA
:101B800043C082C0839003B9E064219003A6701320
:101B9000E07013121BA8A37407F0A3E4F09003A64F
:101BA0000480027404F0801C9003B37496F0A37454
:101BB00003F0A3E4F02280028000C082C08390037F
:101BC000A67404F0D083D0822280EF22222518C58B
:101BD00082C0E0E51934FFC583C0E0E518C39582F3
:101BE00024F910AF08858319858218800885831928
:101BF000858218D2AFCEF0A3E520F0A37808E608DE
:101C0000F0A3DEFAEFF0A3E58124FBF8E608F0A3E9
:101C1000E608F0A30808E608F0A3E608F0A315819B
:101C20001581D0E0FED0E0F815811581E8C0E0EE26
:101C3000C0E02212010002020000205104A816098F
:101C40000001020301090243000201008019090496
:101C50000000010202010005240010010424020218
:101C60000524060001052401000107058203400048
:101C70004009040100020A00000007058402400038
:101C800000070504024000004E1C0000711C00000B
:101C900074F8121BCD7408121F88E0FEA3E08015B3
:101CA000A3AA82AB838C828D83A3AC82AD83EE2406
:101CB000FF1EEF34FFFFEE4F60198C828D83E0F83A
:101CC0008A828B83E0F9E86960D6E9C398FA95E0E7
:101CD000FB80047A007B007F01021D6CE47921788F
:101CE00007B800028004F709D8FCE490030278C129
:101CF00079018002F0A3D8FCD9FA7AC27B03900064
:101D00008E78C479018015E493A3AD82AE838A8274
:101D10008B83F0A3AA82AB838D828E83D8E9D9E727
:101D2000121188121F9274F7121BCDEAF8EBF974A6
:101D300009121F88E0FEA3E0FF80188C828D83E0EB
:101D400088828983F0A3A882A9838C828D83A3AC27
:101D500082AD838E088F09E50824FF1EE50934FF54
:101D6000FFE508450970D47F02021D6C8519838543
:101D70001882E0A3FEE0A3F5207808E0A3F608DFD0
:101D8000FAE0A3FFE0A3C0E0E0A3C0E0E0A3C0E06E
:101D9000E0A3C0E010AF088582188583198008850C
:101DA0008218858319D2AFD083D082227403800039
:101DB000CCC0E0EDC0E0E518C39CCCAD1950011DCE
:101DC00010AF068C188D1980068C188D19D2AF12A1
:101DD0001DD9D0E0FDD0E0FC22CAC0E0E0A3C5825E
:101DE000CCC582C583CDC583F0A3C582CCC582C5D1
:101DF00083CDC583DAE6D0E0CA22C008C3E096F5F9
:101E00000808A3E096420808A3E096420808A3E069
:101E10009645087001D3D00822C5822518C582C511
:101E200083351910AF07F5198582188007F51985D4
:101E30008218D2AFC5832200C0D0251810AF08F594
:101E400018500C05198008F51850020519D2AFD0AA
:101E5000D0222518F58210AF08F518400C1519800E
:101E600008F51840021519D2AF85198322BB01026B
:101E7000E722C082C08389828A83BB0003E080029C
:101E8000E493D083D082226016080808C6C313C624
:101E900018C613C618C613C618C613C6D5E0EA225C
:101EA000BB000EC082C0838A838982F0D083D08237
:101EB00022BB0101F722251810AF08F518400C15B8
:101EC000198008F51840021519D2AF227403800456
:101ED00074028000C0E0F404121E52D0E0121F7B96
:101EE00022E066701008A3E066700A08A3E066703E
:101EF0000408A3E06622E026F608A3E036F608A36D
:101F0000E036F608A3E036F622E627F60809E637BB
:101F1000F60809E637F60809E637F622700422606B
:101F20000D18C6C333C608C633C6D5E0F41822253B
:101F300018FAE43519FB222518FCE43519FD227541
:101F4000D00075813F751802751903021CDC600C06
:101F500008C6C313C618C613C6D5E0F422E6F008B7
:101F6000A3E6F008A3E6F008A3E6F022E0F608A353
:101F7000E0F608A3E0F608A3E0F622CAC0E0E6F027
:101F8000A308DAFAD0E0FA222518F582E43519F52B
:101F9000832200000080FBE473FFFFFFFFFFFFFFD1
:101FA000FFFFFFFFFFFFFFFFFFFFFFFFFFFFFFFF41
:101FB000FFFFFFFFFFFFFFFFFFFFFFFFFFFFFFFF31
:101FC000FFFFFFFFFFFFFFFFFFFFFFFFFFFFFFFF21
:101FD000FFFFFFFFFFFFFFFFFFFFFFFFFFFFFFFF11
:101FE000FFFFFFFFFFFFFFFFFFFFFFFFFFFFFFFF01
:0A1FF600850609433886000000004C
:020000040003F7
:01FFF000F020
:020000040000FA
:10200000022D6F02222DFFFFFFFFFFFFFFFFFFFFEB
:10201000FFFFFFFFFFFFFFFFFFFFFFFFFFFFFFFFD0
:10202000FFFFFFFFFFFFFFFFFFFFFF022B39FFFF57
:10203000FFFFFF02224FFFFFFFFFFFFFFFFFFFFF3A
:10204000FFFFFFFFFFFFFFFFFFFFFFFFFFFFFFFFA0
:10205000FFFFFF02216DFFFFFFFFFFFFFFFFFFFFFD
:10206000FFFFFFFFFFFFFFFFFFFFFF022A02FFFF4F
:10207000FFFFFFFFFFFFFFFFFFFFFF022889FFFFBA
:10208000FFFFFF0221C1FFFFFFFFFFFFFFFFFFFF79
:1020900010201020010020FD00020000703100001F
:1020A00000000A31F4314031B23100003431000017
:1020B0000000000000000000000000000000000020
:1020C00000000000000006FFFFFF00035F005F004C
:1020D0003000580000000000000000000000000078
:1020E00000000000000000000000000000000000F0
:1020F00000000000AB260027002700270027082744
:1021000001010400CB18000000E8030000FFFF46B7
:102110001903E803000064006400B801A0BB0D00CF
:10212000A0BB0D0002020008000005020704010523
:102130001E02051E020A0A01080803B80B02803EAF
:102140000102FEFFE8030A050001FFFF0A1401E097
:10215000010105030101FF0F10FEFF174E000000F3
:1021600000894C00000000FF000000FF00C0E07488
:10217000F212264CA2AFE433F508D2AFAFA7AEA15E
:10218000EE5F54106006122EA075A1EFEE5F5408AA
:102190006008122EA675A1F78023EEA2E092F0EF60
:1021A000A2E082F05017906198E0F890054CE0C3EF
:1021B00098A2D265D0335002E8F075A1FEE5088000
:1021C00063C0E074F212264CA2AFE433FED2AF90AB
:1021D00061A4E0F8759B00E591585408600875917A
:1021E000F7122EEE8023E59158541060087591EF98
:1021F000122EF48014E591A2E092F0E8A2E082F0C1
:102200005007E0C2E0F012303E9061A3E0F8E5E94B
:10221000585404600E12301475E9FB906193E0A2EB
:10222000E640F2EEA2E092AF7F01022708C0E07420
:10223000F212264CA2AFE433FED2AF9061A5E0F8D3
:10224000E5BF585404600675BFFB12305680D4C0F9
:10225000E074F112264CE59DA2E650FA906206E089
:10226000F9A2E25034AA2CEA90620BF0F508852D11
:102270000974047808122D8EE508906207F08A0828
:10228000852D0974097808122D8EE508543E906258
:1022900009F0906201E0D2E0F0E9782946F6906218
:1022A00002E0F50875090074047808122CBF78293B
:1022B000E50846F608E50946F6906204E0F508757B
:1022C000090074097808122CBF782AE50946F6E956
:1022D000A2E05003752B017406596003752B00E5CD
:1022E0008BA2E55006758BDF752B00123572758B4E
:1022F00000C2E87F02022708C3E498F8E499F912C3
:1023000023398026C3E49AFAE49BFBE920E7E9122B
:102310002339E498F8E499F922C3E498F8E499F9A8
:10232000122339E498F8E499F9C3E49AFAE49BFBA0
:1023300022EB20E7CFE920E7E0B90010BB0008E876
:102340008AF084F8AAF022E4FBC8FA22EB70227B20
:1023500010C833C8C933C9335007C39AC3DBF280EE
:10236000069A50012ADBEAC833F4C8C933F4C9FA23
:102370002275F008E4C833C8C933C933C99AC99B68
:102380005004C92AC93BD5F0ECFBC833F4C8E4C9F2
:10239000FA2274F512258374FA122BB675080475A7
:1023A00009007808122B267404122B967AF87B0702
:1023B00079031248F87402122AE890811F780812F3
:1023C0002D7F7402122E007808122C0D70487508AB
:1023D000027509007808122B267402122B967AF6E1
:1023E0007B0779031248F87402122AE8851882855F
:1023F0001983E0F47003A3E0F4601B85188285194B
:1024000083E0F8A3E08882F5837402F0A3F0A3745C
:1024100069F0A374A5F0C2AF75D69F0200007406E0
:10242000122AE87F040228CC080808EAC0E0EBC0C2
:10243000E086F0E7A4FA180986F0E7A42AFA18095A
:1024400086F0E7A42AFA180986F0E7A42AFA198682
:10245000F0E7A4FBE5F02AFA190886F0E7A42BFBC5
:10246000E5F03AFA190886F0E7A42BFBE5F03AFA12
:1024700018180986F0E7A4C5F02BFBE43AFA19080E
:10248000E7C5F0C6A426F6E5F03BFBE43AFA188669
:10249000F0E7A4F6E5F00826F6E43B08F6E43A088F
:1024A000F6D0E0FBD0E0FA22E4CFC0E0E4CEC0E01A
:1024B000E4CDC0E0E4CCC0E075F020E626F608E606
:1024C00033F608E633F608E633F6181818EC33FC52
:1024D000ED33FDEE33FEEF33FFC3EC9709ED9709C3
:1024E000EE9709EF97191919400FFFEC97FC09EDCA
:1024F00097FD09EE97FE191906D5F0BFECF709ED27
:10250000F709EEF709EFF7191919D0E0FCD0E0FD53
:10251000D0E0FED0E0FF222518C582C0E0E51934E6
:10252000FFC583C0E0E518C3958224F810AF088585
:1025300083198582188008858319858218D2AFCEC9
:10254000F0A3E520F0A37808E608F0A3DEFAEFF0A8
:10255000A3E58124FAF8E608F0A3E608F0A3E6086C
:10256000F0A30808E608F0A3E608F0A3158115819A
:10257000D0E0FED0E0F8158115811581E8C0E0EECD
:10258000C0E0222518C582C0E0E51934FFC583C02C
:10259000E0E518C3958224F910AF08858319858278
:1025A000188008858319858218D2AFCEF0A3E52064
:1025B000F0A37808E608F0A3DEFAEFF0A3E58124A3
:1025C000FBF8E608F0A3E608F0A30808E608F0A385
:1025D000E608F0A315811581D0E0FED0E0F8158162
:1025E0001581E8C0E0EEC0E022122DF5B90003022B
:1025F0002636E47921780DB800028004F709D8FC6A
:10260000E49004D1785579188002F0A3D8FCD9FA67
:102610007A257B1C90209478DA79018015E493A3C5
:10262000AD82AE838A828B83F0A3AA82AB838D8234
:102630008E83D8E9D9E77582AE7583AD7406122A08
:10264000CA75828475834A7400122ACAC0D02518BC
:10265000C582C0E0E51934FFC583C0E0E518C39525
:102660008224F310AF08858319858218800885833A
:1026700019858218D2AFC8F0A3E9F0A3EAF0A3EB62
:10268000F0A37908E709F0A3D8FAECF0A3EDF0A3E2
:10269000EEF0A3EFF0A3D0E0F0A3D0E0F0A3D0E001
:1026A000F0A3E520F0A3E5F0F0A32212010002025E
:1026B0000000205104A81609000102030109024389
:1026C0000002010080190904000001020201000556
:1026D000240010010424020205240600010524013F
:1026E00000010705820340004009040100020A00BE
:1026F00000000705840240000007050402400000B6
:10270000C6260000E9260000851983851882E0C0EE
:10271000E0A3E0F9A3E0FAA3E0FBA37808E0F60861
:10272000A3DFFAE0FCA3E0FDA3E0FEA3E0FFA3E04B
:10273000C0E0A3E0C0E0A3E0F5D0A3E0F520A3E073
:10274000A3F5F010AF08858319858218800885836A
:1027500019858218D2AFD082D083D0E0F8D0E03291
:1027600075F0108E218F228582268583258518821B
:10277000851983E0CEA3E0CF852682852583EBC92A
:10278000EAC8EDCBECCAC3E833C8E933C9EA33CAB7
:10279000EB33CBC3EA9EF524EB9FF523B35004AB98
:1027A00023AA24EC33CCED33CDD5F0DAAE21AF2221
:1027B00022D083D082ECC0E0EDC0E0E493A3FCE43F
:1027C00093A3FDED4C600D12290CEC24FFFCED34BD
:1027D000FFFD80EFE493A3FCE493A3FDED4C600DBB
:1027E0001229ADEC24FFFCED34FFFD80EFD0E0FDBD
:1027F000D0E0FCE493A3C0E0E493C0E022D083D017
:1028000082E9C0E0E493A3C386F0C5F095F0F9082F
:10281000E493A386F0C5F095F0700BE493A3C399FD
:102820004005E9048002A3E475F002A42582F58244
:10283000E5F03583F583D0E0F9E493A3C0E0E493B9
:10284000C0E022851983851882E0A3FEE0A3F5206D
:102850007808E0A3F608DFFAE0A3FFE0A3C0E0E019
:10286000A3C0E0E0A3C0E0E0A3C0E0E0A3C0E010AC
:10287000AF08858218858319800885821885831999
:10288000D2AFD083D082022AD0C0E074F212264C9C
:10289000A2AFE433FED2AFE58AA2E2500790050F63
:1028A000E0D2E0F0E58AA2E3500790050FE0D2E124
:1028B000F0758A00C2EB7A107B0090050BE0F912EC
:1028C0003320EEA2E092AF7F0102270885198385AD
:1028D0001882E0A3FEE0A3F5207808E0A3F608DF65
:1028E000FAE0A3FFE0A3C0E0E0A3C0E0E0A3C0E003
:1028F000E0A3C0E010AF08858218858319800885A1
:102900008218858319D2AFD083D08222C0E0C3E47D
:102910009396087401939618400FE4936670080824
:10292000740193661870007019A3A3C3E49396080A
:102930007401939618A3A3400DD0E0D0E0D0E0023C
:1029400027EDA3A3A3A3A3A3D0E02274048008745B
:1029500003800474028000CCC0E0EDC0E0E518C341
:102960009CCCAD1950011D10AF068C188D19800636
:102970008C188D19D2AF122A4CD0E0FDD0E0FC2289
:1029800074028000CCC0E0EDC0E0E518C39CCCAD83
:102990001950011D10AF068C188D1980068C188DEA
:1029A00019D2AF122A2AD0E0FDD0E0FC22C0E0C04C
:1029B000F088F0E49366700808740193661870005C
:1029C000A8F0A3A3700BD0F0D0E0D0E0D0E00227B5
:1029D000EDA3A3D0F0D0E022D083D082CCC0E0E43D
:1029E00093A36006122A6D1470FAE493A360061292
:1029F0002BE21470FAD0E0FCE493A3C0E0E493C0AF
:102A0000E022C0E074F212264C758900C2C590190C
:102A1000F3E0700E7A007B109005E2E0F9123320AB
:102A20008003123C027F01022708CAC0E0E493A39E
:102A3000C582CCC582C583CDC583F0A3C582CCC574
:102A400082C583CDC583DAE5D0E0CA22CAC0E0E002
:102A5000A3C582CCC582C583CDC583F0A3C582CC76
:102A6000C582C583CDC583DAE6D0E0CA22C0E0E4E2
:102A700093A3D39C5010E493A3C39C400AD0E0D00E
:102A8000E0D0E00229F5A3A3A3D0E0227009080852
:102A900008226016181818C6C333C608C633C608FD
:102AA000C633C608C633C6D5E0EA22C008C3E096DE
:102AB000F50808A3E096420808A3E096420808A398
:102AC000E09645087001D3D00822C09FF59FE473BB
:102AD000D09F22D083D082C09FE493C0E074019342
:102AE000C0E0740293F59F2200C0D0251810AF08F3
:102AF000F518500C05198008F51850020519D2AFC9
:102B0000D0D0222518F58210AF08F518400C151901
:102B10008008F51840021519D2AF85198322740474
:102B2000800A74038006740280027401C0E0F40419
:102B3000122B03D0E0122DAC22C0E0C0D0E8C0E0E0
:102B4000A8A8D2AFC2C7E8A2E792AFD0E0F8D0D031
:102B5000D0E032BB0102E722C082C08389828A832F
:102B6000BB0003E08002E493D083D0822260160889
:102B70000808C6C313C618C613C618C613C618C697
:102B800013C6D5E0EA222518F8E43519F9222518EC
:102B9000FAE43519FB222518FCE43519FD22C3E0BF
:102BA000C696F608A3E0C696F608A3E0C696F60811
:102BB000A3E0C696F622251810AF08F518400C15AC
:102BC000198008F51840021519D2AF22BB000EC0BB
:102BD00082C0838A838982F0D083D08222BB0101A4
:102BE000F722C0E0E493A36C7009D0E0D0E0D0E01D
:102BF0000229F5A3A3D0E022E76670100809E76672
:102C0000700A0809E76670040809E76622E0667042
:102C10001008A3E066700A08A3E066700408A3E049
:102C20006622C3E09608A3E09608A3E09608A3E016
:102C300096A2D265D03322C3E697F60809E697F646
:102C40000809E697F60809E697F622C3E493960882
:102C5000740193960874029396087403939622C3A2
:102C6000E096F008A3E096F008A3E096F008A3E051
:102C700096F022E026F008A3E036F008A3E036F054
:102C800008A3E036F022E647F60809E647F6080909
:102C9000E647F60809E647F622E627F60809E6378A
:102CA000F60809E637F60809E637F622E056F60890
:102CB000A3E056F608A3E056F608A3E056F6227005
:102CC0000422600D18C6C333C608C633C6D5E0F467
:102CD0001822E056F008A3E056F008A3E056F008EA
:102CE000A3E056F022E493F608740193F608740208
:102CF00093F608740393F622E026F608A3E036F66E
:102D000008A3E036F608A3E036F622E657F60809EF
:102D1000E657F60809E657F60809E657F622E4C32F
:102D200096F608E496F608E496F608E496F622C3CA
:102D3000E09608A3E09608A3E09608A3E09622C6D2
:102D4000F4C608C6F4C608C6F4C608C6F4C62260AF
:102D50000D08C6A2E713C618C613C6D5E0F322C3F2
:102D6000E7960809E7960809E7960809E7962275A5
:102D7000D00075813F7518D1751904000225E9E06E
:102D8000F608A3E0F608A3E0F608A3E0F622600C3C
:102D900008C6C313C618C613C6D5E0F422E6F00869
:102DA000A3E6F008A3E6F008A3E6F022CAC0E0E636
:102DB000F0A308DAFAD0E0FA22ECF0A3EDF0A3EEEB
:102DC000F0A3EFF022E0FCA3E0FDA3E0FEA3E0FF10
:102DD00022E0FAA3E0FBA3E0FCA3E0FD22E0F8A3DD
:102DE000E0F9A3E0FAA3E0FB22E8F0A3E9F0A3EA0C
:102DF000F0A3EBF022E5C754F84401F5C7790122AE
:102E00002518F582E43519F58322122AD36AA20621
:102E1000122AD3B1A206122AD374A306122AD39C73
:102E2000A306122AD3C2A306122AD3D6A306122AB5
:102E3000D3EBA306122AD3F4A306122AD3B77A003F
:102E4000122AD3E37A00122AD3657D00122AD3BC5A
:102E50007D00122AD3FC7D00122AD3107E00122A94
:102E6000D3297E00122AD31A7F00122AD3CB7F00E7
:102E7000122AD3DF7F00122AD3A8B206122AD3CC9B
:102E8000B206122AD3E5B206122AD317B306122AC3
:102E9000D347B306122AD374B306122AD3D6B30685
:102EA000122AD3E5B306122AD3EFB306122AD3FCB3
:102EB000B306122AD335A406122AD355A406122A21
:102EC000D394A406122AD3AFA406122AD3CEA40602
:102ED000122AD334A506122AD33DA506122AD39A64
:102EE000A506122AD3BEA506122AD37FA606122A49
:102EF000D38CA606122AD39DA606122AD3C8BE06D4
:102F0000122AD3E0BE06122AD30CBF06122AD3E639
:102F10008406122AD3408606122AD34E8606122A27
:102F2000D3618606122AD3768606122AD38B8606AA
:102F3000122AD39E8606122AD3128706122AD37724
:102F40008706122AD3198806122AD3DD8806122A88
:102F5000D3ED8806122AD3FC8806122AD35EBB065C
:102F6000122AD382BB06122AD3AABB06122AD3D2B4
:102F7000BB06122AD3CBA606122AD3F2A606122A21
:102F8000D311A706122AD379A706122AD3BD9E060B
:102F9000122AD3D69E06122AD3E29E06122AD3F60E
:102FA0009E06122AD3149F06122AD31E9F06122AA7
:102FB000D3289F06122AD33B9F06122AD3C89F0606
:102FC000122AD337A006122AD366A006122AD3B437
:102FD000A006122AD303A106122AD31EA106122A82
:102FE000D328A106122AD339A106122AD37CA1061E
:102FF000122AD3A4FF05122AD3C3D005122AD3ED77
:10300000D005122AD30AD105122AD31DD105122ABE
:10301000D333D105122AD391D105122AD3C4D105B5
:10302000122AD3B5D505122AD315D705122AD348AB
:10303000D705122AD392D705122AD3E5D805122A2A
:10304000D30DD905122AD322D905122AD332D90594
:10305000122AD376D905122AD3D1D905122AD3E15F
:10306000D905122AD3B4FE03122AD3CEFE03122AA4
:10307000D3F6FE03122AD30FFF03122AD333FF0322
:10308000122AD351FF03122AD368FF03122AD396C0
:10309000FF03122AD3B1FF03122AD3BAFF01122A67
:1030A000D323FC02122AD333FC02122AD338FD02A6
:1030B000122AD36AFD02122AD390FD02122AD3B338
:1030C000FD02122AD3CAFD02122AD304FE02122ADA
:1030D000D36DFE02122AD3AFFE02122AD3EEFE02F5
:1030E000122AD31FFF02122AD356FF02122AD3310B
:1030F0009106122AD3969106122AD33C9206122ADE
:10310000D3739206122AD3A49305122AD33B9405B3
:10311000122AD3689605122AD3539905122AD3E1AD
:103120009A05122AD34D9B05122AD39C9E05122A7A
:10313000D3E79F05122AD361B506122AD3ACB50690
:10314000122AD39FF903122AD345FC03122AD3EA89
:10315000FC03122AD316FD03122AD344FD03122ABC
:10316000D379FD03122AD3A1FD03122AD301FE0352
:10317000122AD302BB05122AD36ABF05122AD352E0
:10318000C105122AD37BC205122AD35BC305122ABA
:10319000D3FEC405122AD3CAC505122AD31EC605FA
:1031A000122AD37EAB06122AD388AB06122AD3A9E1
:1031B000AB06122AD3ADF104122AD3ADF604122ABB
:1031C000D31BF804122AD3D7F904122AD352FA04D3
:1031D000122AD3F1FA04122AD3EAFB04122AD31CCE
:1031E000FD04122AD334FE04122AD314FF04122A37
:1031F000D325BA04122AD35DBA04122AD361C404B7
:10320000122AD342C504122AD38EC604122AD3D757
:10321000C704122AD38DC804122AD361C904122A02
:10322000D348CA04122AD330CB04122AD3D2CB04F7
:10323000122AD3FCCB04122AD3ACCD04122AD31CFD
:10324000CE04122AD335CE04122AD38CCF04122AEC
:10325000D33DD004122AD3BFD004122AD36BD10499
:10326000122AD3DBD104122AD377D204122AD3F341
:10327000D204122AD311D304122AD313D404122A4B
:10328000D3C9D404122AD36FD504122AD33AB10673
:10329000122AD364B106122AD378B206122AD37B3B
:1032A000B206122AD396BC06122AD3D8BC06122A1A
:1032B000D31ABD06122AD32ABD06122AD3CFF0058F
:1032C000122AD30DF105122AD376F105122AD393CF
:1032D000F105122AD3ACF105122AD35EF205122AA7
:1032E000D367F205122AD3ACF205122AD3E2F20513
:1032F000122AD3F9F205122AD36BF305122AD3F856
:10330000F305122AD32EF405122AD385F405122AC6
:10331000D3E9F405122AD30CF505122AD370F5056A
:10332000122AD3CCF505122AD307F605122AD33C6C
:10333000F605122AD34EF605122AD360F605122A94
:10334000D398F605122AD3E4F605122AD322F705FC
:10335000122AD34EF705122AD38EF805122AD3B1BA
:10336000F805122AD3C2F805122AD3B7FA05122A91
:10337000D3D7FA05122AD33DA906122AD373A90678
:10338000122AD3BBA906122AD317AB06122AD300DE
:103390008005122AD3318105122AD36B8105122AA6
:1033A000D32A8305122AD3548305122AD3E1850533
:1033B000122AD3218605122AD3B88705122AD34BA5
:1033C0008805122AD3A38805122AD3468905122A12
:1033D000D37E8905122AD3C08905122AD32F8B05E3
:1033E000122AD3818C05122AD3A48E05122AD3D295
:1033F0008E05122AD3F98E05122AD3028F05122ABE
:10340000D3528F05122AD3E48F05122AD3D4920502
:10341000122AD3579305122AD34EBE06122AD3641A
:10342000BE06122AD36EBE06122AD3358906122A88
:10343000D34B8906122AD3F08906122AD32F8A0683
:10344000122AD34C8A06122AD37D8A06122AD3CA9C
:103450008A06122AD3FD8A06122AD3388B06122A2C
:10346000D3248D06122AD395B706122AD3EAB706BB
:10347000122AD335B806122AD382B606122AD3F4FA
:10348000B606122AD332B706122AD373B706122A07
:10349000D3D7F701122AD3DDF701122AD31DF80181
:1034A000122AD30FFA01122AD33FFA01122AD3AEFD
:1034B000FA01122AD37CFB01122AD3BDFB01122A86
:1034C000D3EBFB01122AD375FC01122AD38CFC0129
:1034D000122AD399FC01122AD3A3FC01122AD33F4A
:1034E000FE01122AD334FF01122AD37DFF01122AD2
:1034F000D311DA05122AD327DA05122AD3BADA054C
:10350000122AD3E6DB05122AD3DBDC05122AD37894
:10351000DD05122AD3B8DD05122AD336DE05122ABC
:10352000D393DE05122AD3A3DE05122AD3CADE0501
:10353000122AD31DDF05122AD38EE005122AD39357
:10354000E005122AD3B3E005122AD3CEBD06122A13
:10355000D3FCBD06122AD331BE06122AD333BE06CF
:10356000122AD335BE06122AD346BE06122AD348E3
:10357000BE06122AD34BBE06122AD3ABAF06122ABE
:10358000D319B006122AD33BB006122AD373B00661
:10359000122AD3A9B006122AD3A59B06122AD3EC6D
:1035A0009B06122AD30F9C06122AD3429E06122A89
:1035B000D35C9E06122AD3879E06122AD3AEFF0240
:1035C000122AD381E205122AD35AE305122AD340E4
:1035D000E405122AD351E405122AD362E405122A23
:1035E000D3AEE405122AD3A2E605122AD3F6E705E4
:1035F000122AD326E805122AD3EDE805122AD34B66
:10360000E905122AD3FFDA02122AD35ADB02122A60
:10361000D301DC02122AD376DD02122AD350DE0255
:10362000122AD30DDF02122AD324DF02122AD37307
:10363000DF02122AD3D7DF02122AD327E002122A8E
:10364000D33AE002122AD39BE002122AD3F4E0021A
:10365000122AD30CE102122AD3A0E302122AD3A425
:10366000E402122AD3DFE402122AD333E502122A3B
:10367000D3D0E702122AD316E802122AD389E8022D
:10368000122AD3D3E802122AD3A7E902122AD3EAD4
:10369000E902122AD304EA02122AD34BEA02122ABE
:1036A000D36BEA02122AD310EB02122AD3F4EB02F4
:1036B000122AD3FFEB02122AD34DEC02122AD3A214
:1036C000EC02122AD3E9EC02122AD34DEE02122A9E
:1036D000D371EE02122AD3F6F002122AD32DF10290
:1036E000122AD335F202122AD359F202122AD3C86F
:1036F000F202122AD38BF302122AD3C6F302122A41
:10370000D32CF402122AD341F502122AD389F502EE
:10371000122AD393F502122AD396F502122AD3A0C5
:10372000F502122AD3B3F502122AD33CF602122A6A
:10373000D365F602122AD378F602122AD3A4F6022F
:10374000122AD3CBF602122AD3EFF602122AD3683A
:10375000F702122AD3DAF702122AD311F802122A38
:10376000D31BF802122AD34AF802122AD360F802B5
:10377000122AD37BF802122AD3A9F802122AD3C93B
:10378000F802122AD312F902122AD34DF902122A90
:10379000D354FA02122AD3B2FB02122AD3C8FB0274
:1037A000122AD3DFFB02122AD3F1FB02122AD3A57D
:1037B000B906122AD3B6B906122AD33FBA06122A7C
:1037C000D3F37F00122AD3C4E905122AD313EA05E2
:1037D000122AD3B3EB05122AD387ED05122AD3C9D7
:1037E000ED05122AD394EE05122AD39CEF05122A76
:1037F000D3BEEF05122AD31AF005122AD39BF00587
:10380000122AD3715000122AD3935000122AD3EBFC
:103810005100122AD3345200122AD3AA5200122A7B
:10382000D3285300122AD38D5300122AD3CF53002A
:10383000122AD33E5400122AD3E95400122AD3612B
:103840005500122AD3A65500122AD3B55900122AC0
:10385000D3BC5B00122AD3EF5B00122AD3415C0079
:10386000122AD3445F00122AD3C05F00122AD36EFB
:103870006100122AD3A06200122AD3B86300122A70
:10388000D33A6400122AD31A6500122AD385650040
:10389000122AD3996500122AD37B6600122AD3AB71
:1038A0006700122AD3C66900122AD3BF6B00122AFE
:1038B000D3A26C00122AD3386F00122AD3D96F001A
:1038C000122AD3D97000122AD33B7400122AD34B88
:1038D0007400122AD3917500122AD32E7600122A70
:1038E000D3587700122AD3E97700122AD316790029
:1038F000122AD35B7900122AD3EF7900122AD31649
:10390000D604122AD3B6D604122AD320D704122AF8
:10391000D339D704122AD3C8D704122AD30CD80417
:10392000122AD32BD904122AD367D904122AD3DA44
:10393000D904122AD325DA04122AD384DA04122AEB
:10394000D32EDB04122AD317DE04122AD334DF0469
:10395000122AD3B1DF04122AD372E104122AD3123D
:10396000E204122AD3B1E204122AD314E304122A85
:10397000D389E304122AD398E404122AD379E50404
:10398000122AD3AFE504122AD3E2E504122AD39611
:10399000E604122AD3C2E604122AD33DE704122A0F
:1039A000D3C0E804122AD33BEA04122AD390EB04D2
:1039B000122AD303ED04122AD30FEE04122AD3B62F
:1039C000EE04122AD324EF04122AD33CF004122A64
:1039D000D3ACDA03122AD317DB03122AD35FDB033B
:1039E000122AD3A3DB03122AD30DDC03122AD356E7
:1039F000DC03122AD391DC03122AD32BDD03122A13
:103A0000D385DD03122AD3DFDE03122AD368DF0356
:103A1000122AD392DF03122AD397E003122AD3A6E5
:103A2000E103122AD3D8E103122AD3C8E203122AEF
:103A3000D3D9E203122AD3F1E203122AD3F1E3032A
:103A4000122AD30EE403122AD3D3E403122AD3FD9D
:103A5000E403122AD314E503122AD33AE503122A07
:103A6000D371E503122AD391E503122AD3B8E503F3
:103A7000122AD3D0E503122AD3AAE603122AD302CC
:103A8000E703122AD378E803122AD307E903122A9C
:103A9000D32BE903122AD342E903122AD30DEA03F6
:103AA000122AD3B0EA03122AD3D6EA03122AD30683
:103AB000EC03122AD325EC03122AD3A6EC03122A14
:103AC000D313ED03122AD357ED03122AD3E5ED03E6
:103AD000122AD350EE03122AD302EF03122AD3F292
:103AE000F003122AD3CAF103122AD31CF203122ABA
:103AF000D316F303122AD323F403122AD334F50383
:103B0000122AD342F503122AD312F603122AD3B291
:103B1000F603122AD3F6F603122AD30BF703122A5E
:103B2000D30BF803122AD3AEF803122AD306F903F3
:103B3000122AD31A9506122AD3539606122AD3199B
:103B40009706122AD37D9706122AD3F19706122AD6
:103B5000D3318D06122AD34F8D06122AD3938D06A8
:103B6000122AD3B98D06122AD3DF8D06122AD3F773
:103B70008D06122AD3F7BB06122AD3278E06122AE5
:103B8000D3928E06122AD3D48E06122AD3E98E0639
:103B9000122AD3F08F06122AD30B9006122AD314BE
:103BA0009006122AD31D9006122AD3269006122AB6
:103BB000D3309006122AD3AD9006122AD300800685
:103BC000122AD31C8406122AD3388406122AD33D23
:103BD0008406122AD32AAE06122AD3859806122A00
:103BE000D331A206122AD30D9A06122AD3379A0687
:103BF000122AD37D9A06122AD3769B06122AD3065E
:103C0000B406122AD353BF06122AD37FBF06122A44
:103C1000D3008002122AD3578002122AD3C3800213
:103C2000122AD34F8102122AD3058202122AD34DBF
:103C30008202122AD3668202122AD3898202122AAF
:103C4000D3AB8202122AD3E98202122AD33883022A
:103C5000122AD3638302122AD3C18302122AD368A1
:103C60008402122AD3108502122AD38C8502122ACA
:103C7000D3598602122AD3A08602122AD3EC8602D6
:103C8000122AD3748702122AD3AD8702122AD303D1
:103C90008802122AD31F8802122AD34E8802122ABF
:103CA000D35A8A02122AD3888B02122AD3B48B02E7
:103CB000122AD3E88B02122AD3098C02122AD318B3
:103CC0008C02122AD3238C02122AD3D28C02122AFB
:103CD000D3428D02122AD3CD8D02122AD3D58D0262
:103CE000122AD3428E02122AD37E8E02122AD34483
:103CF0008F02122AD3179002122AD36C9002122A32
:103D0000D30B9102122AD3659102122AD3AA9102EF
:103D1000122AD3439402122AD3869502122AD37010
:103D20009802122AD3549902122AD3389A02122ADC
:103D3000D35D9A02122AD36E9A02122AD3E09A0213
:103D4000122AD3779B02122AD3EB9B02122AD3DBCF
:103D50009C02122AD3009D02122AD3189E02122A14
:103D6000D3369E02122AD3529E02122AD3C59E0235
:103D7000122AD3D49E02122AD35C9F02122AD3594C
:103D8000A002122AD366A002122AD36FA002122A1E
:103D9000D351A202122AD37DA302122AD38DA302E9
:103DA000122AD3C8A402122AD347A502122AD37812
:103DB000A602122AD3B4A602122AD38EA802122A6D
:103DC000D34BAC02122AD35FAC02122AD369AC02E5
:103DD000122AD373AC02122AD37DAC02122AD387E3
:103DE000AC02122AD3A0AC02122AD3AAAC02122A25
:103DF000D321AD02122AD32CAD02122AD35BAD021D
:103E0000122AD383AD02122AD38EAD02122AD3F323
:103E1000AD02122AD3FDAD02122AD308AE02122A35
:103E2000D32CAE02122AD350AE02122AD3C2AE0253
:103E3000122AD30BAF02122AD327AF02122AD39829
:103E4000AF02122AD3E4AF02122AD32DB002122AF3
:103E5000D36BB002122AD3ECB002122AD393B10270
:103E6000122AD358B302122AD3BDB302122AD3EBBB
:103E7000B402122AD311B502122AD359B602122A59
:103E8000D393B902122AD391BB02122AD35CBD028A
:103E9000122AD3F5BD02122AD3F6BF02122AD3ABDF
:103EA000C002122AD3E4C002122AD354C102122A39
:103EB000D35EC102122AD387C302122AD38AC40254
:103EC000122AD3C7C502122AD31EC602122AD3C988
:103ED000C602122AD379C802122AD3C6C902122AEC
:103EE000D3E6C902122AD33BCA02122AD33CCB0220
:103EF000122AD364CB02122AD3C3CB02122AD3BB19
:103F0000CC02122AD332CD02122AD345CE02122A73
:103F1000D3B3CE02122AD3B2CF02122AD30CD202CA
:103F2000122AD335D202122AD39BD302122AD31DCE
:103F3000D502122AD374D502122AD322D602122A0B
:103F4000D3C7D602122AD32AD702122AD3E8D7021D
:103F5000122AD37AD802122AD3D9D802122AD31B12
:103F6000D902122AD34CD902122AD3A3DA02122A76
:103F7000D3008003122AD3328003122AD36B80032A
:103F8000122AD3348203122AD3788203122AD34E00
:103F90008303122AD3AD8303122AD3C38403122AC4
:103FA000D30F8503122AD39D8703122AD3818A0354
:103FB000122AD3C88B03122AD3608C03122AD36C23
:103FC0008C03122AD3B58C03122AD3F78D03122A3D
:103FD000D3ED8E03122AD3178F03122AD36D8F03CA
:103FE000122AD3C68F03122AD3399003122AD36F11
:103FF0009203122AD3F19303122AD3DC9403122AD8
:10400000D3269603122AD35E9803122AD35B9B030E
:10401000122AD36A9B03122AD3FE9B03122AD3A926
:104020009C03122AD3EC9C03122AD3359D03122A37
:10403000D3859D03122AD3E99D03122AD35B9E03E5
:10404000122AD3779E03122AD3A69E03122AD3E5FF
:104050009E03122AD3E09F03122AD38FA003122AB1
:10406000D30CA303122AD33EA403122AD316A5030A
:10407000122AD398A503122AD3CDA903122AD3FC5E
:10408000A903122AD357AA03122AD38AAA03122AEF
:10409000D302AB03122AD335AB03122AD396AB0358
:1040A000122AD3E6AB03122AD3B3AC03122AD36C81
:1040B000AD03122AD330AE03122AD3AAB003122AB8
:1040C000D30CB203122AD35DB303122AD381B403F3
:1040D000122AD384B403122AD3B3B403122AD3AB63
:1040E000B603122AD36AB703122AD399B703122A46
:1040F000D3B7B803122AD37FB903122AD340BB0324
:10410000122AD3B0BB03122AD3E2BB03122AD30272
:10411000BC03122AD371BC03122AD36ABD03122A2C
:10412000D38EBD03122AD301BE03122AD32AC003A1
:10413000122AD389C003122AD3DDC003122AD30C5A
:10414000C303122AD3EFC303122AD377C403122A5C
:10415000D35BC503122AD3E5C503122AD3F9C503DD
:10416000122AD30DC603122AD321C603122AD3352D
:10417000C603122AD362C603122AD392C603122A96
:10418000D34DC803122AD323C903122AD3C7C903A4
:10419000122AD31CCA03122AD37FCA03122AD3C8F5
:1041A000CA03122AD3EFCA03122AD3B7CB03122AA7
:1041B000D35DCC03122AD3E3CD03122AD36ECE03F0
:1041C000122AD3B5CE03122AD327CF03122AD37CC7
:1041D000D003122AD325D103122AD359D103122A8C
:1041E000D371D103122AD314D203122AD390D40349
:1041F000122AD338D603122AD356D603122AD374DE
:10420000D603122AD340D703122AD38EDA03122AF6
:10421000D3948101122AD3D68101122AD343870174
:10422000122AD38F8701122AD3D58701122AD326C7
:104230008901122AD38B8901122AD3CF8901122A2C
:10424000D3358B01122AD3908E01122AD3C38F014A
:10425000122AD3529B01122AD3E29B01122AD3CCF9
:104260009E01122AD331A001122AD394A001122A4E
:10427000D3B0A101122AD31AA301122AD3F9A301A0
:10428000122AD367A601122AD3F9A701122AD38AC8
:10429000A801122AD3A9A901122AD336AA01122AE7
:1042A000D340AA01122AD368AA01122AD30BAB0168
:1042B000122AD3F6AB01122AD3BEAC01122AD34B79
:1042C000AD01122AD361AD01122AD37EAD01122AAB
:1042D000D3A7AD01122AD3D4AD01122AD318B0014D
:1042E000122AD3EBB001122AD32FB101122AD3B173
:1042F000B101122AD352B201122AD384B201122A76
:10430000D3CBB201122AD3FEB201122AD342B30197
:10431000122AD391B301122AD396B301122AD3F2EF
:10432000B301122AD336B401122AD320B501122ABE
:10433000D385B501122AD3E3B501122AD362B6019F
:10434000122AD3DAB901122AD3DDBA01122AD373A1
:10435000BC01122AD3B6BF01122AD358C001122AB7
:10436000D3A1C201122AD35CC301122AD39BC30179
:10437000122AD35FC501122AD37CC501122AD38524
:10438000C501122AD38EC501122AD399C501122A5A
:10439000D3B8C501122AD3DCC701122AD339C80108
:1043A000122AD343C801122AD34DC801122AD3B00E
:1043B000C801122AD30CC901122AD319CA01122A20
:1043C000D37ACA01122AD38BCB01122AD3D4CB01C0
:1043D000122AD39ECC01122AD3B5CD01122AD37949
:1043E000CE01122AD3C5CF01122AD3C9D001122A75
:1043F000D3C2D101122AD3DAD101122AD311D201A8
:10440000122AD31BD201122AD325D201122AD33069
:10441000D201122AD34ED201122AD396D201122AE5
:10442000D3F4D201122AD31BD301122AD32DD301E4
:10443000122AD3D6D301122AD30FD401122AD34081
:10444000D501122AD39DD501122AD38ED601122A64
:10445000D3C4D601122AD334D701122AD3B0D7013C
:10446000122AD331D901122AD358DA01122AD31AC7
:10447000DB01122AD3E8DB01122AD36DDC01122AF8
:10448000D31CDD01122AD304DE01122AD39DDE01E2
:10449000122AD379DF01122AD3E1DF01122AD3A035
:1044A000E001122AD3FCE001122AD360E101122AB2
:1044B000D326E201122AD349E201122AD303E301EF
:1044C000122AD325E301122AD386E301122AD3B696
:1044D000E501122AD3AFE601122AD35BE701122AC3
:1044E000D378E901122AD3C1E901122AD30CEA01D7
:1044F000122AD368EA01122AD3C6EA01122AD3EAA1
:10450000EA01122AD30EEB01122AD343EB01122A3D
:10451000D36BEB01122AD3B0EB01122AD30EEC01BC
:10452000122AD367EC01122AD361ED01122AD30DAE
:10453000EF01122AD352EF01122AD37BEF01122A84
:10454000D304F001122AD377F001122AD385F001A7
:10455000122AD3A9F001122AD3FFF001122AD31A8A
:10456000F101122AD3D5F101122AD301F201122A44
:10457000D344F201122AD3A7F201122AD3B7F401CD
:10458000122AD3E3F401122AD39EF501122AD38210
:10459000F601122AD316F701122AD343C605122AAE
:1045A000D37BC605122AD39CC605122AD3DEC605C4
:1045B000122AD342C705122AD34CC705122AD35C4C
:1045C000C705122AD393C705122AD33CCB05122A5A
:1045D000D304CD05122AD3E8CE05122AD38ACF05FB
:1045E000122AD314D005122AD3508004122AD3F9E8
:1045F0008004122AD3D88104122AD3E48204122A16
:10460000D3048304122AD3268404122AD3D6850421
:10461000122AD3438604122AD3148704122AD31AE7
:104620008804122AD3928804122AD3CD8804122A2D
:10463000D3268904122AD3618904122AD3AA8904B1
:10464000122AD33E8A04122AD3D48A04122AD3A966
:104650008B04122AD37C8C04122AD30A8D04122ACA
:10466000D3308D04122AD35D8D04122AD38E8D048B
:10467000122AD35B8E04122AD36B8E04122AD3BE65
:104680008E04122AD3CB8E04122AD3D88E04122A77
:10469000D3E18E04122AD3458F04122AD3A38F04A8
:1046A000122AD3EE8F04122AD3099004122AD3308F
:1046B0009004122AD34D9004122AD3599004122A3E
:1046C000D3EA9104122AD3039204122AD37F9204CC
:1046D000122AD3929204122AD3A29204122AD34607
:1046E0009304122AD3B29404122AD3C59504122A31
:1046F000D3659604122AD36F9604122AD3EE960439
:10470000122AD3FF9604122AD33E9704122AD36C9E
:104710009704122AD3399804122AD3909804122AA3
:10472000D3C99804122AD31F9904122AD33D99049D
:10473000122AD38B9904122AD3569A04122AD3A48C
:104740009A04122AD3F19A04122AD3749B04122ACF
:10475000D39E9B04122AD3D49B04122AD3E39B0436
:10476000122AD3429C04122AD3BA9C04122AD3FBE5
:104770009C04122AD34B9D04122AD3769D04122A3C
:10478000D3909D04122AD3AA9D04122AD37F9E049B
:10479000122AD3899E04122AD3C49E04122AD3D487
:1047A0009E04122AD3DD9E04122AD32E9F04122ABD
:1047B000D3429F04122AD364A004122AD377A00400
:1047C000122AD38CA004122AD31FA104122AD39335
:1047D000A104122AD338A204122AD343A204122A13
:1047E000D3A6A304122AD3C2A304122AD30EA4046C
:1047F000122AD37CA404122AD3AEA404122AD3C84A
:10480000A404122AD328A504122AD3C7A504122A65
:10481000D312A604122AD365A804122AD3FDA80431
:10482000122AD374A904122AD3D1AB04122AD3E9D1
:10483000AB04122AD3ECAB04122AD3F8AB04122A2D
:10484000D30CAC04122AD314AC04122AD34BAC04FC
:10485000122AD33FAD04122AD3C9AD04122AD34B76
:10486000AE04122AD3CBAE04122AD3A2AF04122A6A
:10487000D3C4AF04122AD35DB004122AD3BAB00451
:10488000122AD3BDB004122AD32CB104122AD37831
:10489000B204122AD38BB304122AD316B404122AF8
:1048A000D329B504122AD3F0B504122AD321B604B1
:1048B000122AD347B604122AD350B604122AD37F41
:1048C000B604122AD32FB704122AD3DFB704122A50
:1048D000D352B804122AD3F5B804122AD368B90403
:1048E000122AD3A7B904122AD3F0B904122AD38CFE
:1048F000B906122AD326B906122AD3A3B806122A59
:10490000D3C4BD06122AD35CBD06122AD344BD0609
:10491000122AD334BD06122AD3E4FF03122AD3F697
:104920007F00122AD33FBB06122AD3A1BA06122A4D
:10493000D390BA06122AD342AD05122AD38FAC0502
:10494000122AD3C3AB05122AD31FAA05122AD3E811
:10495000A905122AD3BAA905122AD367A905122AD2
:10496000D3BEA805122AD326A805122AD300A8056B
:10497000122AD3B5A705122AD389A705122AD3FD77
:10498000A605122AD39CA605122AD387A106122AAD
:10499000D357A605122AD30FBF06122AD337FF0515
:1049A000122AD378FD05122AD3A4FC05122AD32B90
:1049B000FC05122AD31DFC05122AD383BC06122A39
:1049C000D372A505122AD390A405122AD338A405C0
:1049D000122AD3A8A305122AD333BC06122AD36302
:1049E000A305122AD347A305122AD3F5A105122A3B
:1049F000D3B7A105122AD39B9806122AD391A105F9
:104A0000122AD3FABB06122AD315A105122AD3CB38
:104A1000BA05122AD384BA05122AD323BA05122A58
:104A2000D3F6B905122AD3CCB905122AD398B90501
:104A3000122AD370B905122AD310B905122AD3FA53
:104A4000B805122AD3BFB805122AD336B805122AE0
:104A5000D37DB405122AD33BB205122AD300B00588
:104A6000122AD382AF05122AD323AE05122AD333DA
:104A7000AF05122AD3C0AE05122AD381AE05122A81
:104A8000D30F8E0600000080FBE4738F000100E767
:104A90001987000100E61935000400A31C25000257
:104AA00000A71C26000200A91C27000200AB1C283E
:104AB000000100B51C29000100B61C84000400B7E9
:104AC0001C86000100BB1C2A000100BC1C2B00013D
:104AD00000BD1C2C000100C11C2D000800C8192EAF
:104AE000000100C21C2F000100C31C30000100C4E3
:104AF0001C31000100C51C32000100D01933000137
:104B000000D11934000100C61C36000100D219384A
:104B1000000100C71C39000100C01C83000200DB3B
:104B20001C63000100E31964000100BE1C65000164
:104B300000BF1C6D000100E41971000800C0196677
:104B4000000100DA1C43000100CB1C44000200CC31
:104B50001C45000100CE1C46000200CF1C47000887
:104B600000DB1948000100D11C4B000100D21C04DD
:104B7000000100DD1CA1000100E01C37000100DF86
:104B80001C88000100DE1C3C000100D3193D00011F
:104B900000C81C49000200D31C67000100E5194D44
:104BA000000200D51C4E000100D71C4F000200D8A7
:104BB0001C3E000100DA1951000100D41952000115
:104BC00000C91C53000100CA1C54000100D5190083
:104BD0000000000000000136360101000102010062
:104BE000010301000104010606050200000701009F
:104BF000340801000F090401010D0100FF0E080037
:104C00000017020000190100FF1A0100011B01003A
:104C1000FE1C0100081D0200001F01000120010010
:104C200001210200002301000F24020000260100E0
:104C30000127010008280200FF2A0100072B0102BA
:104C4000402C0100002D0100012E0100012F010068
:104C5000FF30010B1D310800003A0100083B010044
:104C60000F3C0100013D0100FF3E04000042040032
:104C700000460400004A0400004E040000520400F4
:104C800000560400005A04000001037103010301EF
:104C900003010301030103220302030103100300C4
:104CA00003000300030003000300030003420300AA
:104CB0000324030603000300030403120325032354
:104CC0000325032303040304030003000300034438
:104CD0000300030003230300036503210035038160
:104CE000030003050300030003000300032503235F
:104CF00003010171010101010111010101310101F2
:104D00000101018001100161013B00140063017386
:104D1000017201620143010001130106013D0135E9
:104D2000000401120100010001000100010401045E
:104D300001330133013C014401320136000001001E
:104D40000165010001350081010001050182018337
:104D500001000103027102300160021102700201C0
:104D600002020202028002100261023A0041006364
:104D70000273027202620243020002130238000050
:104D800002000204021202000200020002000204F9
:104D9000020402370037003C0244020002390000DE
:104DA0000200026502000235028102000205028251
:104DB00002830200020304710402046004110470FF
:104DC0000402040204010402041004610400041437
:104DD00004630473047204620443040004130406AD
:104DE000040004000404041204000400040004008D
:104DF000045104640000040004000444040004009E
:104E00000400040004650400043504810464000502
:104E100004000483040004030071003001600011E9
:104E20000070003102200350048000100061000077
:104E3000001400630073007200620043000000135E
:104E40000006000000000004001200000000000046
:104E500000000004000400370037003C024400005A
:104E60000000000000000065000000350081000027
:104E7000000500000083000000360001000600006D
:104E8000000F000000000000000000000000000310
:104E9000FFFF00000403FFFF0000FFFF0FF401000D
:104EA00005C4040320000100000B00000000000006
:104EB000000003010F0000000000000000000000DF
:104EC00000000000000000000000000000000000E2
:104ED0000000000000000000003E3913009C381F55
:104EE00000A2381F80A83801003E39020024380390
:104EF000002A3804003038050036380600423830C1
:104F000000603831005A3832006C3833007238355E
:104F100000783834007E3836008438110090381418
:104F200000963815005438FFFF00000A0000000208
:104F30000000000400000008000000100000002035
:104F400000000040000000800000000001000000A0
:104F50000200000004000000080000001000000033
:104F600020000000400000015642068C42088642A4
:104F70000BA44210203F0AB642025C42057A420767
:104F800062420C3E420D4A4264F83CFF000007ECCE
:104F9000FDFDFDECDCDCCCBCACAC9C9C8C7C7C6C6E
:104FA0006C5C5C5C4C4C3C3C2C2C1C1C03EAF5E51A
:104FB000D5D5C5B5A5959585857575656555554551
:104FC000453535252515150500160F00000B150B69
:104FD000020002220F3300000E5A696742656541E4
:104FE0006C6C69616E6365303901030507090B0D4F
:104FF0000F00020406080A0C0D00011916181616F7
:1050000018230300303017181921301B1D1F3030B2
:105010003016181920231A1C1E3000393D3F373C2A
:105020003C362C442D00034A49434E181A250502EC
:105030000C0E020B040B0A0708000F020402010108
:1050400001010902E803000000BE040A0000E803B1
:105050000E0000007F001E1E050303000404100A5A
:105060000C10080C280009040903010C050810089D
:10507000FFC082C08390193EE4F0A3F07C177D1A34
:105080007AAB7B18123488123D28123F6E123D2EE7
:1050900002659274F512251774F5122BB6E9FF8A92
:1050A00008EBFE8C09E9705B74026A703E790812A5
:1050B0003794750A00780A122B2AE509F50A780A4E
:1050C000122B2AEEF50A780A122B2A9018C71229F9
:1050D0004B901CBBE0F97CDB7D19901CDB12643625
:1050E000123D527407122AE80251BA74016A600331
:1050F0000251BF79081237947B00EEFAF9123D9401
:105100000251BA74016F600874026F60030251BFEC
:10511000EA600574036A70477902123794901CBBE9
:10512000E0F99018C7122DD1123D40E9F89018D639
:10513000E0A2E34010E9700D901942E004F064042D
:1051400070031251D9740365087071901943E0F926
:10515000740129F0E9C3940540621251D9805D744D
:10516000016A705B74016F790A702E1237947401B2
:10517000122E00E4F07402122E007403F004122EBA
:1051800000E4F0A3F0A3F0A3F07408122E00E4F002
:10519000AA18AB191242688036123794901CB112CB
:1051A000294B7A007B20125B8B122AE8901CBBE013
:1051B000F99018C7122DD1123D76E9F8E8601090E9
:1051C000811712294B7A017B00125B8B122AE8743B
:1051D0000B122AE87F030228439018C7E4F0A37457
:1051E000F8F0A374FFF0A37407F02274F6122517E9
:1051F000E9FFEAFE7AD1F91232FC8A828B83E582DA
:105200004583702A7A027B001232DEEA4B700E7AF6
:10521000107B009018CBE0F912332080148A828B27
:105220008374D1F0EFA3F0EEF91232EA8003EFA31A
:10523000F002543974F712251789089004D11277B7
:1052400039FF901C9EE0F47003A3E0F470319005E8
:10525000E2E0901C9EF0A3E4F080248E828F83A372
:1052600012629A600F8E828F83A3A3126297FAA9AB
:105270000812380C8E828F83126160E8FEE9FFEE1F
:105280004F70D8901C9EE0F47003A3E0F4600A9085
:105290001C9EE0FAA90812380C1243769018951259
:1052A00059AF1243707F0102284374F01225178909
:1052B0000B8C0C7509007508007410122E00126119
:1052C000607412122E001269AAFD8047125374F501
:1052D0000EA3E0F50FAE08EE2EFEE433FFEA2EF546
:1052E00082EB126641650E7004A3E0650F7019AE83
:1052F00009EE2EFEE433FFEC2EF582ED3FF583E55B
:105300000EF0A3E50FF00509050AE50AC3950C4068
:10531000BB0508E508C3950B5005750A0080EBA98D
:105320000980007F0802284374F4122517890B7D39
:1053300000740C122E0012616080010DEDC3950BFC
:10534000502E750A008002050AE50AC39C50ECED58
:1053500025E0FEE433FFEA2EF582EB3F126BA31249
:10536000537465087004A3E0650970DB790180025D
:1053700079008014AE0AEE2EFEE433FFE82EF582AB
:10538000E9125B7522122AE87F0402284374F612A0
:1053900025171254237003A3E06D70177508D47598
:1053A00009187808122B26EEFA1239447402122AD0
:1053B000E8801A7508027509807808122B268A0879
:1053C00089097808122B26125411122AE8806A746F
:1053D000F61225171254237003A3E06D7017750899
:1053E000E17509187808122B26EEFA12394A740270
:1053F000122AE8801A7508037509807808122B268E
:105400008A0889097808122B26125411122AE8807A
:1054100028EE240E125B72FD7C80126649123968F8
:10542000740422EAFEEBFF126660FCE439FD90187A
:1054300095E06C227402122AE87F0202284374F677
:1054400012251774FE122BB6EAFEEBFF8518828533
:105450001983E41254E212679BFBECFA8882898379
:10546000A3A3E0F9750900750800600574FF697071
:1054700005750882803E901895E06A7003A3E06B82
:10548000701BAA18AB19124A36E9FA8518828519D9
:10549000831269B570037508838A0980179019E62D
:1054A000E06004640170057508818008E0640270A2
:1054B000037508808518828519831269AAFDA908D9
:1054C000EEFAEFFB123950E5096014851882851950
:1054D000831269B56009851882851983126FD2021B
:1054E0005434F0A3F01276122274F2122517EAFE59
:1054F000EBFF75080075090012665CF50AE439F5E2
:105500000B124376EA650A7003EB650B7012124AC0
:1055100024E914F50879017A0A7B19124A1E8003DE
:10552000750980EE240E12663EF50C780C122B2ABB
:10553000750C0A750D19780C122B267808122B2A77
:10554000780A122B26E509F5087808122B2A12642E
:105550002512663EF97A057B801239567407027867
:105560007774F6122517E9FF7E0080328A828B83DA
:10557000E0F508A3E0F8E4C8F9E50828E439F509FE
:10558000EE25E0F8E433F9EC28F582ED39F583E512
:1055900008F0A3E509F0EA2402FA50010B0EEEC36D
:1055A0009F40C902543974E812251774FC122BB6B7
:1055B0008A168B177511007402122E00E4F0A312E4
:1055C00067A31254E23517125B83F50B850A82F547
:1055D000831279DDFEE439FF850A82850B83A3A35C
:1055E000E0FA850A82850B83A3A3A3E0F9EAF50814
:1055F000E439F509EEFAEFFB124412E96401601692
:10560000EEFAEFFB124412E97038901895E06E70D4
:1056100003A3E06F602C127379122B2AE4F508F5CE
:10562000097808122B267808122B2A90189512292F
:10563000537508807808122B2A12597D122AE80225
:10564000595C850A82850B83A3A3A3A3E0F510E52B
:105650000A2405F50A5002050BE51060281278EEC1
:105660007402122E001259AF7402122E001269B584
:1056700060137402122E00125973A91012383C8A5A
:105680000A8B0B8003751000850A82850B831278C4
:105690008860241278EE851882851983EAF0A3EBDE
:1056A0001269BBE849601085188285198312597305
:1056B000A90F12383C8003750F009004D1805285E9
:1056C0000A82850B83A3A3A3A3A3A3A3A3E4F0A3AC
:1056D000F0AA0AAB0B851482851583A3A3E0F81208
:1056E0006297F91232EA851282851383E0C0E0A83E
:1056F00011740A28F582E43419F583D0E0F005111D
:10570000A2005007AA12AB131233868514828515A6
:1057100083E0F514A3E0F515E51445157003025870
:10572000D9851482851583A312629A60DE8514825E
:10573000851583A3A3A3A3A3A3A3A3E0A2E050CBB7
:10574000851482851583A3A3A3A31269B58514824A
:10575000851583A3A3601E12629BFA7901851482CA
:10576000851583A3A3A3A3125966124A898A128BB3
:1057700013D200800F125966A3A3A3E0F512A3E091
:10578000F513C200E512451370030257008512821B
:10579000851383A3E065087004A3E06509600F74B6
:1057A000FF6508700474FF650960030257008512E5
:1057B00082851383A3A3A3A3A3A3A31229538512B2
:1057C00082851383A3A3A3A3A3A3E0FC7404122ED6
:1057D00000126436A91012381E7402122AE8E97009
:1057E0003C851282851383A3A3A3A3A3A3A3A3A38E
:1057F000A3122953851282851383A3A3A3A3A3A372
:10580000A3A3A3E0FC7402122E00126436A90F12A7
:10581000381E7402122AE8E97003025700E50F25CA
:1058200010C333240AFA7B001232DE8A0A8B0BEA99
:105830004B70030256E68A828B8374D2126BAD8A58
:10584000828B83A3A3E8F0A3E9127857A3E5101293
:1058500079E7E50FF0E510602CEA240AFAE4350B4D
:10586000FB850A82850B831259AA7402122E00123C
:10587000599D122B22AC10EC2CFCE433FD1270ABC2
:10588000122AE8800D8A828B83A3A3A3A3A3E4F04A
:10589000A3F0E50F70030256BFA810E828F8E43320
:1058A000F9E50A28F8E50B39F9E8240AFAE439FBA6
:1058B000850A82850B83A3A3A31259AA8518828522
:1058C000198312599D122B22AC0FEC2CFCE433FDF2
:1058D0001270AB122AE80256D1E5116025127379D5
:1058E000122B2A75080A7509197808122B26E5115A
:1058F000F5087808122B2A9018951229537508007C
:105900008029EEFAEFFB124412E9702A1273791221
:105910002B2A75080A7509197808122B26750800B4
:105920007808122B2A9018951229537808122B2ADE
:1059300012597D122AE87402122E001269B560080D
:105940007402122E00126FD2851882851983126993
:10595000B56009851882851983126FD27404122AE2
:10596000E87F1002284312596A22E0F8A3E0F58389
:10597000888222E0FCA3E0FDAA0AAB0B22E51624F4
:1059800002FCE43517FDE516240FF582E43517F522
:1059900083E0F97A067B80123956740722E0F50C11
:1059A000A3E0F50D750E00780C22A3A3A3A3A3EA30
:1059B000F0A3EBF02274F112251774F4122BB68ABF
:1059C000088B09ECFEEDFF740B122E007403F0122D
:1059D0002B8E12348812650E7403122B8E123482B1
:1059E000E9600A125B7A6010E06401600B8518823E
:1059F0008519837484025B268E828F83A3A3A3A35D
:105A0000A3A3A3A3E06013F46010125B7A7016EEF8
:105A1000241412663E6003F4700B85188285198386
:105A20007482025B261276FDE064217002A3E060BE
:105A300003025AFD851882851983748CF0125B7AF3
:105A40006003025AE77401122B96EE240BFAE43F2E
:105A5000FB12409AE96003025AE71237828A0A8BE6
:105A60000BEA4B7003025B278E0C8F0D750E0078CE
:105A70000C122B227C157D001270AB122AE88508CF
:105A800082850983A3A3E50A2415FCE4350BFD7484
:105A900009122A4C12732EC0E0E50A241E125B5F25
:105AA000D0E0125FB7C0E0E50A241F125B5FD0E0D0
:105AB000F0E50A2420125B5F7405F0EE240BFE5023
:105AC000010FFAEFFB12495E7D007C007900EEFACF
:105AD000EFFB12390E90811712294B7A007B1012BE
:105AE0005B8B122AE88073125B67122B2A125B967B
:105AF00012407C7401122AE8E9702C8014125B6752
:105B0000122B2A125B961240827401122AE8E97065
:105B10000D851882851983E4F012375280098518A3
:105B2000828519837488F012732EF50A780A122B75
:105B30002A7401122B86880A890B780A122B26E513
:105B400008240CF582E43509125B834480F50B7858
:105B50000A122B261264F0122AE8740C026EC1F5A8
:105B600082E4350BF58322EE2414125B72F50A7879
:105B70000A22F582E43FF583E022EE2413125B72E1
:105B8000640322F583E0F50AA3E0229018CBE0F944
:105B9000123440740422EE240BFCE43FFD8E828F0D
:105BA00083A3A3A3A3A3A3A3A3A31273698E828F2A
:105BB00083A3A3A3A3A3A3A3A3E0F922C082C083CA
:105BC00074F3122BB6851882851983E4F004122E23
:105BD000001259AF7403122E00AA82AB83123C2C20
:105BE000AA18AB19123C68740D122AE80265927467
:105BF000F6122517126637F8A3E0125C32F89018F7
:105C0000DCE058F508A3E059F509E5084509601FEF
:105C10007808122B26901895122953EE240E12663E
:105C20003EFD7C001266451239627404122AE802B5
:105C300054398882F583125C3A22E0FAA3E0F9EA4B
:105C40002274EA12251774DB122BB68A148B157591
:105C5000120075130012760E3515F58312629BF54E
:105C60000EAC18AD197A007B00799C123DA67A041F
:105C70007900123C92EAF50C851882851983E02A96
:105C8000F0F8E50EC3984003025E65E0C3950EF59B
:105C900009C394044003750903E50975F01AA4FAD1
:105CA000ABF01233808A128B13EA4B7003025E68EA
:105CB000750D00AE12AF13850E08025D457C087DA0
:105CC0000079FFEE240AFAE43FFB1232C6850A820D
:105CD000850B83A3A3A3A3E0702D850A82850B8384
:105CE0001269B5700C127542F0EE241812754580D9
:105CF00010125EEDF0901A89E014C0E0125ED0D070
:105D0000E0125F20E48034901A89E004C0E0125E63
:105D1000D0D0E0125F13C39403EE4003025DCE12B5
:105D200076037402125F1364017003025DDBEE24DC
:105D300015125EF0F0EE2416125EF0F0EE241AFE5C
:105D400050010F050DE50DC395094003025E06E500
:105D500008C3950C4003025DE4AA087B00123CE0F6
:105D60008A0A8B0B0508901A76125EF9850A8285DD
:105D70000B83126160125EC8F583E8F0A3E9125F3D
:105D800030850A82850B83A3A3A3A3A3A3A3A3A304
:105D9000A3E0C0E0125EBED0E0F07401122E00E479
:105DA000F0850A82850B831261607402122E00E86E
:105DB0001277477401122B8E123C56E9640160037E
:105DC000025CBD7404122E00125EDE025CCD125E17
:105DD000EE125F1364036003025D2EEE241512754C
:105DE00045025D34E50CC3950E4005750800801D25
:105DF000E50EC3950CF5088014125EEDF0EE241A42
:105E0000FE50010F050DE50DC39509505B740E1290
:105E10002B96AA087B007987123DA60508741812F4
:105E20002E00125EF97410122E00125EDEEE2412A5
:105E3000F8E43FF9740E122E0012643688828983CA
:105E4000EAF0A3EB125F207403125F30741D122E70
:105E500000E0C0E0125EBED0E0127824E8497099FC
:105E60001275428097750900750A00780A122B2A6C
:105E70007812122B267809122B2AE50EF5097809DB
:105E8000122B2A7405122E00E0FD7C00E51412632B
:105E9000B33515FBE5141275333515F583E0F912AA
:105EA000399E7405122AE8E51245136007AA12AB61
:105EB000131233867425122AE87F0E022843EE243B
:105EC00019F582E43FF58322EE2412F582E43F22A5
:105ED000125ED422EE2418F582E43FF58322AC82D0
:105EE000AD83EE240AFAE43FFB12348822EE241438
:105EF000F582E43FF583740122126BBA8E828F83A0
:105F0000E8F0A3E9F07C8A7D1AEE1263B33FFB123E
:105F1000348822F0850A82850B83A3A3A3A3E02201
:105F20001275867402F0EE2416F582E43FF58322A2
:105F3000F0EE2417F582E43FF5837402F0125ED48C
:105F400074FFF02274F612251774F9122BB612762C
:105F50000A3509127A9B851882851983122DE98EDC
:105F6000828F83A3A3A3A3E0C0E07404122E00D009
:105F7000E0127839F87405122E007401F0740612DC
:105F80002E007401F090189FF09018A80412762843
:105F9000FAA3E0FB9018A01259AFE89018A9125F7D
:105FA000B790189EF0AA18AB19123D46E96003128B
:105FB0003D4C7407025436F0E508240F1273362264
:105FC00074F212251774FF122BB67508007E007F3D
:105FD000001242988A0A8B0B126140800805081251
:105FE000614C126160E84970F49019E6E060076462
:105FF0000160030260B8126140800612614C1261B8
:1060000060E849603388828983126436901A76E0AA
:106010006A7003A3E06B600A12614C126436EA4BAB
:1060200070D988828983126160901A76E068700363
:10603000A3E06970030260B87A167B001277BC6037
:1060400077901A761261608A828B83E81277479084
:106050001A6B126C9CF01243FAE98E828F83A3A311
:10606000A3A3A3F0901CBCE08E828F83A3A3A3A361
:10607000A3A3F07C8A7D1AEE240B125EE5AA18AB6E
:10608000197941123B5A851882851983E06008907E
:106090001895126160800478FE79FF8E828F83A349
:1060A000A3A3A3A3A3A3E8127747EE1261543F1260
:1060B00061648E0A8F0B05089018A9E0F8E508C303
:1060C00098500479008027E508C398F9C3940640E6
:1060D0000279057800800DE50A126154350B125BD8
:1060E00083F50B089018A9E0FAE8C39A40E975090E
:1060F000007809122B2A780A122B26E9F50978096B
:10610000122B2A9018A9E0F5097809122B2AAD085C
:106110007C007AA07B1890189EE0F91239987405DB
:10612000122AE89019E6E060046401700BEE4F60FB
:1061300007EEFAEFFB123386123D4C7401027877BA
:106140001242988A0C8B0DA80CA90D22E8126154FA
:1061500039F583222414F582E42285188285198377
:10616000126BBA22F583E50AF0A3E50BF02274F076
:1061700012251774FF122BB68A0A8B0B7E008E0E27
:106180008E0F12760E125B6212629BFFAC18AD1975
:106190007A007B00799D123DA6851882851983E0DF
:1061A000F8EFC3984003026242E0C39FFEC3940B22
:1061B00040027E0AEE75F007A4FAABF01263AB8AD8
:1061C0000E8B0FEA4B6079750C00801A850882856A
:1061D0000983A3A3A3A3A37403F0E5082407F50888
:1061E00050020509050CE50CC39E5056AC08AD09DC
:1061F000E50C2FFAE43400FB798B123DA68508826A
:10620000850983A3A3A3A3A3E01460081460131457
:10621000601F80B8850882850983A3A3A3A3A3E494
:1062200080B7850882850983A3A3A3A3A3740180F3
:10623000A8850882850983A3A3A3A3A374028099D8
:106240007E007508007808122B2A780E122B26EE95
:10625000F5087808122B2AEFF5087808122B2A7413
:1062600005122E00E0FD7C00E50A1263B3350BFB3E
:10627000E50A127533125B62E0F91239A474051253
:106280002AE8E50E450F6007AA0EAB0F123386749D
:1062900001122AE802532312596CA312596AE02210
:1062A00074EE12251774FE122BB68A0C8B0D751026
:1062B0000075110012760E350DF58312629BF50AFA
:1062C000AC18AD197A007B0079A312408812615A8C
:1062D000C3E50A98E4995074851882851983A80A41
:1062E000E0C398FEA3E09400FFC3EE9404EF940093
:1062F00040067E037F008004EE4F6050EEFAEFFB15
:10630000EA75F015A4FAA8F075F015EBA42812634D
:10631000AA8A108B11EA4B6033750B00750E008052
:106320001FAC08AD09A80AE50E28FAE43400FB7991
:10633000A2124088E5082415F50850020509050E4B
:10634000C3E50E9EE49F40D9EEF98005750B8B796D
:10635000007508007808122B2A7810122B26E9F510
:10636000087808122B2AE50AF5087808122B2A74F7
:1063700005122E00E0FDAC0BE50C1263B3350DFBEE
:10638000E50C127533350DF583E0F91239AA740561
:10639000122AE8E51045116007AA10AB11123386E6
:1063A0007402122AE87F0A022843FB1233808A080B
:1063B0008B09222402FAE42274F612251774FF12C4
:1063C0002BB6EAFEEBFF1264111264368A82F58363
:1063D000A3A3A3A3A3A3A3A3E0F9123D6AE985188D
:1063E00082851983F07508007808122B2A7401122F
:1063F0002B86880889097808122B267508357509B7
:10640000807808122B26126419122AE874010254AB
:1064100036EA1276133FF583227901126425FAE4F5
:106420003F12650722EE2402FCE43FFDEE240F221A
:106430008518828519831273692274F412251774E2
:10644000FA122BB612760A12709D127739FFEEFA05
:10645000EFFB123C32E9600F12650EEEFAEFFB1211
:106460003482E96401700A7401122E00E4F0A38002
:10647000097401122E00EEF0A3EF127864F8A2E680
:1064800050087403122E007401F0E8A2E75008745B
:1064900004122E007401F07405122E00E4F00412B0
:1064A0002B8E123D9AE9851882851983F0908147D9
:1064B000122DD11243947A007B001243A07A007B04
:1064C0000012439A750A00780A122B2A7401122BC3
:1064D00086880A890B780A122B26750A34750B8078
:1064E000780A122B261264F0122AE87406025385E9
:1064F0007901E5082402FCE43509FDE508240FFADA
:10650000E4350912650722FB123902740522124391
:10651000708A0A8B0BAC0AAD0B2274F61225177425
:10652000FF122BB6126637F8A3E08882F583E0F5F8
:1065300009A3E0F508A909123D58E98518828519D3
:1065400083F09019E6E0700B740165087005A909E5
:10655000123A64EE240B12663E7027750800780824
:10656000122B2A7401122B86880889097808122BAD
:10657000267508367509807808122B2612641912C0
:106580002AE802640CC082C0839019E6E07003120E
:106590003A6AD083D082022AD074F412251774EF9D
:1065A000122BB6EAFEEBFF12665CF508E439F5093A
:1065B000901895E06A7003A3E0697052A818A919B1
:1065C000880A890B780A122B26750A11750B007838
:1065D0000A122B267C007D007A817B0012340A741B
:1065E00004122AE8E97027750A00780A122B2A7427
:1065F00001122B86880A890B780A122B26AC08AD6B
:106600000912664512395C7403122AE88024750A5F
:1066100011750B80780A122B267808122B26EE248F
:106620000E12663EFD7C84126645123968740412AF
:106630002AE87411025385EAFEEBFFEA2413F5827F
:10664000E4125B752212664922EE2402FAE43FFB53
:10665000EE240FF582E43FF583E0F9221266602212
:10666000EA2413F582E43FF583126F338882F583C1
:10667000E0FAA3E0F8E4C8F9EA282274F112251739
:1066800074EB122BB6EAFEEBFF12760E12679BFA42
:10669000E4CAFBEC2AF508901895E06C7003A3E0BF
:1066A0006B600302674088828983A3A3E094105043
:1066B0000F88828983A3A3E08518828519838008C7
:1066C0008518828519837410F0E0C0E07404122EDE
:1066D00000D0E0127728A982AA83890C8A0D750E52
:1066E00000780C122B227407122E00E0FC7D00743F
:1066F00008122E00AA82AB831270AB122AE874042F
:10670000122B86880A890B780A122B26750A1175B6
:106710000B00780A122B267C007D007A817B001208
:1067200034047404122AE87404122E00E09018D481
:106730006005E0D2E48003E0C2E41267A3E48008CD
:106740008518828519837484F0E0C0E07401122EEC
:1067500000D0E0F07402122E00E508F07403122E4F
:1067600000E508F01267943F127382122B2A74021C
:10677000122B86880889097808122B26750814754B
:1067800009807808122B26790312641B122AE874F8
:1067900015026EC1EE240EF582E4223F12774CFC06
:1067A000A3E022F08518828519832274F61225173A
:1067B00074E0122BB6EAFEEBFF901A78E0640860F2
:1067C00008E06404600302698FAC18AD191238EA5E
:1067D0009019E6E0640270271243707402122E00D2
:1067E000AC82AD83123482E96015126994851882F7
:1067F000851983E0687003A3E069700302698F1252
:1068000045447402122E00AC82AD831264301244EF
:1068100042E96401700302698F7418122B8E1243CF
:10682000827402122E00AC82AD837418122B8E1269
:106830003482E9602D12437C8A088B09A808A909D3
:10684000851882851983E0687003A3E069601312DC
:10685000615A901A6CE81277477A6C7B1A794B125E
:106860003B609019E6E0600464017067126994EE81
:10687000241112663E687003A3E069605674021228
:106880002E00AA82AB83123CBC8B09A909EA49609D
:10689000268A828B83A3A3A3A3E06401600D8A826E
:1068A0008B83A3A3A3A3E06402700C7402122E00D6
:1068B000AA82AB83123CC8901B061269B560149083
:1068C00019DAE06401700C126430901B0712596DE4
:1068D000124A897900126430123EEA901A761269DF
:1068E000AAFD1264301244FC740B122E00E41269EB
:1068F000BB740C122E00E8127747740B122B8E1209
:106900003C56E9603F7C087D0079007418122B8E9C
:106910001232C6740E122E00AC82AD837418122B84
:106920008E123482E9601D7402122E00AC82AD8397
:10693000740E122E00AA82AB83123C2C740B122B05
:106940008E123C687402122E00AC82AD83740E125B
:106950002E00AA82AB83123C2C740B122B8E123C9D
:106960005CE9602B740C122E001261608518828520
:106970001983E0687003A3E069601412615A740C13
:10698000122E00E8127747740B122B8E123C68749B
:10699000200254361243768A088B09A808A90922D6
:1069A000FAE433FB123380901940E0FCA3E022F5B7
:1069B00082E438F583126BBAE84922F085188285A3
:1069C0001983126BBA2274E812251774F7122BB6CA
:1069D0008A168B177F008F088F091238F08A128B66
:1069E00013EA4B7003026B897E00800DEE75F00C8C
:1069F000A4F8126B8E123CC80E851282851383E0B8
:106A0000F8EEC3984003026AC7750CFF750DFF7559
:106A10000EFF750FFFEE75F00CA4F8A9F0126B8E47
:106A2000123CBCEA4B60D18A828B83A3A3A3A3E070
:106A30006401600D8A828B83A3A3A3A3E064027028
:106A4000B7126C6C700C126C96122D7F126C601267
:106A50002B9EEE75F00CA4F8A9F0E51228F582E55E
:106A600013126C87122AAB40837A0E7B001233809C
:106A70008A0A8B0BEE75F00CA4F8A9F0126B96AC99
:106A800082AD831278BE780C122D9DE50A240C127B
:106A90005B5FE4F0A3F0E5084509700E850A1085F8
:106AA0000B118510088511098019E510240CF8E4F4
:106AB0003511F9888212616488828983E0F510A318
:106AC000E0F5110F0269F8EF7003026B827408128F
:106AD0002E007402126BAD851882851983E8127737
:106AE000477E00EF75F00CA4FAABF01233808A0CED
:106AF0008B0DEA4B7003026B82805185081085096B
:106B000011EE75F00CA4F8A9F0E50C28F50AE50DD6
:106B100039F50BAC08AD09AA0AFB127417A3A3A39D
:106B2000A3A3A3A3122DDD850A82850B83A3A3A3B0
:106B3000A3A3A3A3A3122DE90EE510240CF582E470
:106B40003511126BA3AA10AB11123386E508450963
:106B500070A97508007808122B2A75081F7509801E
:106B60007808122B26780C122B26EFF97405122BBD
:106B700096E516240FFAE43517FB1239387405121E
:106B80002AE8AA12AB13123386740902595E126BFB
:106B900096AA82AB8322E51228F582E51339F583A4
:106BA000A3223BF583E0F508A3E0F50922F0851662
:106BB00082851783A3A3126BBA22126F33F9227452
:106BC000F01225171238F08A088B09AE08AF09EACF
:106BD0004F7003026C5D750800806F750CFF750DBA
:106BE000FF750EFF750FFFE50875F00CA4F8A9F00E
:106BF000126C79123CBCEA4B604E8A828B83A3A351
:106C0000A3A3E06401600D8A828B83A3A3A3A3E006
:106C100064027034126C6C700C126C96122D7F1220
:106C20006C60122B9EE50875F00CA4F8A9F0EE2814
:106C3000F582EF126C87122AAB500DE50875F00C47
:106C4000A4F8126C79123CC805088E828F83E0F894
:106C5000E508C3984085EEFAEFFB12338602532312
:106C6000EA2417F582E43BF583780C22EA241BF52D
:106C700082E43BF583E0640122EE28F582EF39F5EA
:106C800083A3AA82AB832239F583A3A3A3A3A3A3DF
:106C9000A3A3A3780C221277CE780C221278D0A36B
:106CA000A32274F112251774F6122BB6EAFEEBFF3D
:106CB0007508009019401269B570457A377B00124B
:106CC00033809019401259AFF9EA4960197C377D39
:106CD0000079001232C6EEFCEFFD901940126436C6
:106CE0001238BAE9700B8518828519837488026E90
:106CF000341277091273B47401F0127359026EBF23
:106D0000E8242EF582E439F5837402F0EAFCEBFD09
:106D100012733F1238BAE9700C8518828519837492
:106D200088F0750801750A0A750B19780A122B2666
:106D3000126FC6F582E438F58312295312770924BD
:106D400028127326FC126FC0126EE02414126EC952
:106D5000122AE8126ED7126F1F2431127326603A7E
:106D60001274011269A0CC2432126F116020750CCC
:106D70000A750D19750E00780C122B22127401FC85
:106D8000E433FD126FBA126F04122AE8800C8518E2
:106D9000828519837488F0750801780A122B2612EF
:106DA0006FB4F582E438F583122953127709241160
:106DB000127326FC126FAE126EE0242B126EC912F3
:106DC0002AE8E9F81277092434126F1F2434127369
:106DD00026602E1273F81269A0CC2435126F116050
:106DE00042750C0A750D19750E00780C122B2212C3
:106DF00073F8FCE433FD1277092435126F04122A6C
:106E0000E8E508A2E04025126ED7127326700890BC
:106E100019401273C460157B007A0079001238C0E3
:106E2000026EBF8518828519837488F08518828563
:106E300019837486F07409122E00740212771D12E1
:106E40006EFD122E00E8F0A3E912771D1273841272
:106E50002B2A7401122B86880889097808122B26A0
:106E60007508207509807808122B2679017406129E
:106E70002B96EEFAEF126507122AE81273AA703CFD
:106E80007409122E007402127426126EF8122E006B
:106E900012742A122B2A7401122B86880889097809
:106EA00008122B267508207509807808122B267980
:106EB000017406122B9612736F122AE81238B474FA
:106EC0000A122AE87F07022843F582E438F583E0B6
:106ED000F9123818740422901940126EEE243122EF
:106EE000F582E438127367126EEB22901940126E2D
:106EF000F222E0F8A3E0C822F5838882A3A3126BF4
:106F0000BA740122F582E4381273671232BA74033C
:106F100022F582E43CF583EAF0A3EBF0EA4B22F59C
:106F200082E438F583126F2AC822E9F0126F30220A
:106F3000901940E0F8A3E022C082C083901940126B
:106F400069B56067E82435F582E4391269B36008F1
:106F50001277092435126FCC126FBA1269AF60062E
:106F6000126FBA126FCC126FB41269AF6006126F53
:106F7000B4126FCC126FC01269AF6006126FC012EC
:106F80006FCC126FC61269AF6006126FC6126FCC5B
:106F9000126FAE1269AF6006126FAE126FCC90190D
:106FA00040126FD2901940E4F0A3F0026592126E85
:106FB000EB242C22126EEB241222126EEB243222CE
:106FC000126EEB241522126EEB242922F582E4388E
:106FD000F5831273691233862274F1122517EAFEC3
:106FE000EBFF8C088D09750A018C0C8D0D750E0058
:106FF000780C122B227C177D001270AB122AE8123B
:107000007572E508241112709AE060271278FC125C
:1070100070C8601CE50824121270BC122B22E5080F
:1070200024111270B1125EC9126F08122AE880038F
:10703000750A00E508241412709AE060251278FCA5
:10704000EE24151270CB6041E50824151270BC12B5
:107050002B22E50824141270B112708F126F0812DF
:107060002AE8E50AA2E0401C125EC81269B3600675
:10707000125EC8126FD012708E1269B36006127061
:107080008E126FD0A90A026EC4750A0080DAEE244F
:1070900015F582E43F22E508240BF582E43509F575
:1070A00083227D00EE2404FAE43FFB1232BA74031B
:1070B0002212733625E0FCE433FDEE22127336F51E
:1070C0000CA3E0F50D780C22EE2412F582E43FF5D6
:1070D00083EAF0A3EBF0EA492274EE12251774ED6F
:1070E000122BB6890B8A0E750C00750D00750AFF00
:1070F0007510FF7511FF75080075090085188285E8
:107100001983E4127426F9E84960167403650B606C
:10711000067402650B700FE0C824301273266B6092
:107120000579000273217CC67D387A007B00123F0E
:10713000807401650B700A851882851983748580B7
:107140003DE50B60067403650B70199019401273CE
:107150008AF07403650B7029E50E60298518828515
:107160001983801A7402650B701BE50E901940702C
:107170000512738A800812770C1273A17402F080D2
:1071800004E50B601E12739070191273BD60051236
:107190006EDA800A1273C4600A12770924341273FB
:1071A0002614F01273BD6018126BA51274011278C8
:1071B000A2CA24321273D5241D12734C24258026B2
:1071C0001273C4602A901940E02417F508A3E03434
:1071D00000F5091273F81278A2CA24351273D52467
:1071E0000612734C240EF582E43AF583E0F50A7436
:1071F00009122E0074021267A3E06003027296E582
:10720000084509700302729612739070047E228002
:10721000027E21850882850983126EFC122E00E809
:10722000127747901944E0C0E01277092430F582C4
:10723000E438F583D0E0F07412122E007403F0AC41
:107240000CAD0D740A122B8E127417E0F50C780C2D
:10725000122B2A780A122B2A740C122B86880C897E
:107260000D780C122B267810122B26E5082406F533
:107270000CE43509F50D780C122B2612732EF974D7
:1072800009122B96EEFA7B001239747408122AE860
:1072900012735902731F126F30126EF8122E001201
:1072A000742A122B2A7401122B86880889097808FF
:1072B000122B267508207509807808122B26790173
:1072C0007406122B9612736F122AE81273AA704C6E
:1072D0001277092419F582E438F583126EFE122E16
:1072E00000E8F0A3126F252418F582E438127382A7
:1072F000122B2A7401122B86880889097808122B10
:10730000267508207509807808122B2679017406E5
:10731000122B9612733F126508122AE81238B479BC
:107320000174130263A2F582E438F583E022E508D4
:10733000240E12733622F582E43509F583E022909B
:107340001940E02417FAA3E03400FB22F50CA3E077
:107350003400F50D901940E0227CC67D38901A1556
:10736000127369123F8022F583E0FAA3E0FB2290BA
:10737000194012736912650822E516240EF582E49D
:107380003517F583E0F50878082212739A74012204
:1073900090194012739AE0640122126EF21273A1E6
:1073A00022242FF582E438F58322126EEB1273B497
:1073B000E0640222242EF582E438F5832212740759
:1073C000901940221273C822126EF22434F582E41E
:1073D00038F583E022F582E43AF583E028F8A3E06B
:1073E00039F9E824FEF582E934FFF583E0F510A3CE
:1073F000E0F511901940E0229019401273C825E081
:107400002212740725E022901940126EF22431F501
:1074100082E438F583E02212741B22123488850836
:1074200082850983A322126F2B22E8F0A3126F2A10
:10743000F5838882A3E0F508780822C082C0837BA8
:10744000007A8579011238C002659274F41225170A
:10745000ECFEEDFFEA240F127818127852126160E8
:107460008C828D83A3A3E8127747EA240E12781842
:107470001254E3126BA2850882F58312790B1277FE
:1074800046E5082402F50850020509FCAD09EE2482
:1074900006127562C0E01267943FF583D0E0F0E514
:1074A000082409F50850020509F582850983127838
:1074B000A9F9EE1275333FF583EA12774712757218
:1074C000850882850983A3A3E0F8EE2411127619BA
:1074D00050020509E860191275391270C86011EE82
:1074E0002412127555241112754D8A088B098007D4
:1074F000EE2411127545F0850882850983E0F812A3
:107500007602E81277DC858208858309601EEE2406
:107510001412663E127539EE24151270CB600DEE12
:107520002415127555241412754D8004127542F0FD
:10753000025388240FF582E422F81278F28B0BA90B
:107540000B22EE2414F582E43FF583E422125B72F1
:10755000F912383C22125B72FCA3E0FDAA08AB09C9
:10756000EE22FAE43FFB12741BA3A3A3A3A3A3A3DD
:10757000E022EE2412F582E43FF583E4F0A31275D5
:1075800086E4F0A3F022F0EE2415F582E43FF583C3
:107590002274F6122517ECFEEDFF12760E126BA286
:1075A000AC08FDEEFAEF1275658E828F83A3A3A35C
:1075B000A3A3A3A3A3F0E5082409F5085002050935
:1075C000F5828509831278AEA3F0A3E9127628F834
:1075D000EE2413127619500205097403687013AC77
:1075E00008AD09EE240B127562C0E0127602D0E0FD
:1075F000800C850882850983127893F0A3E9F00254
:107600005439EE1261543FF583228A088B091276B1
:107610001222EA2413F582E422F582E43FF583E89E
:10762000F0E5082403F508221277E0A3E02274F2C3
:10763000122517EAFEEBFF750A00EA241012663ED7
:10764000C3940C400D12641112770C240B12732694
:10765000F50AA80AE828F8E433F9E8240D12787F3F
:1076600070030276F6EE12663CFEA3E0FF8E82F512
:1076700083E0F88A828B8312771DAE82AF837076A7
:10768000EEFCEFFDEA240312771050010FF5828F14
:1076900083125C36850882850983127746127096BC
:1076A000E4F0E50A6050E508240DF8E43509F98EA8
:1076B000828F83A3A3E0C0E0127096D0E012783EE0
:1076C000C0E01276FDD0E0F0EE2404FE50010F85FC
:1076D0000A0B8E828F831269AAFBEC88828983123F
:1076E00059B0E82402F8500109EE2402FE50010FBF
:1076F000150BE50B70DCAA08AB0902787AE50824C3
:107700000CF582E43509F58322901940126EEE22C1
:10771000FAE43509FB123488EE2408FE22127721A0
:1077200022F08E828F83A32212772C2212773022AE
:10773000F088828983A3A3A322E0FEA3E022A3E032
:10774000F9EA8C828D83A3F0A3E9F022F583126F0E
:1077500033F98882F583E02274F11225171277CA73
:10776000E0F508A3E0850882F583E0F50BA38582A8
:1077700008858309A3A3E0F50A1277B560308A82F1
:107780008B83E50BF0850882850983E0FA1278D6B1
:10779000E50A1277DCA3A3A982AA83890C8A0D8843
:1077A0000E780C122B22AC0A1270A2122AE8EEFA02
:1077B000EFFB026EC42404FAE43400FB1233808A27
:1077C0000C8B0DAE0CAF0DEA4F221277CE22127742
:1077D000D222EA2413F582E43BF583221277E022D9
:1077E000F0850882850983A32274F7122517EA24FD
:1077F00013F8E43BF98882F5831278A9F5838A822D
:1078000012781E1278248882F583A3E0FA88828990
:1078100083A312773E0252A5F582E43BF583E08C08
:10782000828D832212782B126BBA22F08882898390
:1078300022FAE439FB1233802212786CE0221277AC
:1078400021A3A3E0221277D2E0FEA3E08E82F5838B
:10785000E022127904A32212785B22F08A828B83C1
:10786000A3A3A32212786CA3A3A3E022F08E828F9D
:1078700083A3A3A3A3A322122AE87F06022843FA24
:10788000E4391263AAEA4B22E0F50FA385820A8548
:10789000830B221278A9F9EE240BF582E43FF583DD
:1078A000EA22F8E433F9901940E0FAA3E022125CEE
:1078B0003A8E828F83A3A3A3A3A3A3A3A3221234EC
:1078C00088850A82850B83A3A3A3A3A3A3A3A322D2
:1078D000E08A828B8322A3E0F8E4C8F9EA8E828BE7
:1078E00083A3F0A3E9F08E828B83A3A3A322127853
:1078F000F22225E0FAE433FB123380221278F28B75
:107900000DA90D22F08A828B83A322125C3A8C820D
:107910008D83A3A3A32274F61225178C088D091258
:107920007954FF125C328C828D83127747E82402EF
:10793000FE50010FFCEFFDE5081263B33509FB12A1
:1079400034888E828F83A3A3A3127A6FA3A3A3A3E9
:10795000F00254391277CE126F332274F2122517C7
:107960001279D275F00CA4A9F024011278318A0C96
:107970008B0DEA4B60558A828B83A38582088583B1
:10798000098A828B83E50BF0750A008037EEFCEFE5
:10799000FDAA08AB0912771550010F7904127AA8D5
:1079A000850882850983A3A3A3A3A3A3A3A3122D60
:1079B000E9EE2404FE50010FE508240CF5085002FE
:1079C0000509050AE50AC3950B40C2AA0CAB0D02D6
:1079D000787A127845F50BA3AE82AF83221278A98C
:1079E000F8E4C8F9EA282212785BA3A3A3A32274BF
:1079F000F61225178C088D0912760E3B127A9B859C
:107A00000882850983122DE98E828F83A3A3A3A305
:107A1000E0F8850882850983A3A3A3A3F0C3940695
:107A200050098E828F83127A74804085088285097E
:107A300083A3A3A3A3E064FE600E85088285098367
:107A4000A3A3A3A3E0F470248E828F83127A6FF035
:107A5000EE2406FE50010F850882850983A3A3A3A7
:107A6000A3E0F47007127A86F0A3E9F00254391209
:107A70007A74A322A3A3A3A3A3E085088285098324
:107A8000A3A3A3A3A3228E828F83125C3A850882CC
:107A9000850983A3A3A3A3A3A3A322F58312773904
:107AA000FF7904EE127AA822FAEFFB1232D2EAF83A
:107AB000EBF9ECFAEDFB22C082C083906180E4F028
:107AC000E04409F0906189E0D2E5F0906182E0D273
:107AD000E0F0E0D2E1F0E0D2E2F09005417401F094
:107AE000027DE674E812251774F6122BB68A168BFF
:107AF00017ECFEEDFFEA4B60228A828B83A3A3A3DF
:107B0000A3A3A3A3A3E0640260168A828B83A3A32A
:107B1000A3A3A3A3A3A3E06403600579E8027D3CCB
:107B2000122E5EE9F46005791E027D3C8516828581
:107B30001783A3A3A3A3A3A3A3A3E0F514122E6A00
:107B40008A088B098C0A8D0B122E708A108B118C6F
:107B5000128D1385080C85090D850A0E850B0F788B
:107B60000C7910122C8674026514751400703B8A0F
:107B70000C8B0D8C0E8D0F74FE5514780C122B6D22
:107B8000E50CA2E0401985080C85090D850A0E85D3
:107B90000B0FE514780C122B6DE50CA2E050460596
:107BA00014E514C39418503D80C5850C08850D0953
:107BB000850E0A850F0B751003751100751200757F
:107BC0001300E514C3337810122A8C780879101248
:107BD0002D0BE5084509450A450B60090514E51418
:107BE000C3940C40C5741865147069851682851796
:107BF00083A3A3A3A3A3A3A3A3E06402606F85163A
:107C000082851783A3A3A3A3A3A3A3A3E064027005
:107C1000617406122E00EEF07407122E00EFF0854C
:107C20001682851783E0C0E07408122E00D0E0F0C1
:107C3000851682851783A3E0C0E07409122E00D058
:107C4000E0F079047406122B96E514F50875090026
:107C50007402802D740C651470A4851682851783B8
:107C6000A3A3A3A3A3A3A3A3E064037091791A021F
:107C70007D3C7908AC16AD17E514F508750900745C
:107C8000037808122CBF2508FA74613509FB127DB0
:107C90004664027903AC18AD19703B7A67127D59BE
:107CA000750C01750D00750E00750F00E514780C4C
:107CB000122A8C7808790C122C867808122B1E74E4
:107CC00007122B8E1233447404122AE87903E91246
:107CD0002B967A6780577A64127D59E514C333FA7C
:107CE000750C01750D00750E00750F00780C122AC9
:107CF0008C7808790C122C86750C01750D00750EA8
:107D000000750F0074012A780C122A8C7808790CFF
:107D1000122C867808122B1E7407122B8E123344F5
:107D20007404122AE87903E9122B967A647B6112B3
:107D30007D46FB7A01A914122E647900740A122A76
:107D4000E87F10022843122F5A851682851783A3D5
:107D5000A3A3A3A3A3A3A3E022127DED8A088B090A
:107D60008C0A8D0B2274F7122517EAFEEBFFEA4FFF
:107D7000602C8A828B83A3A3A3A3A3A3A3A3E06401
:107D80000260118A828B83A3A3A3A3A3A3A3A3E06E
:107D90006403700A122E5EE9F974FF69700479E8D1
:107DA00080158E828F83A3A3A3A3A3A3A3A3E0FB29
:107DB0007A00122E6479007F01022843C082C083BA
:107DC000740169900542700B7401F090618AE0D2F1
:107DD000E28008E4F090618AE0C2E2F08008127D5F
:107DE000ED7403122AE8D083D082022AD07B61127C
:107DF0002F607903AA18AB191232D222C082C08335
:107E0000900542E06401700479FE800279FF80D61B
:107E1000C082C083900542E06004790180099061CE
:107E200063E0F8744058F980BD74EC12251774F4BF
:107E3000122BB68A828B83A3A3A3A3A3A3A3A3E03D
:107E400064027040EC851882851983F07401122E4B
:107E500000EDF08A828B83E0C0E07402122E00D025
:107E6000E0F08A828B83A3E0C0E07403122E00D07E
:107E7000E0F0A818A919881289137E047510011260
:107E80002E6A800C8A128B137E08751002122E70D7
:107E90008A0C8B0D8C0E8D0F7F00850C08850D09CB
:107EA000850E0A850F0BEF7808122B6DE508A2E00E
:107EB0005053E510F5F0EF84F50BEEF97404122B36
:107EC00096E50B89F0A4FAA8F0E428FB74613BFB6B
:107ED000122F607404122B8688088909750A0078AD
:107EE00008122B22EEFC7D00851282851383A98265
:107EF000AA837B001232C07403122AE8E96401707D
:107F000004A90B800BE5102FFFC39418408C79FF58
:107F1000740C122AE87F0C02284374EF122517E92B
:107F2000FEEBFF74016A702374026F700F127F936F
:107F3000122A8C780C7908122C868026127FAE12B9
:107F40002A8C780C7908122C86803274026F701B90
:107F5000127F93122A8C7808122D3F780C79081220
:107F60002D0B780C122B1E7A838019127FAE122AE9
:107F70008C7808122D3F780C7908122D0B780C1292
:107F80002B1E7A867B611233447404122AE87F091F
:107F9000022843122E6A8A0C8B0D8C0E8D0F7508E9
:107FA00001750900750A00750B00EE780822122E83
:107FB000708A0C8B0D8C0E8D0F750801750900757C
:107FC0000A00750B00EEC333780822C082C08374A8
:107FD000FD122BB67903AC18AD197A83027DDEC091
:107FE00082C08374FD122BB67903AC18AD197A8662
:107FF000027DDE022AD0022AD0FFFFFFFFFFFFFF33
:108000000000000000000000000000000000000070
:108010000000000000000000000000000000000060
:108020000000000000002403540049002000430029
:10803000430032003500330031002000550053006A
:108040004200200043004400430024035400650024
:10805000780061007300200049006E007300740016
:10806000720075006D0065006E0074007300F449C5
:10807000D84714427A3F10400E36CA37F434D6340B
:1080800004490000000000000000000000000000A3
:1080900000000000000000000000000000000000E0
:1080A00000000000000000303132333435363738FC
:1080B0003941424344454602000206031BEE3301A8
:1080C00002000000000000000000FFFFFFFFFFFFB4
:1080D000FFFFFFFFFFFFFFFFFFFF0008000400029C
:1080E00000010000000000000000FFFFFFFFFFFF95
:1080F000FFFF02050200080174000000000000827A
:10810000003A003B000000000000000300000000F7
:108110000000FF10270000E803000019E0FCFF0941
:10812000433886E71F0300805101003C0000001027
:108130000E000004000000FFFFFFFF0000FF00FA38
:108140000000000403090400000000FEFFFFFF9789
:1081500051180060EA0000E204000058020000BC70
:108160000200003200000000F8FF0764000000E990
:108170000300000B0000000A000000F8FF000000F0
:108180000000000048000001000000300000000076
:108190000000000A74F7122517E9901AC3F0901A2C
:1081A00078E4F012328A901ADBE4F0A3F0901AC45B
:1081B000F0A3F01244E49019E6E060046401700654
:1081C000123C8C123E541232909019FFE4F0A3F04E
:1081D000123B9602B3ED74EC12251774D7122BB62E
:1081E000EAFEEBFF54806068901AC3E0F91232F6A1
:1081F0008A088B09EA4509604F7C0080010CEC7508
:10820000F003A4F8A9F0746728F582744F39F58358
:10821000E493F4602CE493F88508828B83E0687023
:10822000DCAA08EC75F003A4F8746828F582744F92
:1082300039F583E493C0E0740193F583D082124A48
:1082400089AA08AB091232E4EEFAEF648002871AB9
:10825000EF5420601E12432E8A088B09EA450960FC
:108260000A12424AAA08AB091232E4EEFAEF64207D
:1082700002871A9019E6E06402705FEEA2E0501FD8
:10828000901A7DE0640F7011790012421AE96009BA
:10829000901CA3122DD1124232EE6401028631EFFE
:1082A000544060369018CEE064067028740BF0904D
:1082B0001CBBE0F9750801750900750A00750B0013
:1082C000901A6BE07808122A8CAA08AB09AC0AADA8
:1082D0000B123D769019D60286D8EE542070030218
:1082E00086027A207B00901AC3E0F9123452EA4BDE
:1082F0004C4D701A901AD7122DDDE8494A4B700E7A
:10830000750C01750D00750E00750F008061750C00
:1083100000750D00750E00750F0012345E8A088B13
:10832000098C0A8D0B901AD7122DDDE8494A4B6053
:108330002A901AD77808122AAB400E750CFF750DDB
:10834000FF750EFF750FFF801285080C85090D8CD7
:108350000E8D0F901AD7780C122B9E7401780C1288
:108360002B6DE50C450D450E450F70030285297CEC
:108370000079047A007B001242F88A088B09028493
:108380005685188285198374FFF07401122E0074CB
:10839000FFF07402122E0074FF12A30DFAA3E0FB8B
:1083A0007403122B9612D1A5124358E9640160039D
:1083B000028438E508240D12AFF04480F8A3E0F9F8
:1083C0007424122E00E8F0A3E912C4FEA3A3A3E0D4
:1083D000C0E07426122E00D0E012CFADA3E0540806
:1083E00060167424122E00A3E0440112873DC0E001
:1083F0007428122E00D0E0F0E50812ED493509127C
:10840000CF86601CE508240F12CC75A3E0C812C407
:10841000C638F583E0F87412122E00E8F0A3E4F0F9
:1084200090814712294B7404122B967407122B8EDD
:10843000123DB87404122AE8850882850983A3A333
:10844000A3A3A3A3A3A3A3740612873DF91242DA40
:10845000850A08850B09E508450970030285297C12
:10846000007904AA08AB091242F88A0A8B0B850826
:1084700082850983A3A3A3A3E0F510A3E0F511E48B
:10848000F512F513780C7910122D5F4023E50824BE
:1084900004F8E43509F9850C10850D11888289836B
:1084A000C3E09510F0A3E0951112F1CC70A2800EFC
:1084B000850882850983A3A3A3A3E4F0A3F085081C
:1084C00082850983A3A3A3A3A3A3A3A3A3A3E06477
:1084D00001850882850983A3A3A3A3A3A3702BE02E
:1084E00054046003028381850882850983A3A3A3C2
:1084F000A3A3A3A3A3A37406F07AB7850882850972
:108500008312892012422C028450A3A3A3A3E0600B
:1085100003028381850882850983A3A3A3A3A3A360
:10852000A3A3A37401F00284501242C87C00790115
:108530007A007B001242F88B09EA4509600C7A2028
:108540007B00901AC3E0F9123320850C0A850D0BCD
:108550007C0079047A007B001242F8EA4B701580A7
:10856000558A828B83A3A3A3A312E688E50898E526
:10857000099940098A828B83A3A312872F7C0079F3
:10858000041242F88B0DA90DEA4970D5C3E50A958E
:1085900008E50B95095013C3E508950AF508E509A8
:1085A000950BF509E508450970147A207B00901AAF
:1085B000C3E0F9123320901AD7129B39803FE508A7
:1085C00025E0F508E50933F509E4F50AF50B780827
:1085D000122B1E7A207B00901AC3E0F912344074EB
:1085E00004122AE812345EEAC0E0EBC0E0ED901A13
:1085F000D7FBECFAD0E0F9D0E0F8122DE9EE6420D8
:10860000802FE06007640160030286F3EE5410607F
:1086100008123E90EE64108018EE54406008123F3D
:1086200008EE6440800BEE5480600B123D5EEE64F9
:1086300080FAEF02871AEF5401600B1244BAEEFA87
:10864000EF640102871AEF54086047123E609019E8
:10865000D0E0640170349019D1E0602EF508E4F5A3
:1086600009F50AF50B908117780C122D7F7808799F
:108670000C1224287808122B1E7A007B08901AC34B
:10868000E0F91234467404122AE8EEFAEF640802A4
:10869000871AEF54106012901AD5E06005E4F012CA
:1086A0003E60EEFAEF64108071EF54406045901A1E
:1086B000FC12CF8860369019DAE06401702E901AAF
:1086C000FD12C8AA124A89901B0212CF88600612B6
:1086D000C8AA124A8990811712294B7A007B4090D0
:1086E0001AC3E0F91234467404122AE8EEFAEF6471
:1086F000408027EF5402600A1244B4EEFAEF64029D
:108700008018EF5404601612CE5C7901901A76122C
:10871000CC89123DD6EEFAEF6404FB80047A007B2C
:10872000007429122AE87F0C0228438E828F83A3CB
:10873000A312873522E0F508A3E0F5092212C5024D
:10874000A3E022C082C08374EA122BB67C167D009F
:108750007900AA18AB191232C67408122E007402DE
:10876000F0901A6C129B0C1287837409122E00125F
:10877000CC987413122E00E412CFBF123B847416EF
:1087800002D578E8F0A3E9F0901A7612D53B22746E
:10879000F712251774DA122BB6EAFEEBFFEE4F60E4
:1087A0002DAC18AD191243587406122E00E0601E4D
:1087B0007417122E00E0FD7401122E00E0FCEEFA98
:1087C000EFFB79001241F0E9600479A4800279009E
:1087D000742602B3EA74F4122517EAFEEBFF8E82C8
:1087E0008F83A3A3A3A3A3A3E05440601912E2EADA
:1087F00012CC89124412E960077AFF7BFF0288CA13
:1088000012E2EA0288BD9019E6E0600764016003A5
:108810000288B2901A63E0A2E140030288B212B467
:108820003012CD88A3A3A3A3E0FA88828983A3A3EF
:1088300012D9078E828F83A3A3A3A3A3A3A3E0547B
:10884000106004794080027900750AFE750BFF788C
:108850000A122B2612890E122953AC08AD0912E216
:10886000EA12CC89123E667404122AE8E5086A709E
:1088700003E5096B600B12BF476A7003A3E06B70DE
:108880003F750A00780A122B2A79028E828F831292
:10889000B4F1FCA3E0FDAA08AB0912445474011220
:1088A0002AE87508CDAA0812891C12422CE9604CEE
:1088B00080579019E6E0640270E8901A6C12CC8937
:1088C00074FE6A700374FF6B60D812E2EA12E15A18
:1088D000124412E98E828F83600B12BC6512F49EE3
:1088E000E4F0A3800312F48CF07C207D428E828F12
:1088F0008312CC89123B8AE9F50870A9EE4F600912
:108900007901EEFAEFFB1242D4A908028FBEEE12F3
:108910008913222411F582E43FF583228E828F830E
:1089200012F475E0F92274F6122517E9FEEAFF7ACF
:108930000F7B001232DEEA4B601F8A828B83740C3D
:10894000F0EEA3A3F0EF8A828B8312B1A6901AC334
:10895000E0F91232EA7900802FEEF91242FE8A081D
:108960008B09A808A909E849601C88828983A3A308
:10897000A3A3A3A3A3A3A3740612ED4FE0F9123F90
:108980001AEEF91242DA791002C90774F4122517A7
:108990008A088B098C0A8D0B901A7DE0640F702C6D
:1089A000EA4509450A450B6023901A78E06408609F
:1089B00005E0640470167808122B1E7A017B009083
:1089C0001AC3E0F91234407404122AE8028FBE740C
:1089D000F2122517EAFEEBFF8C0A8D0B8908740E44
:1089E000122E0012E68D850C82F583E4F0A312CEE0
:1089F00051F5838882E0F91243EEE9602612CC7CBF
:108A0000124412E96402701B8E828F83A3A3A3A376
:108A1000A3A3A3A3A312BAD2850C82850D8312CC83
:108A200098800375080012B4E814602E1460431493
:108A3000606414606C146048147003028AC124FEE0
:108A40007003028ADB147003028AE4147003028A42
:108A5000F7147003028B05028B1B780C122B26ACCB
:108A60000AAD0BEEFAEFFB123E787402122AE8020E
:108A70008B00AC0AAD0BEEFAEFFB123E7E028B25AB
:108A800012CC7C124412E96003028B1BEEFAEFFB5E
:108A9000123ECC028B25A908EEFAEFFB12445A8055
:108AA0005F12B96664027073E508700A12E2107012
:108AB00003A3E069706FEEFAEFFBA9081243E280AE
:108AC0003F12E2107003A3E069705012B9666402AD
:108AD0007049EEFAEFFB1243CA804AEEFAEFFB123E
:108AE00044D8804112E2107003A3E069702DEEFAC1
:108AF000EFFB124466802EEEFAEFFBA908124472D7
:108B0000E9F50880209019DAE064017009EEFAEFC7
:108B1000FB12447E800F750800800A7508007AD326
:108B20007B001237BEA9088007A90A7403122AE83D
:108B30007F0602284374F412251774D6122BB68AC6
:108B4000088B098A828B83A3A3E0F91242FE8A0A6A
:108B50008B0BAE0AAF0BEE4F7003028C6785088259
:108B6000850983A3A882A983E0C0E012CC63D0E08A
:108B700012E69AE064F16033850882850983A3E0F8
:108B800064CD6027850882850983A3E0641A601B91
:108B9000850882850983A3E064E9600F85088285E2
:108BA0000983A3E064E16003028D5F9019E6E06051
:108BB0000764016003028C888E828F83A3A3A3A322
:108BC000A3A3A3E054087003028C888E828F83A332
:108BD000A3A3A3A3A3A3A3A37405F09019E6E06045
:108BE0000464017053850882850983A3E064E96009
:108BF00047901AF812CF88600612C8AA124A8990C4
:108C00001AFA12CF886031901A63E0A2E15029125B
:108C1000D17BA3A3A312B9A48882898312CC891221
:108C20004514EA4B6012850882850983A3E0F99018
:108C30001AFA12E2EE124A898E828F83A3A3A3A3AB
:108C4000A3A3A3A3A3E0640270108E828F83A3A3C7
:108C5000A3A3A3A3A3A3A37406F085088285098315
:108C6000A3A3E0F91242DA1242C89019E6E06402C6
:108C70007011901CA9E0F508A3E0AA08FBE4FCFD34
:108C8000124232742A028FBB79001242D4E9700377
:108C9000028D5F9019E6E0600764016003028D3485
:108CA000901A63E0A2E14003028D3412CF83700377
:108CB000028D348E828F8312CC897404122B96120B
:108CC000D1A5124358850882850983A3E064E97021
:108CD00023128E69122B2A850882850983A3E0F569
:108CE0000A780A122B2A128E7612CC8912438E74BD
:108CF00002122AE8740D122E0012CF7912F0F71228
:108D0000CC987409122E00E060047940800279004A
:108D1000740F122E0012B9A4740D122E0012CC89F9
:108D2000123E72E9600E8E828F83A3A3A3A3A3A336
:108D3000E04420F0EE2404F50AE43FF50B8E828F28
:108D40008312AFFDE0F9850A82850B8312CC89126C
:108D5000329C850A82850B83EAF0A3EB028BDA85CD
:108D60000882850983A3E0C0E07402122E00D0E0DF
:108D700012A7ED12E0F6E508240B12AFF0C0E07484
:108D800003122E00D0E012E95DE0AA18AB19703191
:108D9000123DB29019E6E06004640170277402127B
:108DA0002E00E0701F12E2EA12CC89124412E97020
:108DB00039901AF812CF88603112C8AA124A8980F5
:108DC000031243E87402122E00E064E9701C128E54
:108DD00069122B2A750AE9780A122B2A128E76124A
:108DE000CC8912438E7402122AE89019E6E06007DB
:108DF00064016003028C38901A63E0A2E140030230
:108E00008C388E828F83A3A3A3A3A3A3A3A3A3E0E1
:108E10006402703C8E828F83A3A3A3A3A3A3E05418
:108E200004602D12E2EA12CC89124412E98E828F7C
:108E300083700F12E2EE74FFF0A312A99D74050275
:108E40008C59A3A3A3A3A3A3A3A3A37403028C5924
:108E5000850882850983A3E064E96003028C38EE0B
:108E6000FAEFFB124490028C388E828F8312DA3D27
:108E7000750A01780A22E508240C12BF66E0F98A17
:108E8000828B83A3A3A3A3A3A3A3A3A312D8FF228C
:108E900074F4122517EAFEEBFF7508007509008EC1
:108EA000828F83A3A3A3A3A3E0603B75080812CC21
:108EB0007C79FF12401C8B0BEA450B601075082C67
:108EC0008E828F83A3A3A3A3A3E0D2E0F08E828F30
:108ED00083A3A3A3A3A3E0540364016003028F9AB6
:108EE000430811028F9AEE241812B9696049EE24E2
:108EF0001A12B9696003F4701D12E2107003A3E046
:108F0000697006750822028F9A901A78E0640460EE
:108F100003028F9A801CEE241BF582E43F12B9B243
:108F2000241A12B969FAEE2419129BC9123EDEE91D
:108F30007068750901806312CC7C124412E96402E6
:108F4000700375080112E2107003A3E0697006E572
:108F500008D2E1F508E50860158E828F83A3A3E0AF
:108F60007006E508D2E58004E508D2E6F50812CCE3
:108F70007C124412E964017006E508D2E0F5088E1F
:108F8000828F83A3A3E0601212B4E8F91243EEE9E2
:108F900064016006E508C2E0F5089019E6E06004A7
:108FA00064017012E508A2E1400CE509A2E0400668
:108FB000E508D2E7F5080289097418122AE87F0447
:108FC00002284374EC12251774C3122BB6EAFEEB89
:108FD000FF85188285198374FEF0A304F0751000D4
:108FE0007511007509009019E6E0640270248E8204
:108FF0008F83A3A3A3A3E06019901CA712CF88605E
:1090000011901CA7E0F50AA3E0AA0AFBE4FCFD12FC
:1090100042327405122B968E828F83A3A3A312CFA4
:109020007B12CC87124358E970030293FF780174D6
:1090300007122E00E0C39402400278007409122E39
:1090400000E0C3940240027800740E122E00E06427
:10905000F87003A3E0F470030293FF740E122E0065
:10906000E064F97003A3E0F470030293FF740E123E
:109070002E00E064FA7003A3E0F470030293FF741F
:109080000E122E00E064FB7003A3E0F47003029361
:10909000FF7408122E00E0F9901A66E0696003027E
:1090A00093FFE8A2E040030293FF9019E6E0640218
:1090B000700B7429122E00E060030293FF12BAC9EC
:1090C0007424122E0012B9D3241C12BACC741212BA
:1090D0002E0012CC98740B122E00E0601D741C122E
:1090E0002E00E0FD7406122E00E0FC8E828F8312AB
:1090F000CC8779011241F0E9703D7405122B8E1274
:109100004244E9F508740B122E00E0702F901A60AB
:10911000E060297422550864226021744255086475
:109120004270147422122E00129AE5600F742212FB
:109130002E00129AEB60057ACF029401E9A2E65064
:109140006C9019E6E060046401701B901A63E0A261
:10915000E150137422122E0012B4F11229D8010129
:109160000B849100FF937422122E0012B4F124FD9F
:10917000601214600F24FD600B24FD600724FE6064
:10918000030293FF7422122E00129B24700F74228C
:10919000122E00A312C8AAA3E0640D601074051279
:1091A0002B8E12444EE964017003029ACEEE242DF8
:1091B000F582E43FF58312A3007003A3E0697021F8
:1091C000750A00780A122B2A780A122B2AEE242F0D
:1091D000129BC9129AF112CC8912438E7402122A80
:1091E000E8740B122E00E07003029290129AF112B2
:1091F000CC891245148A0A8B0BEA450B7003029343
:10920000277406122E00E0F88E828F83A3A3E02835
:10921000F8A3E03400F9E8240D129AD3F88A828B7F
:1092200083A3A3A3E068600EE88A828B83A3A3A331
:1092300012B194129B3979047406122E0012A650B2
:10924000E02AF8A3E034008882F583A3AA82AB83E6
:109250001232D28A0C8B0D8C0E8D0F850A82850BF3
:1092600083A3A3A3A3780C122AAB4003029ACE9047
:109270008187780C122CF8850A82850B83A3A3A31F
:10928000A3E50CF0A3E50DF0A3E50EF0A3E50FF0C8
:109290009019E6E0640260030293D4901A78E064C7
:1092A000046008E064096003029ACEE508A2E54084
:1092B00003029362EE242F12B969C0E07402122EE9
:1092C00000D0E0129B4AC0E07403122E00D0E012DE
:1092D0009B42C0E07404122E00D0E0F07416122EEF
:1092E00000E0640170267410122E00129B017003BE
:1092F000A3E0697017740E122E0012CC891244126A
:10930000E9640270077416122E00E4F0129B2F120B
:10931000294B7406122B967409122B8E123DB874C9
:1093200004122AE8029ACE901ABDE064016003029A
:1093300092907422122E00129AE57009E508A2E6B6
:1093400050030292907412122E00E0F47003A3E016
:10935000F4600CEEFCEFFD7405122B8E12425002ED
:109360009ACEA2E64003029ACE7422122E0012D1A7
:10937000887016741C122E00E0640270547405127A
:109380002B8E79001243E280487422122E00129A2A
:10939000EB7014741C122E00E06404703474051217
:1093A0002B8E1243D6802A7422122E00129B247018
:1093B0000C79007405122B8E12445A8014742212F8
:1093C0002E0012B4F3640C70087405122B8E124434
:1093D0008A029ACEE0600764016003029ACE901A76
:1093E00063E0A2E14003029ACE7429122E00E060ED
:1093F000267410122E0012CC89123CAAE9700A7A47
:10940000D37B001237BE029ACE8E828F83A3A31223
:10941000E2EEA3E0C2E5F07416122E00E0601DEE4D
:109420002402F8E43FF9E8FAE9FB12D18E14F012B5
:10943000D18EF87416122E00E8F07006E508C2E727
:10944000F508E508A2E35061751110A2E250187406
:109450000A122E00E054E3F0740A122E00E01313F7
:1094600013541FF8E0802CA2E4502A740A122E0034
:10947000E01313543F5407F86009740768600B1831
:10948000E87007C3E508C2E7F508E8333354FCF891
:10949000E054E348F0740A122E00E0C0E08E828FA0
:1094A00083A3A312B0DBD0E0F0901A78E0640460EC
:1094B00008E064096003029585740E122E0012E222
:1094C0001D7003A3E069601F740E122E0012CC8978
:1094D000124412E96402600F740A122E00E0540371
:1094E00064016003029ACE7407122E00E07041EE10
:1094F000242F12B969C0E07402122E00D0E0129B32
:109500004AC0E07403122E00D0E0129B42C0E07407
:1095100004122E00D0E0129B2A12294B7406122B43
:10952000967409122B8E123DB87404122AE88052E8
:109530007422122E0012D1887016741C122E00E0B4
:109540006402703E7405122B8E79001243E2803261
:109550007422122E00129AEB7014741C122E00E06A
:109560006404701E7405122B8E1243D6801474226C
:10957000122E00129B24700A79007405122B8E1291
:10958000445A029ACE74615508700302968CE5081D
:10959000A2E0506D12B99B7405122B8E123F0EE99A
:1095A000705C124388E9F5097416122E00E0700F02
:1095B0007410122E00129B017003A3E0696042A98F
:1095C0000912B99B7405122B8E123F14E96024E531
:1095D00008A2E3500C85188285198374FFF0A380DC
:1095E0000C740E122E00129B0CE8F0A3E9F075101B
:1095F00004800EE508C2E5F50875090080035308EC
:109600009FE508A2E5503FEE242F12B969C0E0742F
:1096100002122E00D0E0129B4AC0E07403122E000A
:10962000D0E0129B42C0E07404122E00D0E0129BE6
:109630002A12294B7406122B967409122B8E123D96
:10964000B87404122AE8E508A2E64003029961A86A
:1096500018A919880A890B780A122B26A909129AC7
:10966000DC122B8E1242387402122AE8E9F50970D6
:10967000030299617422122E0012B4F16401600396
:1096800002996174104510F5100299617407122E49
:1096900000E06401705D7422122E0012B4F16405C2
:1096A000701EA818A919880889097808122B261293
:1096B0009ADA122B8E1242387402122AE8029ACEDB
:1096C0007422122E00129B247029740E122E001286
:1096D000CC89123CAAE9601BA818A919880A890B31
:1096E000780A122B26129ADA122B8E124238740242
:1096F000122AE87416122E00E070257407122E004C
:10970000E06401700C7422122E00E0F8129B2460B9
:109710000CEEFCEFFD7405122B8E124250029ACE15
:109720001242CEE96003029ACE741D122E00E07040
:10973000030297DA7420122E0012B9A4741F122E9D
:1097400000E0FA741E122E00E0F9123EDEE9607DA0
:10975000741F122E00E0701E740E122E00129B0C4D
:1097600012F4AEFAA3E0FB123CB68B0BEA450B6099
:109770000302995B80517420122E0012CC89741F51
:10978000122E00E0F9123ED885188285198312E165
:109790005A7808740D122E00E060027810740C12D2
:1097A0002E00E06004740828F8740A122E00E060AD
:1097B0000108088E828F83A3A3E028FAA3E0340077
:1097C0008A82F583E014F075104002995B750800F9
:1097D0007808122B2A790B029914740E122E00129B
:1097E000CC8D7409122E00E0600302992FE508A2C7
:1097F000E3500302992F7407122E00E06401607A8F
:10980000790085188285198312CC89123F328A0A21
:109810008B0BA80AA90BE849601C88828983A3A343
:10982000A3A3A3E06401605288828983A3A3A3A3B6
:10983000A3E064026044EE242D12B99E851882854F
:10984000198312CC891245148A828B83E582458361
:10985000600FA3A3E0F9124532E96005C394084004
:10986000197410122E0012CC89123CAAE97003025E
:10987000990A7409122E007404F07800E8F509784A
:1098800009122B2A741E122E00AC82AD83740F12A3
:109890002E0012CC89740A122E00E0F9123F447493
:1098A00001122AE8E9600F7510208E828F83A3A32E
:1098B00012B4F1543FF0741D122E00E06023740EB8
:1098C000122E0012B9A4741E122E00AA82AB8312AB
:1098D000435285188285198312E15A74404510F568
:1098E000107407122E00E0640160157900741012E4
:1098F0002E0012B9A4740E122E0012CC89123EE46E
:10990000E508A2E3503779408035750800780812E1
:109910002B2A7902740F122E0012B9A47411122E80
:109920000012CC891244547401122AE8029ACEE53E
:1099300008A2E3400302987A784002987C79007488
:1099400010122E0012B9A4740E122E0012CC89121D
:109950003E72E9600674204510F510124388E9F55F
:1099600009851882851983E064FE7003A3E0F47012
:10997000037509009019D3E064016003029A14EEA4
:10998000241312B969F47003A3E0F47003029A146B
:10999000740E122E00C3E094F9A3E094FF507512E8
:1099A000BAC97410122E00E0687003A3E069606405
:1099B0007410122E0012CC89123CB68A0A8B0BA8A6
:1099C0000AA90BE849604D88828983A3A3A3A3E079
:1099D0006401600D88828983A3A3A3A3E06402705D
:1099E000337430122E00740112E6A4F8A3E0F97467
:1099F0003B122E0012CC987430122B8E123C62E96E
:109A000060127433122E00AA82AB83123CC8E96044
:109A100003123752E508A2E74003029ACEE5097027
:109A200003029ACE8E828F83A3A3A3A3E0FA7B00C6
:109A30001233808A0A8B0BEA450B7003029ACEEE32
:109A40002404F512E43FF5138E828F83A3129B1634
:109A5000122B22851282851383E0FC7D001232BA1C
:109A60007403122AE87407122E00E0C0E0742B126F
:109A70002E00D0E0F0742E122E00E4F0A3F0742B30
:109A8000122B86880C890D780C122B26750800780D
:109A900008122B2A7810122B26E509F508780812EF
:109AA0002B2A12B95D122953851282851383E0F99E
:109AB0007408122E0012B9A4AA0AAB0B1243467402
:109AC00008122AE8E96007AA0AAB0B123386743D34
:109AD000028723F582E412EEE222790012B96112C4
:109AE000B9A874072212B50B64062212B50D6407DB
:109AF00022EE242BF582E43FF58312B9B812B96245
:109B00002212D53BEE241312BF4E682212D53B859C
:109B1000188285198322A3E0F50CA3E0F50D750EDC
:109B200000780C2212B50D640322F0129B2F22EE56
:109B30002425F582E43FF58322E4F0A3F0A3F0A30B
:109B4000F022F0EE243112BF4E22F0EE243012BF8C
:109B50004E2274F4122517EAFEEBFF8C088D099053
:109B600019D0E0600F12E2107003A3E069700512D3
:109B70003E608052790012CC7C123F328A828B8305
:109B8000E58245836035A3A3A3A3A3A3E054186093
:109B90002AE508241C12CC75122953E50824131257
:109BA000CC75122953EE2418129BC9129BCE12CCED
:109BB00089123F4A7404122AE8800B7900129BCE66
:109BC00012CC89123E8A028FBE12BF4EF9228E82BB
:109BD0008F83A3A3A3A3A3A3A3A3A312B9B812CC57
:109BE000682274F012251774EA122BB68A0A8B0BBE
:109BF000EA2402F50EE4350BF50F0A0AFB123CBC11
:109C00008A088B09AE08AF09750801850A82850BA1
:109C100083A3E0F509750C01AC0EAD0F740B122E89
:109C200000AA82AB831234887413122E0074FEF0E3
:109C3000A304F07415122E007402F07408122E00A2
:109C4000E4F0901CE1E0700EEE4F700AE50970063A
:109C50007508C3029E1E901A78E0640860067508B5
:109C6000C2029E1A850A82850B83A3A3A3A3A3A382
:109C7000A3A3A3A3E0A2E1500EA2E35005750C0438
:109C8000800C750C038007A2E35003750C02EE4FA5
:109C90007003029D2D8E828F83A3A3A3A3E064048F
:109CA000600D8E828F83A3A3A3A3E06403700C7462
:109CB00004650C602C7403650C60268E828F83A370
:109CC000A3A3A3E06402600D8E828F83A3A3A3A34A
:109CD000E0640170317402650C60067401650C70FB
:109CE000188E828F8312CC89124430E9703F12A9FA
:109CF00093122E0012CC9880348E828F83A3A3A35C
:109D0000A3E06402600D8E828F83A3A3A3A3E0640B
:109D100001700A8E828F8312CC89123EA8E50A2434
:109D200002FAE4350BFB123CC87E007F007413126C
:109D30002E00E064FE7003A3E0F47046123C6EE96E
:109D40007040E509601B901CEA12CC89124430E98E
:109D5000700F901CEA12A997122E00E8F0A3E98078
:109D600020850A82850B83A3A3A3A3A3A3A3A3A3F4
:109D7000A3E05402F9123E9C7413122E00EAF0A3E1
:109D8000EBF07413122E00E064FE7003A3E0F47095
:109D9000067508C7029E1AE509F50D780D122B2AE3
:109DA000850A82850B83A3A3A3A3A3A3A3A3A3A331
:109DB000E0F9E50A2402FCE4350BFD7414122E00D0
:109DC00012CC89123DDC7401122AE8E9704CA90C0E
:109DD000E50A2402FCE4350BFD7413122E0012CCAC
:109DE00089123C988A0E8B0FAE0EAF0FEE4F601F9C
:109DF00074026509700D8E828F83A3A3A3A3A3E0D1
:109E0000D2E3F07415122E00E4F0750800800B7494
:109E100013122E0074FEF0A304F0E5097009AA18CD
:109E2000AB19123B6C800AFCA90CAA18AB1912439F
:109E3000D0E9FCEE4F6053E50960208E828F83A34A
:109E4000A3A3A3A3E0D2E6F074026509700D8E828D
:109E50008F83A3A3A3A3A3E0D2E5F0850A82850B99
:109E600083A3A3A3A3A3A3A3A3A3A3E0A2E6500D4C
:109E70008E828F83A3A3A3A3A3E0D2E7F08E828F69
:109E800083A3A3A3A3A3A3E004F0E508703BEC60C5
:109E9000337D007A017B10123296EE4F600CE50A9A
:109EA0002402FAE4350BFB123CC87413122E00E0B6
:109EB00064FE7003A3E0F4600B7413122E0012CC46
:109EC00089123EA8741602D929FC80C574F71225A0
:109ED0001774F7122BB6EAFEEBFF901A78E06403D2
:109EE000600DE064016008E06409600302A01B8E5D
:109EF000828F83A3E06003029FD97C007D007A02F9
:109F00007B0012329612A0208A828B8312BAD290E2
:109F10001A6912CC987953123B60901A78E0640960
:109F20006009901A7612CC8912450E85188285191F
:109F300083740112CFBF7942123B60901A78740487
:109F4000F07401122B8E794A123B5A7401122B962F
:109F50007A6E7B1A1234889018CEE0640B70057408
:109F600006F0800B7900901A7612CC89123DD690BB
:109F700019E6E060046401701F901A6CE064FE70E2
:109F800003A3E0F4602A79007401122B96901A6CF6
:109F900012CC89123C988018E064027013901A6900
:109FA00012B9A47A037B0012329612A87F1232965D
:109FB000901A63E0A2E35004D2F08002C2F012CF04
:109FC000B57952123B609019E6E06402704A901C29
:109FD000A3122DD1124232803FFC7D007A037B1008
:109FE0001232969019E6E06402701B9018CEE0647D
:109FF0000B7003740AF09019D4E4F0FA7B40901AC5
:10A00000C3E0F912344C8E828F8312A02A12CC89BD
:10A01000123DD6901A78E4F012429E740902B3EA17
:10A02000EE2402FAE43FFB22E0F8A3E0F9901A766E
:10A0300022C082C0839019FF12CF88701F901A78B7
:10A04000E014600924FC600A14600C800F901A0A66
:10A050008034901A06802F901A08802AE8496008F8
:10A06000901A0012A661700C8A828B83A3E0F91209
:10A070003DBE801D9019FF12D192640270051244FA
:10A08000A8800E901AF612CF88600612C8AA124A4B
:10A090008902C57574F412251774FE122BB68A084E
:10A0A0008B097A007B04901AC3E0F912344CAA1889
:10A0B000AB197950123B5A7A0F7B001232DE8A0AB2
:10A0C0008B0BAE0AAF0BEE4F6020850882850983AB
:10A0D000A3E07016901A76E0F47003A3E0F4603BFE
:10A0E00012A2FA7003A3E0696031850882850983B2
:10A0F000A374EA12A7E5123B607A6C7B1A794B12C3
:10A100003B607A767B1A7950123B607A6B7B1A79C6
:10A11000E1123B60EE4F700302A1A48E828F837424
:10A1200002F0901A76E0F47003A3E0F4600A12A241
:10A13000FA7003A3E069704F85188285198312A015
:10A1400028E8F0A3E912A7E5123B5A901A6912B069
:10A150000E12CC987A6C7B1A794B123B5A7A6B7B35
:10A160001A79E1123B5A750A00780A122B2A780AEA
:10A17000122B2A901C5712A02B12AD4412CC89121C
:10A18000438E7402122AE885088285098312A1A9E8
:10A19000A3F0901A787403F0EEFAEFFB901AC3E084
:10A1A000F91232EA7402028FBBA3E08E828F8322FF
:10A1B00074F412251774E8122BB6EAFCEBFD8C82BE
:10A1C0008D83A3A3A3A37808122D7F7808122D3FB7
:10A1D000901A797808122CD27F7F7E7F7900901AAE
:10A1E000797808122D7FE97808122B6DE508A2E036
:10A1F00050297800901AC48014850882850983A3A9
:10A20000A3E069700108E508241412CC7512AA2E87
:10A2100070E7E8C39F5004E8FFE9FE09E9C3941B17
:10A2200040BC8C828D83A3A3A3A3122DDDE8494AF1
:10A230004B6079EC2404F508E43DF509850882F5C6
:10A2400083122DDD901A79122DE97C187D0079009A
:10A25000AA18AB191232C6850882850983122DDD32
:10A26000851882851983122DE97404122E00740159
:10A27000F0901A7FE0C0E07405122E00D0E0F07478
:10A2800007122E00E412CFBF123B78806A901A7634
:10A2900012CC89123E0C8A0A8B0BA80AA90B901AC1
:10A2A0007612A309687003A3E069602D901AC412A6
:10A2B000AA2E602585088285098312A3007003A356
:10A2C000E069700C850882850983A3A3E06E60BDF8
:10A2D000E508241412CC7580D6EE901A6BF0124269
:10A2E00080E96013901A78E4F0901A0C12CF88601D
:10A2F0000612C8A8124A89028FB985188285198367
:10A3000012D53B901A76E06822E8F0A3E912A31177
:10A3100022F0850882850983E02274F412251774DF
:10A32000E8122BB68A828B83A3A3A3A3A3A3A3A320
:10A33000A312DA397C00901A797808122D7FEC7814
:10A3400008122B6DE508A2E0502FECF8EA2812BAAB
:10A35000C1F8901CE9E0C398501F75080175090009
:10A36000750A00750B00EC7808122A8C7808122DFB
:10A370003F901A797808122CD20CECC3941B40B68B
:10A38000901A79122DDDE8494A4B604E7C187D0009
:10A390007900AA18AB191232C6901A79122DDD85F0
:10A3A0001882851983122DE97404122E007401F0AD
:10A3B0007407122E007401F0901A7FE0C0E074055B
:10A3C000122E00D0E0F07407122E00E412CFBF125C
:10A3D0003B78901A787406F0801C901A78E4F0FCB0
:10A3E000FD7A047B10123296901A0C12CF88600608
:10A3F00012C8A8124A89028FB974F512251774D1B0
:10A40000122BB68A088B098A828B8312BC5D741C5E
:10A41000122B968A828B83A3A3A3A3A3A3A312A622
:10A420005912CC801242B0741C122E00E0702C85A0
:10A430000882850983A3A3A3A3A3A3A3A3E0C39432
:10A440000B40188E828F83A3A3A3A3A3A3A3A3E08F
:10A450006402700712CC63E0F4600302A64B901A0A
:10A4600078E06402700302A530E06406700302A580
:10A47000309019FF12CF88600812A661700302A500
:10A4800064901A78E064086008E06404600302A63F
:10A490004B741E122E0012A650A3A3A3A312BC5DE0
:10A4A0009019FFE0F849600712D198640260779034
:10A4B0001A76E06E7003A3E06F600302A64B74018E
:10A4C0006A60167423122E00AC82AD837A8A7B1ADE
:10A4D000123482E9600302A64B7A007B02901AC311
:10A4E000E0F9123452EA4B4C4D600302A64B901A2D
:10A4F00079122DDD851882851983122DE9901A7F36
:10A50000E0C0E07404122E00D0E0F07405122E00BA
:10A510007401F07406122E00740212CFBF123D4671
:10A52000E9600302A648EEFAEFFB1244A202A64B32
:10A530009019FF12CF88702C7508007808122B2A0A
:10A540007808122B2AEE2410F582E43FF58312CF0F
:10A550007CA3A3A3A3A312B9C112CC8912438E7406
:10A5600002122AE88E828F8312BAD27407122E004A
:10A57000E8F0A3E912A99D12BAD27409122E0012B2
:10A58000B9D312BF58C0E0740B122E00D0E0F01205
:10A59000CC63128731740F7808122D8E740C122E32
:10A5A00000E508F07420122E00E0C0E0740D122EB9
:10A5B00000D0E0F07422122E00E0C0E0740E122EE3
:10A5C00000D0E0F0741D122E00E0C0E07410122ED6
:10A5D00000D0E0F0741E122E00E0C0E0740F122EC6
:10A5E00000D0E0F0EE241012B969C0E07411122E10
:10A5F00000D0E0F07421122E00E0C0E07412122EA0
:10A6000000D0E0F0742E122E00E0C0E07413122E81
:10A6100000D0E0F07423122E00A982AA8389088A50
:10A6200009750A007808122B227C087D0074171225
:10A630002E00AA82AB831232BA7403122AE874077E
:10A64000122B8E123DD08003123D4C742F02B65A4D
:10A65000E0FA8E828F83A3A322A3E0F98A828B8300
:10A660002212D19964012274F712251774C9122B92
:10A67000B61244C0901A78E06408601F90506EE4EF
:10A6800093901A5AF090506EE493901A58F0901AE2
:10A6900081740112A7DCA30412A7DC7C237D00795E
:10A6A000007414122B8E1232C6901A89E07009744D
:10A6B0001E122E0074018006741E122E00E412A7D2
:10A6C000ED740FF0901CE812CFBF7946123B607416
:10A6D00001122E00E4F0901CBCE0C0E07402122EC7
:10A6E00000D0E0F0901A66E0C0E07403122E00D0B3
:10A6F000E0F07404122E00E4F07405122E00E4F071
:10A700007407122E00E4F0901A89E0C3940F500CE5
:10A71000E0C0E07406122E00D0E080077406122E0E
:10A7200000740FF07C8A7D1A7408122E00AA82AB86
:10A73000831234887C037D0079FF7410122E00AAE6
:10A7400082AB831232C6901AC2E0C0E07413122E9C
:10A7500000D0E012CBC97401122B8E1242AA7AC625
:10A760007B1A7945123B601243BE901A7DE0C0E02F
:10A77000741C122E00D0E0F0901A7EE0C0E0741D30
:10A78000122E00D0E0F0901A6BE0C0E0741A122E86
:10A7900000D0E01287877418122E0012CC98742013
:10A7A000122E00E4F0901A80E0C0E0741F122E0018
:10A7B000D0E0F07434122E00E4F07429122E00E47C
:10A7C00012A7E5123B607A6C7B1A794B123B6074DE
:10A7D00014122B8E123B7E743702B3EAF0A3E4F01E
:10A7E000A3F0A3F022F07A697B1A79532212A7F121
:10A7F00022F085188285198322C082C0838A828BC9
:10A8000083A3E0901A786004E4F080707408F090FC
:10A810001A89E07028901A0C12CF8860087900120B
:10A82000C8AA124A89901A7612B9A47A057B001236
:10A830003296901A7612CC8912450E801879001241
:10A840003DCA901A6912B9A47A067B001232961298
:10A85000A87F123296901AFC12CF88601F9019DAE6
:10A86000E06401701790811712294B7A007B4090A9
:10A870001AC3E0F91234467404122AE802C575902E
:10A880001A6C12B9A87A047B002274F4122517748A
:10A89000EA122BB68A088B09EA2402FAE43509FB8E
:10A8A000123CBC8A0A8B0BAE0AAF0BEE4F70030250
:10A8B000A98E8E828F83A3A3A3A3E06401602A8E56
:10A8C000828F83A3A3A3A3E06402601D8E828F8383
:10A8D000A3A3A3A3E0640360108E828F83A3A3A32A
:10A8E000A3E06404600302A98EE5082402FCE435B9
:10A8F00009FD740B122E00AA82AB8312348812A9B0
:10A9000093122E0012CC987415122E007401F0745C
:10A9100008122E00E412CFBF124A7EE9FC7D007AB5
:10A92000077B001232968E828F83A3A3A3A3A3E09A
:10A93000C2E012A99D740112E96C5001097A027BF0
:10A9400000122331E88E828F83A3A3A3A3A3A3A322
:10A95000A3F09019DAE0640170349019D4E0640235
:10A96000702C8E828F83A3A3A3A3E06401600D8E5D
:10A97000828F83A3A3A3A3E06402701212B95D12B5
:10A980002DDD12C24C122DE9EE241B12CF6F74166E
:10A99000028FBB8E828F8312D53B74132212A9A122
:10A9A0002212C282A3A3A3A32274F212251774F861
:10A9B000122BB6EAFEEBFF8C0A8D0B890D9080EA14
:10A9C000AC18AD197408122A4C750C00EEFCEFFDA2
:10A9D000AA18AB19123482E97003750C01901AC4DD
:10A9E000801AEEFCEFFDE508240BFAE43509FB12B2
:10A9F0003482E97023E508241412CC7512AA2E6063
:10AA000024E50CA2E040DB850882850983E0650A25
:10AA10007004A3E0650B70DD850882850983A3A31C
:10AA2000E0650D70D0AA08AB097408028B2D12875F
:10AA300035E508450922C082C083901AC402C57258
:10AA400074F7122517901AC412F0F2800C12D7A1D5
:10AA500012BC60123386EEFAEFFBEA4B70EF901AED
:10AA6000C4E4F0A3F002B3ED74F4122517EAFEEB90
:10AA7000FFEE241312B9696403700CEE240BFAE4A0
:10AA80003FFB123CBC800EE06402707C12CC63126F
:10AA9000CC89123CB68A088B09E508450960698EA5
:10AAA000828F83A3E0700F850882850983A3A3A307
:10AAB000A3A3A3E4805164F1600A8E828F83A3E094
:10AAC00064E17027850882850983A3A3A3A3A3A3B8
:10AAD000E06401701685088285098312CC89123ED4
:10AAE000A8EE240BFAE43FFB123CC88508828509D6
:10AAF00083A3A3A3A3A3A3E0600E85088285098393
:10AB0000A3A3A3A3A3A314F0028FBE74F11225176D
:10AB10008A088B09ECFEEDFF890A8A828B8312DB9F
:10AB2000DC8A828B8312A1A912ABDD8A828B83A37C
:10AB3000A3E0C454F0FA88828983E04A12ABED1294
:10AB4000A1A912ABE7E0333354FCF88E828F83E087
:10AB50004812ABE7A3E033333354F8F88E828F8387
:10AB6000E04812ABDD8508828B83A3A3A3A3A3A334
:10AB7000E0A2E0E4331313FA88828983E04AF0E527
:10AB8000082407F50CE43509F50D750E00780C1254
:10AB90002B227C087D00EEFAEFFB1232BA7403120E
:10ABA0002AE8EE2408FE50010FE508240FF50CE416
:10ABB0003509F50D780C122B227C037D00EEFAEF9F
:10ABC000FB1232BA7403122AE8E50AC3940F400A52
:10ABD00012CC7112A1AAA3A3A3F002E93EF0EEF8F1
:10ABE000EFF9A30EAF832212ABEDA3A322F08508E9
:10ABF000828B83A3A32274F1122517EAFEEBFF894F
:10AC00000A8C088D098E828F83E08C828D8312BF1F
:10AC100089AE82AF83E012C33812C522C412C33892
:10AC200012ACB5E012C33F12C520A2E2E4338C821D
:10AC30008D8312C51F131313541F12C33812C51E60
:10AC4000A2E7E4338C828D83A3A3A3A312ACB58EB9
:10AC50000C8F0D750E00780C122B227C087D00E500
:10AC6000082407FAE43509FB1232BA7403122AE801
:10AC7000EE2408FE50010F8E0C8F0D780C122B2243
:10AC80007C037D00E508240FFAE43509FB1232BA93
:10AC90007403122AE8E50AC3940F40118E828F8351
:10ACA000A3A3A3E0C0E012CC71D0E0800412CC7169
:10ACB000E4F002E93EA3A312BF8D0EAF832274F528
:10ACC0001225178A088B098A828B83A3AE82AF83F1
:10ACD000E0F9123DF48E828F83E064EB60248508F6
:10ACE00082850983A3E064E1601885088285098371
:10ACF000A3E064F1600C850882850983A3E0641AEF
:10AD00007009850882850983A3E4F0901CA3122DA5
:10AD1000D1124232750A01780A122B2A85088285DF
:10AD20000983A3E0F5087808122B2A7900901A7697
:10AD300012AD4412CC8912438E7402122AE81242D8
:10AD4000C802B65D12B9A8901A6C22C082C083E90D
:10AD5000901AD67003E480027401801EE0F902C5E7
:10AD600075C082C0837C207D428A828B8312CC890D
:10AD7000123B8A02C575EAF0A3EBF002C57574F6C2
:10AD8000122517901AD6E0701B7C0079017A007B9F
:10AD9000001242F8EA4B600C8A828B8312CF8860E3
:10ADA0000312422602C907C082C08379041242F20C
:10ADB000E9F890506CE493C398401079FF1242F286
:10ADC000E9F890506BE493C39850047901800279BC
:10ADD0000002C57574F01225178A088B09890B7556
:10ADE0000C008A828B83A3A3A3A3A3A3A3A3E0F94C
:10ADF0001242FE8A0E8B0FAE0EAF0F750A01EE4F98
:10AE0000600302AEBF85088285098312AFFDA3A34C
:10AE1000A3A3A3A312C04612CC891242E68A0C8BCC
:10AE20000DAE0CAF0DEE4F700302AFE88E828F8334
:10AE3000A3A3A3A3E4F0A3F0E508240CFAE43509E6
:10AE4000FB8A828B83E0C0E012E962D0E0F0E50883
:10AE5000240D12AFF512DBAA12CC9812441EEE2478
:10AE60000F12E154E508241112AFF512890F12CC2C
:10AE700098E508241312AFF0C0E012B95DD0E0F0FD
:10AE8000750C01EE240612BF3EE0547FF0A3E0549F
:10AE9000FC12E69AE05404600302AF36901CB5E061
:10AEA000F50875090074077808122CBF8E828F830D
:10AEB000A3A3A3A3A3A3E04508F0A3E04509F08E54
:10AEC000828F83A3A3A3A312872F74077808122D60
:10AED0008EE5085407FCE50B606C8E828F83A3A37C
:10AEE000A3A3A3A3A3A3A3740212C52312B2C46095
:10AEF0000B901A6412B00EA3A312CC98EC7003024C
:10AF0000AFB1EE240612F440547FF508A3E054FCE0
:10AF1000F509EC24FFF50EE434FFF50F7407780E05
:10AF2000122CBFE508450EF8E509450FF98A828B1A
:10AF30008312CC98807B8E828F83A3A3A3A3A3A329
:10AF4000E0448002AEBEEC7005750A0080638E821C
:10AF50008F83A3A3A3A3A3A3E05420600C1232D831
:10AF6000EA547F7900245F80198E828F83A3A3A384
:10AF7000A3A3A3E05410601A1232D8EA540F790048
:10AF8000240A5001098E828F83A3A3A3A3F0A3E90F
:10AF9000800D8E828F83A3A3A3A37401F0A3E41278
:10AFA000A99D7404F07A207B00901AC3E0F9123353
:10AFB00020E50CA2E0503412B9BDA3A3A3A3A3A320
:10AFC000A3A3A3E0F9EEFAEFFB1242ECE9601C1236
:10AFD000ED483F12CF86600912B51B12CC8912339F
:10AFE00086EEFAEFFB123386750A00A90A02D92C05
:10AFF00012BF66E02212BF6612D53BEE22A3A3A3C6
:10B00000A3A3A312B9A8850882850983A32212D518
:10B010003B8E828F83A3A32274F412251774F71238
:10B020002BB67E001242FEEA4B700302B0D48A8235
:10B030008B83A3A3A3A3A3A3A3A3A3E0640660039A
:10B0400002B0D48A828B83A3A3A3A3A3A3A3E0FF0C
:10B050008A828B8312B0DBE0C0E07408122E00D02D
:10B06000E012B50212CC8E12431CEF5408606385C7
:10B07000188285198312B9A47A007B001242E08BF2
:10B080000BEA450B704C12F59A123BA27C007D0036
:10B090007A007B0080288E828F8312B4F1F47003D3
:10B0A000A3E0F4602D901A7612B9C512CC89123B38
:10B0B0009CE9641A601C7C007D00EEFAEFFB1242F2
:10B0C000E08A0A8B0BAE0AAF0BEE4F70C979001203
:10B0D0003BA87E01EEF97409028FBB12BC6912B065
:10B0E000E2222408F582E438F58322C082C083EA94
:10B0F0004B7005901ADB80068A828B83A3A312B261
:10B10000F860258A828B83A3A3A3A3A3A3A3E054FF
:10B110000860E5EC4D60158A828B8312B4F16C7087
:10B1200003A3E06D70D280047A007B0002C57574C1
:10B13000F2122517EAFEEBFF890A8C088D097A14B2
:10B140007B00123380EA4B603F8A828B83A3A3A3E8
:10B15000A3A3A3A3A3A3E412B4F7A3E50A12B19493
:10B16000A3A312DD178A828B83A3A3A3A3E4F0A376
:10B1700012B51512B1A612E0F2EA12ED493BF583C1
:10B18000E4F012B18BF0A3F0028B30A3F08A828B33
:10B1900083A3A32212B1982212B19C22F08A828B3F
:10B1A00083A3A3A3A322A3F012F4613BF583E4F0ED
:10B1B0002274F4122517EAFEEBFF89088C0A8D0B26
:10B1C000EE4F700302B24D740165087012790112DE
:10B1D00042F2E9F890506DE493C3985022801674BF
:10B1E000046508701479041242F2E9F890506CE496
:10B1F00093C398500A7911805674026508704E8E78
:10B20000828F83A3A3A3A3A3A3A3A3A3E50812B937
:10B21000CD12DBB7E4F0A3F0901ADB12CF886017F1
:10B220008003E0F8A312CD8FA3A312B2F88882891D
:10B2300083A3A370ED8003901ADB12E0F67A207BE3
:10B2400000901AC3E0F91233207900800279C1021C
:10B250008FBEC082C083E9F87900901ADB801D8A16
:10B26000828B83A3A3A3A3A3A3A3A3A3E0686005E6
:10B2700074FF687001098A828B83A3A312B2F870ED
:10B28000DE02C57574F7122517EA4B7005901ADBBC
:10B2900080068A828B83A3A312B2F860208A828BF5
:10B2A00083A3A3A3A3A3A3A3A3A3E06970E4EC6077
:10B2B000108A828B83E012B2C470D780047A007B3C
:10B2C0000002B3ED12F496E0540422C082C08390D1
:10B2D0001ADB80068A828B83A3A312B2F860128ADB
:10B2E000828B83A3A3A3A3A3A3A3A3E06970E58098
:10B2F000047A007B0002C57512D1BDEA4B2274F7B7
:10B30000122517EAFCEBFD901ADB80068A828B83FC
:10B31000A3A312B2F860248A828B8312B4F16C70FA
:10B3200003A3E06D70E68A828B83A3E0C812BC564B
:10B3300012D918A2E0E43370D380047A007B0002B3
:10B34000B3ED74F21225178A0A8B0B8C0C8D0D75D8
:10B350000800750900EA450B6030901ADB80068E04
:10B36000828F83A3A312BC60EE4F601EAC0CAD0DA8
:10B37000EEFAEFFB850A82850B83124A89E96401A4
:10B3800070DDEEF8EFF988088909AA08AB09028B8D
:10B39000307900022AD074F7122517901ADB12BAFE
:10B3A000D27C007D00800DE8FCE9FD88828983A3C2
:10B3B000A312BAD2E8496030EA687002EB6970E71C
:10B3C000901ADB12CC89E86A7002E96B8882898363
:10B3D000A3A3700812BAD2901ADB800912BAD28CD9
:10B3E000828D83A3A312CC988003122AE87F0102E6
:10B3F000284374F7122517EAFEEBFFEE4F602F1279
:10B40000431612B43012CC891233868E828F831287
:10B41000CC8912338612ED483F12CF86600912B5EF
:10B420001B12CC89123386EEFAEFFB12338680BDF5
:10B4300012CF8EF5832274F61225178A828B83121F
:10B44000B4F1F508A3E0F509901ADB12BAD27D0039
:10B450007C00802F88828983A3A3A3A3A3A3A3A393
:10B46000A3E0640570140C12DBD3F5838E82E065D3
:10B47000087004A3E0650970010D88828983A3A385
:10B4800012BAD2E84970CD905069E493F8EDC398B0
:10B49000500890506812EED0400F8A828B83A3A38D
:10B4A000A3A37401F0A3E48010901A64E0F812A63C
:10B4B00059A3A3A3A3E8F0A3E912B515740512B428
:10B4C000F7E0440812B502F47003A3E0F4601190B1
:10B4D0001A7612D8FB12CC89123B9CE9641A7005CB
:10B4E0007901123BA802C907EE241DF582E43FF55D
:10B4F00083E0F812B50D2212B4FB2212B19CA3A373
:10B50000A322F08A828B8312B50B22E0F8A3E0F528
:10B51000838882E02212B4FBA3A322EE12CD742210
:10B52000C082C083EAFCEBFDEC4D6017EC24FBF518
:10B5300082ED34FF12CF86700712B57AE0F460070F
:10B540001232E479058030901AC3E0C0E012B57A77
:10B55000D0E0F090505FE493F97ADD7B1A12331A51
:10B56000E9640170107A007B20901AC3E0F912336D
:10B570002079008002790402C575EC24FFF582ED84
:10B5800034FFF5832274F4122517A2AFE433F508D3
:10B59000C2AF901ADD12BC60EE4F603AEE24FBF5AC
:10B5A00082EF34FF12CF867A007B20901AC36007A7
:10B5B000E0F91233208005E0F9123326E4F50AF5AC
:10B5C0000B780A122B26EEFCEFFD7ADD7B1A123384
:10B5D000147402122AE8E508A2E092AFEEFAEFFB3B
:10B5E000028FBE74F51225178A088B09750A009020
:10B5F0001ADB12DBD7805A8E828F8312B4F1650872
:10B600007004A3E06509703D8E828F83A3A3A3A37A
:10B61000E4F0A312C293540460118E828F83A3A31B
:10B62000A3A3A3A3A3A3E0F9123F1A8E828F83A33F
:10B63000A3A3A3A3A3A3A3A37406F07AF012891C67
:10B6400012422C050A8E828F83A3A312BAD2E8FE7F
:10B65000E9FFEE4F70A1A90A8003122AE87F0302D6
:10B66000284374F012251774D4122BB6EAFEEBFFB0
:10B67000750B00750A007508FE7509FF1242CEE9C8
:10B68000600302B950EE241512B9696044901CD2CF
:10B69000E0C43354E0F8E0333354FC48C0E012D740
:10B6A0002AD0E012B9CD12CC8979FF12401C8B0D43
:10B6B000EA450D600F750B017508FF12CF7312CEAE
:10B6C00049D2E0F09019E6E0600464017003750A65
:10B6D000408E828F8312CC87124412E9600312B924
:10B6E00075EE241312B969700D905056E493C0E0C2
:10B6F00012B95DD0E0F08E828F83E0A2E75004544F
:10B70000038019EE241412B9697012901A55E0C022
:10B71000E012F436D0E0F0901A55E004F012F45242
:10B720007016901CBEE0600D901A60E0700A8E8268
:10B730008F83E0700312CD649019E6E06004640129
:10B74000704B901A63E0A2E15043E50BA2E0402168
:10B750008E828F8312CC87124412E960308E828FE2
:10B7600083E0600DEE240B12B4EBF91243EEE960B6
:10B770001C12B981700302B902EE241312B9696474
:10B7800001600302B90212B51BE054FBF08E828FF8
:10B7900083E06401700DEE240B12B4EB64027003BD
:10B7A00012B98E12B981600302B868E50BA2E050AD
:10B7B0000302B8689019E6E060076401600302B80C
:10B7C00068901A63E0A2E1400302B868E50AF50B4D
:10B7D000780B122B2AEE2406FCE43FFD8E828F8329
:10B7E00012CC87EE2412129BC9123F447401122A14
:10B7F000E8E9600612B97512B9878E828F83A3A318
:10B80000A3A3A3A3E0603CEE2402F50CE43FF50DF6
:10B81000850C8212B9B22407FAE43FFB1243528A24
:10B82000088B09850C82850D83E065087004A3E010
:10B830006509700C8E828F83A3A3A3A3A3A3E4F056
:10B8400012B98E8E828F83E06401600BA90A12B94F
:10B85000C112CC87123EE4A90A12B9BD12CC8712DC
:10B860003E72E9600312B987AC18AD19EEFAEFFB2E
:10B8700012434C8A0A8B0B74FE6508700474FF65D2
:10B8800009700312872BEA450B700302B9548E82AC
:10B890008F83E0C0E07401122E00D0E0F074041237
:10B8A0002E0012E0F6EE241E12BACC7402122E0004
:10B8B00012CC987401122B86880C890D780C122BEF
:10B8C00026EE242012B96D122B2A12B51B12295311
:10B8D000EE240E12B96D122B2A901A691229537494
:10B8E00008122E00E0F9AC08AD09124346740812A4
:10B8F0002AE8E9FE74106E705DAA0AAB0B1233865B
:10B900008054EE241312B969C0E07417122E00D0CF
:10B91000E012F4A7740F122E0012B9D3240412F40B
:10B920004512BAD27411122E00E8F0A3E912BFAE8C
:10B93000C0E07418122E00D0E012E95812A65A1274
:10B94000B9A47406122B8E123F14E9600302B78D5E
:10B95000791180047E10EEF9742C02D92912B96194
:10B9600022EE12CDAC22EE241712BF4E2212BF4E91
:10B97000F50C780C22EE2412F582E43FF583E4F016
:10B980002212B99554402212B9954420F02212B9DE
:10B99000954440F022EE12CD78E022EE2413F58299
:10B9A000E43FF58312B9A82212B9AC22E0FCA3E06F
:10B9B000FD22F58312B9B82212B9ACEE228E828F25
:10B9C00083A3A3A3A312B9A88E828F832212DBC301
:10B9D00022A3A3E8F0A3E9F0EE22C082C08374D7CB
:10B9E000122BB69080007403122B967426122A4CE8
:10B9F0008A828B83A3A3A3A312BAD2740E122E0041
:10BA0000E8F0A3E912D534740C122E0012BAD62431
:10BA10000D12BAC1C0E0741A122E00D0E0F012D795
:10BA2000AB12BAD07420122E0012BAD6241512BA54
:10BA3000C1C0E07408122E00D0E0F0EA241CF582A8
:10BA4000E43B12BAD07412122E0012BAD62411128C
:10BA5000BAC1C0E07409122E00D0E0F0EA2412123C
:10BA6000BAC1C0E07407122E00D0E0F0EA241EF53F
:10BA700082E43B12BAD07424122E0012BAD62420CB
:10BA800012BAC1C0E07426122E00D0E012A7ED74E5
:10BA9000FFF07401122E0074FFF07402122E007475
:10BAA000FFF090814712294B7404122B96740712F1
:10BAB0002B8E123DB87404122AE87900742902D53D
:10BAC00078F582E43BF583E022EE2413F582E43F2F
:10BAD000F58312D53B22E8F0A3E9F0EA2274EE12D6
:10BAE000251774EC122BB68A0E8B0F8C088D0989E2
:10BAF0000C750A107A217B0012338012D57EE8493A
:10BB0000700302BC4F750B007C217D007900851805
:10BB100082851983E0FA1232C67429122E0012BCF3
:10BB2000609019E6E060046401703EAA08AB091257
:10BB30003CB68A108B11A810A911E84960238882AD
:10BB40008983A3A3A3A3E06401600D88828983A3F2
:10BB5000A3A3A3E064037009EE5440700474044F7F
:10BB6000FFEF54046003750B01901A7612CC89859F
:10BB7000188285198312BC652409F582E43812E124
:10BB8000587426122E0012BAD27411122E00E8F048
:10BB9000A3E912BC6E12F45812BC6E12B0E2740229
:10BBA00012F4B2F8A312C8AA12DE8112BC6E12F40B
:10BBB00068E50CF07428122E00E0F50885188285DF
:10BBC000198312F471E50812BC6E12BC56F583E5B8
:10BBD0000EF0A3E50FF07406122E0012E0F67408C2
:10BBE000122E00E508F0742C122E0012E2EEC08234
:10BBF000C083740C122E00AC82AD83D083D08274CB
:10BC000005122A4C742B122E00E0C0E07413122E81
:10BC100000D0E0F0A90BAA18AB191242D4E96401D4
:10BC200070219019E6E0600464017012E50BA2E057
:10BC3000500CA9081242FEEA4B6003124322750A17
:10BC400000800C85188285198312CC89123386A94D
:10BC50000A741402C299241FF582E43822A3A3A314
:10BC600012DBD7FF2212BC692212D598C82212D546
:10BC70008DC82274EE122517EAFEEBFF8C088D09A1
:10BC80008E828F83A37408F0EE241612B9696008BF
:10BC90008E828F83A37410F012B96660098E828F32
:10BCA00083A3E02408F0EE241512B96960088E829F
:10BCB0008F83A3E004F08E828F83A3A3A3A3A3A307
:10BCC000E060198E828F83A3A3A3A3A3A3A3E0C3E1
:10BCD000332402F88E828F83A3E028F012BF4760DE
:10BCE00005750B0E8003750B009019E6E064027079
:10BCF0001E9019DAE0640170168E828F83E0640171
:10BD0000600D9019D4E0600712BF347401800412F2
:10BD1000BF34E412BF89E012BF5628250B8C828DF8
:10BD200083F012BF476013901A61E0F91241F6E9FF
:10BD3000F8850882850983E029F0850882850983D2
:10BD4000E0C39475400975080075090002BF2DE035
:10BD5000FA7B001233808A088B09EA4509700302D6
:10BD6000BF2D8E828F83E0FA901A6612BF82740212
:10BD7000780C122CBFEA450CFAAB0DEE241212B966
:10BD8000695403F50C750D007406780C122CBFEA8B
:10BD9000450CFCEBFDEE241512B9696004780180B6
:10BDA000027800EE2416FAE43FFBE8F9ED49FD12B3
:10BDB000BF47F50C7409780C122CBFED450DFD8AB8
:10BDC000828B8312BF82740B780C122CBFED450D51
:10BDD000FDEE241712BF7C740C780C122CBFED45BD
:10BDE0000DFD8E828F83A3A3A3A3A3A312BF82748E
:10BDF0000A780C122CBFED450DFDEE242312BF7CFA
:10BE0000740D780C122CBFECF8ED450DF9E885089F
:10BE100082850983F0E9A3F0EE240212BF3E12C02E
:10BE20005012BFA4F0EE240412BF3E12BF6E12BF28
:10BE3000A4A3A312CDA212BF6EA3A3A3A312BFAE4D
:10BE4000850882850983A3A3A3A3A3A3A3F0750AEE
:10BE5000088A828B83E06015EE241812B99EE508EB
:10BE60002408FAE43509FB123488750A1012B96601
:10BE70006019EE241A12B99EA80AE50828FAE435DA
:10BE800009FB1234887408250AF50A8E828F83A371
:10BE9000A3A3A3A3A3E06057EE2407F510E43FF5A6
:10BEA00011851082F583E0C0E012BF5DD0E012BFC3
:10BEB00094E0C0E00812BF5FD0E012BF94129B165E
:10BEC000122B22851082851183E025E0FCE433FDEE
:10BED000A80AE50828FAE43509FB1232BA740312FD
:10BEE0002AE8851082851183E0C333250AF50AEE1E
:10BEF000241512B9696008C0E012BF5DD0E0F012ED
:10BF0000CC63129B17122B2212BF57FC7D00A80B8B
:10BF10008E828F83A3E0FAE5082AFAE43509FBEA6A
:10BF200028FAE43BFB1232BA7403122AE8AA08ABDF
:10BF30000902C29CEE2423F582E43FF58322F8E453
:10BF40003FF9888289832212BF4B22EE2411F582A9
:10BF5000E43FF583E022F8EE12DBAEE022A80AE52A
:10BF6000082812BF6622F582E43509F5832212BF44
:10BF70007222E0850882850983A3A322F582E43F2B
:10BF8000F583E0F50C750D002212BF8D22F08E8234
:10BF90008F83A322F0050A8E828F83A3A3A3A3A37A
:10BFA000A3A3A322A3A312E6AA12BF72A322F0EEB8
:10BFB000241412BF4E2274F412251774FD122BB6EE
:10BFC0008A088B09ECFEEDFF7401122B86880A8922
:10BFD0000B780A122B267402122B96EEFAEFFB1244
:10BFE0003EC07402122AE8E97053851882851983CD
:10BFF00012C050F07401122E00E0F812C046A3A344
:10C0000012F4AE602914850882850983A312F4B264
:10C0100012DA327401122E00E028F8A3E039F9E8B0
:10C0200024FEF582E934FFF58312F0F2800C8508D6
:10C0300082850983A3E4F0EEFAEFFB80047AFE7BAD
:10C04000FF7403028FBBA3E0F98508828509832270
:10C05000E08508828509832274EE1225178A0A8BEF
:10C060000B8910ECFEEDFF750F017C267D00790039
:10C07000EEFAEFFB1232C6E510C39408500302C17A
:10C08000E58E828F83E510F0EEFCEFFD850A828558
:10C090000B8312C4F012435EE96003750F0012C4F3
:10C0A000D28E828F8312C52AEE12C4C63F12C514E7
:10C0B000C0E012890ED0E012C50CC0E0EE2412F5EB
:10C0C00082E43FF583D0E012BF89740812C27AA3DC
:10C0D000A3E06018E50A2408F8E4350BF912B95D0D
:10C0E00012CC988E828F83A3E02408F08E828F83F7
:10C0F000A3A3A3A3A3A3A3A3E060178E828F83A30C
:10C1000085820885830912C4E512D72A12A309245F
:10C1100008F0EE241912B978EE241B12B978A31294
:10C12000C27AE0600F12C2618E828F83A3A3A3A3A1
:10C13000A312C28DEE241812B969700302C1D51280
:10C14000C261FAEE2419F582E43FF583EA12C28D4A
:10C15000F8E50A28F582E412F594F812DCEBE8120F
:10C16000C28DE8C39AEE5068241912B969F890504C
:10C1700060E493C398500575110C8008EE241912E1
:10C18000B969F5118E828F83A3E0F8E50A28F50CD2
:10C19000E4350BF50D750E00780C122B22AC11EC6A
:10C1A0002CFCE433FD7A817B0A1232BA7403122A22
:10C1B000E8EE241BF582E43FF5837481F0A3740A52
:10C1C000F0E511C333F8850882850983E0288004EF
:10C1D00012CD5BE4F08E828F83A3E0F88E828F8392
:10C1E000E0C398500479008061A3E0FAE50A28F8DA
:10C1F000E4350B12C256E8F0A3E912C523C39AC076
:10C20000E012C24CD0E012C293603DEE2417F8E475
:10C210003FF9880889098882F583E024F2F0EE244A
:10C220001D12BF3EE0240EFAA3E03400FB88828991
:10C230008312E15A901A61E0F91241F6E9F8850893
:10C2400082850983E0C398F0A90F8050EE2417F58A
:10C2500082E43FF58322F9EE241DF582E43FF58365
:10C26000228E828F83A3858208858309E0F8E50A00
:10C2700028F582E4350BF583E02212C27E2212C239
:10C280008222F08E828F83A3A3A3A3A32212A311E1
:10C2900004F02212C27EA3E022122AE87F0A0228BA
:10C2A0004374F41225178A088B09EA12C33FA3A32B
:10C2B000F0EA1313543F12C338A3A3A3F0EAC41344
:10C2C0001312C33F12C3527409780A122D8E12C37F
:10C2D00046A3A3A3A3A3A3F0EB12C34812C35174B4
:10C2E0000A780A122D8EE50A5401C0E0EC2418F5F4
:10C2F00082E43DF583D0E012C356740B780A122D08
:10C300008E12C34612C34F740C780A122D8E12C3BC
:10C3100046A312C34F740D780A122D8EE50A5401FC
:10C32000C0E0EC2424F582E43DF583D0E0F0740E07
:10C330007808122D8E028909540F8C828D83225425
:10C34000038C828D8322E50A54018C828D8322A383
:10C35000A3A3A3A3A3A3F08A0A8B0B22C082C0834A
:10C3600079008A828B83A3A3A3A3A3A3E0901A607E
:10C37000600EE070238A828B83A3A3E0701A80167C
:10C38000E060158A828B8312CC80901A69E06A7013
:10C3900003A3E06B6002790102C57574F2122517E0
:10C3A0008A0A8B0B890C8C088D098A828B8312C4B4
:10C3B000F012435E12C4D285088285098312C52A11
:10C3C000E50812C4C6350912C514C0E0E5082411F9
:10C3D00012CC75D0E012C50CC0E012CC71D0E012C6
:10C3E000CF9C740812C4FEE06017E50A2408F8E444
:10C3F000350BF9E508241312C4CA12CF9CE02408B7
:10C40000F0850882850983A3A3A3A3A3A3A3A3E024
:10C410006017850882850983A312C4E1E508241505
:10C4200012C4CA12C5232408F0850882850983A393
:10C43000A3A3A3A3E06019850882850983A3AE8224
:10C44000AF8312C26C85088285098312C51E04F071
:10C45000AA08AB09124364E9F50D7064850882856A
:10C460000983A3A3A3A3A3A312C050A3701AE0FA45
:10C47000E50A2AF8E4350BF9E508241D12CC7512FB
:10C48000CC98E50CC39A802C12C4E1E8240EF85035
:10C490000109E508241D12CC7512CC98901A61E0B0
:10C4A000F91241F6E9F88E828F83E0F9E50CC39921
:10C4B00024F2C398C0E0E508241712CC75D0E0F050
:10C4C000A90D028B30EA12F4622212BF66E8F0A3D3
:10C4D000E922850A82850B83A3A312C540E0F9EA0D
:10C4E00022AE82AF83E0F8E50A28F8E4350BF922A2
:10C4F000E0FAA3E0F8E4C8F9EA28E439FB2212C51F
:10C50000022212CFA4A3A3A3A3A3A32212C553A3C1
:10C51000A3A3E022F583E812C54CA3A3E022A3A3C2
:10C52000A3A3A3F08E828F83E022A3A3A3A3A3A33C
:10C53000A3A3A312C54C12C540A3A3E0F9EAF822B5
:10C54000E0FA850A82850B83A3A3A322F0A3E91254
:10C55000C55322F0850A82850B83A3A3A3A322C01F
:10C5600082C0837AEB7B1A79E2123B5A7AEB7B1A10
:10C57000800312CC89D083D082022AD0C082C083AB
:10C58000901A6980EDC082C083901A6C80E4C082EA
:10C59000C083794A123B5A80DC74F6122517901A30
:10C5A000F3E0FE04F0EEF91242FE8B09EA45097051
:10C5B000EDEE60EAF902C90774EE122517EAFEEB08
:10C5C000FF8C0E8D0F890C750A00750B0012451437
:10C5D0008A088B097412122E00E0F50D7413122EC6
:10C5E00000E0F510EA45097017E510600302C6DAAD
:10C5F000A90CAC0EAD0FEEFAEFFB12453802C7D90D
:10C60000E510700302C6A59019E6E06004640170AD
:10C610000E901AF812CF88600612C8AA124A89E54D
:10C620000D700E850882850983E4F0750B0102C642
:10C63000FD9019E6E060076401600302C6FD901AF0
:10C6400063E0A2E1400302C6FD901AFA12CF8860AF
:10C650000CA90DAA08AB0912C8AA124A898508823A
:10C66000850983E0FA12E94D500109C3EA98E4997B
:10C67000A2D265D0335009850882850983E004F091
:10C68000850882850983E0F8905059E49368706DBD
:10C69000750A01EEFAEFFB123F5085088285098387
:10C6A000A3E4F08058E50D701CEA240212AFF0A854
:10C6B0000C28F8E4340013E813F070098A828B83A5
:10C6C000A3A37401F08A828B83A3A3E0F8901C5784
:10C6D000E0C3985052750B01804D74016510701DB8
:10C6E000E50D60199019E6E060046401700F901A7E
:10C6F00063E0A2E15007EEFAEFFB123F509019E61B
:10C70000E06402702274016510701CE50D901B0A34
:10C710006013E004F0901CB6E0F8901B0AE0C398A8
:10C720004005750A01E4F0E50BA2E092F0E50AA2EB
:10C73000E072F0400302C7D99019E6E0600464019A
:10C740007041901A63E0A2E15039EEFAEFFB123C1F
:10C75000B68A088B09A808A909E8496026E50BA252
:10C76000E0500D88828983A3A3A3A3A3E0C2E0F0D5
:10C77000E50AA2E0506388828983A3A3A3A3A3E070
:10C78000D2E0F0E50AA2E050509019E6E0600464BF
:10C7900001701D901A63E0A2E15015EEFAEFFB1252
:10C7A0003CA4E9600BEEFAEFFB7900123DEE802924
:10C7B000901A6CE06E7003A3E06F701DEEFAEFFB51
:10C7C0007901123DEE9019E6E06402700C7A017B6B
:10C7D00000901AC3E0F912344C02C29C74F4122582
:10C7E000178A088B098C0A8D0B9081877808122C88
:10C7F0000D700E7A017B00901AC3E0F9123320808D
:10C8000035901CA37808122D9DEA4509450A450B71
:10C8100060187808122B1E7A017B00901AC3E0F989
:10C820001234407404122AE8800C7A017B00901ABA
:10C83000C3E0F912344C028FBEC082C083901CA7A3
:10C8400002AD76C082C083901CA902AD7674F61248
:10C85000251775085575091A7808122B267C6E7DE8
:10C86000007A217B001233F87402122AE8E9F508F5
:10C87000123C80E942089019E6E060046401700609
:10C88000123CFEE942089004DA12CF88600912C80F
:10C89000AA124A89E94208124040E9FE123ACAE95E
:10C8A000F8E5084E48F9805F79C4E0F58388822274
:10C8B00074F612251712329075085575091A780802
:10C8C000122B2675086E7509007808122B267C003D
:10C8D0007D007A217B001234047404122AE8123C91
:10C8E000869019E6E0600464017003123D04900430
:10C8F000DC12CF88600612C8AA124A89124046127A
:10C900003ADC8003122AE87F0202284374F61225DB
:10C910001774FF122BB67E0075085575091A780832
:10C92000122B267C6E7D007A217B001233F8740274
:10C93000122AE8E9600302C9F17808122B2675086B
:10C940006E8E097808122B267C007D007A217B00F0
:10C9500012340A7404122AE8E9600302C9F1901A39
:10C9600069E064FE7003A3E0F4700302C9F17E0184
:10C97000901A78E064086005E06404706F8518829E
:10C98000851983EE12CFBF7942123B607A807B1A01
:10C990007943123B607A7D7B1A7947123B607A6E4D
:10C9A0007B1A794A123B607A6C7B1A794B123B6096
:10C9B0007A767B1A7950123B607A697B1A79531226
:10C9C0003B607A7E7B1A7954123B607A6B7B1A79D2
:10C9D000E1123B60901A63E0A2E35004D2F08002BF
:10C9E000C2F012CFB57952123B6080051232907EB0
:10C9F00000123C749019E6E0600464017003123D7B
:10CA0000169004DE12CF88600612C8AA124A891254
:10CA10004052EEF9740102C90474F6122517E9FEBA
:10CA2000A2E0502675085575091A7808122B26754C
:10CA3000086E7509007808122B267C007D007A218B
:10CA40007B001234047404122AE8EEA2E3500312AD
:10CA50003C7A9019E6E0600464017008EEA2E150AF
:10CA600003123D1CEEA2E2500E9004E012CF88604B
:10CA70000612C8AA124A8902C90774F61225177449
:10CA8000EC122BB67401122B96901CE8E0F97AC6D2
:10CA90007B1A1242B07405122E00E4F07407122EB5
:10CAA00000E4F07A04F9123C9290506EE493F8C3DB
:10CAB000EA98EB94005058123C6EE9705290505234
:10CAC00012CB6B60197A047903123C928A088B09A5
:10CAD00090506EE493F890505212CB755008740544
:10CAE000122E007401F090504C12CB6B60197A0238
:10CAF0007901123C928A088B0990506EE493F89069
:10CB0000504C12CB7550087407122E007401F0902F
:10CB10001CE8E0F97CC67D1A7401122B8E1242AA21
:10CB20007AC67B1A7945123B607407122E00E070BA
:10CB3000117405122E00E07009851882851983E4AE
:10CB400080088518828519837401F0901CE2E0F852
:10CB5000901CE1E058F8851882851983E05812CFBF
:10CB6000BF7941123B60741402C904E493F8740164
:10CB700093F9E84922E493FA740193FBE8C39AF825
:10CB8000E49BF9C3E50898E509992274F712251783
:10CB900074ED122BB6E9FE901AC2F0AC18AD1990E4
:10CBA0001CE8E0F97AC67B1A1242B07412122E0009
:10CBB000EE12CBC9AA18AB191242AA7AC67B1A790F
:10CBC00045123B60741302B3EAF0901CE8E0F97C74
:10CBD000C67D1A2274F4122517EAFEEBFF901CEAB8
:10CBE000E064FE7003A3E0F470767A167B001232E4
:10CBF000DE8A088B09EA450960668A828B837401A4
:10CC000012C2938A828B83A360047402800274012F
:10CC1000F0EA240AF8E4350912C25612F0F7A3121A
:10CC2000DCF5F0A2E3400912CC6312CC8912433444
:10CC3000EE241512B99EE5082402FAE43509FB1228
:10CC40003488E508241312CC75E4F0AA08AB0990E7
:10CC50001AC3E0F91232EA12CC6312D52D12CC9825
:10CC6000028FBE12CC6722EE240BF582E43FF583DF
:10CC700022E5082412F582E412BF69228E828F8396
:10CC8000A3A3A3A3A3A3A3A3A312D1BD22E0F8A3AC
:10CC9000E0F9851882851983E8F0A3E9F02274F29F
:10CCA00012251774FD122BB68A088B09890A8C0B82
:10CCB0007401122E00740412CFBF1243F48A0C8B3D
:10CCC0000DAE0CAF0DEE4F700302CD4C12CD817442
:10CCD0000712DCFBE5082413FAE43509FB8A828B92
:10CCE0008312CD978A828B8312CD96E50824151284
:10CCF000CC7512DCF512DD02E508240BF8E43509E9
:10CD0000F912CD5AE8F0A3E912DE9512437012DC55
:10CD1000E312CDA27401F07403650A600674016524
:10CD20000A700712CD6B7404800412CD6BE4F0908E
:10CD30001CEA12B00E12CC987401650B700312CD70
:10CD400064EEFAEFFB123D34E9F980027910901C91
:10CD5000EA74FEF0A304F0028B2BEE2418F582E4B3
:10CD60003FF58322EE128913E4F02212CD73744052
:10CD7000F0A322EE12CD7822240FF582E43FF58352
:10CD800022EE12F4623FF58312CD8C22E0F8A3E08C
:10CD9000F98882898322A3E088828983F0A308A985
:10CDA000832212CDA622F0EE12CDAC222413F582FE
:10CDB000E43FF5832274F4122517EAFEEBFF7A00B4
:10CDC0007B04901AC3E0F912344C12CE5C901A78AE
:10CDD0007409F01243708A088B09AC08AD0912B9C6
:10CDE0005D12CC89123482E96401705A7A0F7B009B
:10CDF0001232DE8A088B09EA4509604A8A828B83EF
:10CE0000740212CE51F988828983A3E0FC8882895A
:10CE100083A3A3E0FBEC8A82850983A3A312E15BD1
:10CE200088828983A3A3A3E08A82850983A312CE83
:10CE300049FAA3E0FB794A123B60AA08AB09901AB1
:10CE4000C3E0F91232EA028FBEF0EE241512BF4E93
:10CE500022F0EE241D12BF4EF8A3E022901A011218
:10CE6000D53B901CA9E8F0A3E9F0901A0312D53B3A
:10CE7000901CA7E8F0A3E9F02274F412251774FDC2
:10CE8000122BB68A088B097401122E00740212CF7D
:10CE9000BF1243F48A0A8B0BAE0AAF0BEE4F70033E
:10CEA00002CF6712F481E412CF9CA3A3A3E0640134
:10CEB000700888828983A37420F08508828509839D
:10CEC000A3A3A3A3A3E06401700988828983A3E0DC
:10CED000D2E6F0850882850983A3A3A3A3A3A3E0D8
:10CEE0006401700A88828983A3E0D2E7800512B9C1
:10CEF0005D740112CFADE06401702185088285095F
:10CF000083A3A312CF88600312CF6C8508828509A2
:10CF100083A3A312AFF812CD5B12CC98850882854B
:10CF20000983A3A3A3A3A3A3A3E06401700712EF43
:10CF3000F2F0A3E4F085088285098312CC891244BB
:10CF400012E9600412CF73F0EE241712CF6F124370
:10CF50007012DCE312A30D12CF7A12B9D1FAEFFBF3
:10CF6000123D34E9F98002791002C041EE24161214
:10CF7000DD0A2212B995440422E0F8A3E0F98E827A
:10CF80008F832212CF8EF58312D53BE849228E8201
:10CF90008F8312BC69241FF582E4382212CFA022AD
:10CFA00012CFA422F0850882850983A32212CFA084
:10CFB000A3A3A3A322A2F0E433851882851983F0EA
:10CFC000AA18AB192274F512251774F3122BB6891F
:10CFD0000AEAFEEBFF7508007509007C0D7D0079FB
:10CFE00000AA18AB191232C612C25712D174741F9C
:10CFF00058600C7AD37B001237BE790002D0C4E8A7
:10D00000A2E55008740C122E007401F0E8A2E7505B
:10D0100008740B122E007401F0E8A2E6740A50089E
:10D02000122E007401F08008122E00E064017013CB
:10D030008E828F83A3A3A3A3A3A3A3E06032EE24D5
:10D040001380128E828F83A3A3A3A3A3A3A3A3E021
:10D05000601EEE2415F582E43FF58312AA2E6010BF
:10D06000AC08AD097402122E00AA82AB8312348878
:10D0700012CC6312CC8D740A122E00E06401703B56
:10D0800012CC7C124412E97039EE240B12BACC9007
:10D090001A6CE0687003A3E0697027E50845096031
:10D0A0001A1243708A088B09AC08AD097402122E5B
:10D0B00000AA82AB83123482E96007AA18AB191266
:10D0C0003DE8A90A740D02B65A74F712251774CDFB
:10D0D000122BB6EAFEEBFF8E828F8312D192A2E072
:10D0E000400302D16F12D17BE054FE12ED5A740D51
:10D0F000122B9612D1A512436AE97073742A122E6C
:10D100000012D18870697C0D7D007900AA18AB19D6
:10D110001232C67416122E0012CC8D742A122E00F2
:10D1200012D174A2E55008740B122E007401F0E8BD
:10D13000A2E75008740A122E007401F0E8A2E6502B
:10D1400004742080027422122E0012B9A4740212F8
:10D150002E00AA82AB831234888E828F83A3A3E031
:10D16000C0E0740C122E00D0E012CFBF123DE2746A
:10D170003302B3EA12E2F2A3E0F8228E828F831226
:10D18000D91FA3A3A3A3A32212B50B6404228A82EE
:10D190008B83E0F812D19822A3E0C82406F582E43C
:10D1A00038F583E022EA241EF582E43BF583E0F9BA
:10D1B000EA241FF582E43BF58312D1BD2212F0F27E
:10D1C000FB22E9F87900740468600A740A68600553
:10D1D00074036870027901022AD074F61225178A46
:10D1E000828B837424F0A3A37401F0123D3A8A0861
:10D1F0008B09AE08AF09EE4F60108E828F8312DE6E
:10D2000093124370EE241A12E154EEFAEFFB02C9B6
:10D2100007C082C083901A6602AD5CC082C0839052
:10D220001CE902AD5CC082C083E9901CE902AD7AC2
:10D23000C082C083901ADF7401F0E9A2E350037446
:10D2400003F0E9A2E15004E0D2E2F002C57574F601
:10D2500012251779007C008A088B0978081227FDAF
:10D26000F8FF0783D281D281D281D281D279D27D57
:10D27000D283D275D27C01800A7C0480067C028035
:10D28000027C08901ADFE05C600479028005EC60A3
:10D2900002790102C90774F4122517EAFEEBFF892F
:10D2A00008123CBC8A0A8B0BA80AA90BE84960410A
:10D2B00088828983A3A3A3A3E06036C39405503179
:10D2C00074016508601A88828983A3A3A3A3E0641C
:10D2D00001600D88828983A3A3A3A3E06402700A7E
:10D2E0008882898312CC89123EA8EEFAEFFB123CA9
:10D2F000C8028FBE74F61225178A828B83E07014E1
:10D30000A3A3A312CF88600C8A828B8312CC8612CF
:10D3100040A080047A007B0002C907C082C08390CD
:10D320001A78E06408700312443602C575C082C0E2
:10D33000837C00EC75F003A4F8ADF0EDF912D40392
:10D340007003A3E06B701890505DE493C0E074E24A
:10D3500028F582741A3DF583D0E0F079C580620C1F
:10D36000ECC3940340CD7C00EC75F003A4F8A9F065
:10D3700074E328F582741A129AD664FE7003A3E04F
:10D38000F4600F0CECC3940340DE7C00EC12D3C4B9
:10D390007026EC75F003A4FCADF074E22CF8741A5E
:10D3A0003DF988828983A312E15A90505DE4938805
:10D3B000828983F0790080090CECC3940340CD7915
:10D3C000C702C57575F003A4F8A9F074E228F582C8
:10D3D000741A12EEE222C082C0837C00EC75F00366
:10D3E000A4F8A9F012D4037003A3E06B700912D360
:10D3F000CB6004790180090CECC3940340DE790012
:10D4000002C57574E328F582741A12EEE26A22747A
:10D41000F212251774DD122BB6EAFEEBFF75080039
:10D420009019E6E060076401600302D526901A694E
:10D43000E06E7003A3E06F7010EE4F700302D51A18
:10D4400075080112443C02D526123CB68A0A8B0BA1
:10D45000EA450B700302D51A8A828B83A3A3A3A388
:10D46000E0640160108A828B83A3A3A3A3E064021B
:10D47000600302D51A851882851983E412D53474A5
:10D480000B122E00E8F0A3E912CFBF123C62E97044
:10D490000302D51A850A82850B8312D52D12CC98EA
:10D4A0007900123E9C850A82850B8312DA48122E7F
:10D4B00000AC82AD837418122E00AA82AB831234A2
:10D4C00088850A82850B8312BAD27420122E00122C
:10D4D000CC987422122E00E4F07C02850A82850B1F
:10D4E00083A3A3A3A3E0F9740D122B8E1243D0855E
:10D4F0000A82850B8312BAD27401122E00E8F0A3BF
:10D50000E912CFBF123C68750801E50A240CF582C8
:10D51000E4350BF583129B39800C901A7612B9B45E
:10D52000FAEFFB1244FCA9087423028B2D12D53BA1
:10D53000901CEA2212B18C12D53B2212D598F92206
:10D54000C082C08374FE122BB69019E6E0600464BA
:10D550000170237901123EA212D57E901A69E8F07B
:10D56000A3E912CFBF7953123B60851882851983D6
:10D5700012CC891236E67402122AE802C5758518A3
:10D5800082851983EAF0A3EB12D58DF922F0851874
:10D590008285198312D59822E0F8A3E02274F41250
:10D5A000251774F3122BB68A088B09ECFEEDFF7574
:10D5B0000A12EA45097005790002D689901A69E0D5
:10D5C00065087004A3E06509701D1243708A0A8B18
:10D5D0000BAC0AAD0BEEFAEFFB123482E970057565
:10D5E0000A018003750A00851882851983E4F00416
:10D5F000122E0012DE8112CFBF123C56E9602A744F
:10D6000003122E00AA82AB83123C32E96401701926
:10D61000750A017403122E00AC82AD83EEFAEFFBA3
:10D62000123482E96003750A009019E6E060046430
:10D630000170177412650A7011EEFCEFFDAA08ABB9
:10D6400009123C9EE96003750A00EEFCEFFDAA0892
:10D65000AB0912451AE9F8740A687005750A018069
:10D660001D74A0687012EEFCEFFDAA08AB0912450C
:10D670002CAA08AB0912453E7401650A70097900AD
:10D68000AA08AB09124448A90A740D028FBB74F6AC
:10D69000122517EAFEEBFF89089019E6E0600464A2
:10D6A00001701E124436E508F5097809122B2A7913
:10D6B0000DEEFCEFFD7AFC7BFF1244547401122A3C
:10D6C000E802C90774F7122517EAFEEBFF8E828F76
:10D6D00083A3A3A3A3A3A3A3A3E0601612D72A1234
:10D6E0009BDB12CC89124442E96401700512CC63C1
:10D6F00080298E828F83A3A3A3A3A3A3A3E0602585
:10D7000012B99B12CC7C124442E9640170178E82DC
:10D710008F83A3A3A3A3A3A3A3A3A312CC8912447F
:10D720002A79018002790002B3EDEE2415F582E436
:10D730003FF5832274F212251774FD122BB68A0866
:10D740008B09ECFEEDFF890B750A017401122E00A6
:10D75000740412CFBF1243F4EA4B60427411122ECC
:10D7600000E0601412DDFAE412E2FA8A828B83E0B0
:10D77000D2E7F012D7A1E4F012D7AB12CD86740332
:10D7800012DA52EE88828983A3A3F0EF888289831C
:10D79000A3A312B18B12DD17123D34E9F50A028BF7
:10D7A00029EA2414F582E43BF5832212F4613B223A
:10D7B00074F0122517EAFEEBFF890A750B01EE12D1
:10D7C000DB143F12D918F50C88828983A3A3E0FAF1
:10D7D0008882898312D90712B9666404600A7AD3F1
:10D7E0007B001237BE02D8F7E50C1229D8020002DE
:10D7F00002D8030BAFD8030C95D80D6DD80EAFD857
:10D80000ACD89019E6E060076401600302D8AF90DD
:10D810001A63E0A2E1400302D8AF7900AB09123FDE
:10D8200032EA4B603D8A828B83A3A3A3A3A3A3E028
:10D830005418602E12CC631229538A828B83A3A3BF
:10D8400012295379008E828F83A3A3A3A3A3A3A33A
:10D85000A3A312D8FB12CC89123F4A7404122AE8FF
:10D86000802E7901AA08AB09123DFA80429019E690
:10D87000E0600464017038901A63E0A2E15030ABBC
:10D8800009124424AA08AB0912442AE964C5701F8E
:10D89000750B00801A9019E6E06004640170109026
:10D8A0001A63E0A2E1500812370A8003750A00EEFD
:10D8B0002409F50EE43FF50FAC08AD09A90C850E5F
:10D8C00082F58312CC89123E12850E82850F831257
:10D8D000CC89124412E9601F12BF47C3940240175B
:10D8E00012CC6312E21D7003A3E069600AE50BA28B
:10D8F000E05004A90A80027900803112D8FF221278
:10D90000B9AC8A828B8322A3A3A3E0F8E4C8F9EA26
:10D9100028F508E439F50922F58312D91FE022120F
:10D92000D598F988828983A322122AE87F080228E1
:10D930004374EE12251774F5122BB68A0A8B0B89E5
:10D940000D8C0E8D0F7E01EE122E00740AF0741DE8
:10D95000122E00E0F50CE9700FE50CC333240AC069
:10D96000E0EE122E00D0E0F0AA18AB191243F48AB0
:10D97000088B09EA4509700302DA2A12C4C5350981
:10D9800012DBC87409F0A3E50DC43354E0450C1252
:10D99000DBE1AC0EAD0FEEFAEFFB123488EE24089B
:10D9A000FE50010FE50D702F7C00741E122E001228
:10D9B000DA39801D12DA31EA28F8EB39F9888289E0
:10D9C0008312DBDC8882898312A1A9F0A30EAF83C6
:10D9D0000CECC3950C40DDE508241712CC757401DE
:10D9E000F0124370E508241AF582E4350912DA468C
:10D9F000122B96AA0AAB0B123C3EE96019E50824EB
:10DA00001612CC757401F07403122B86E5082418E5
:10DA100012CC7512CC98850882850983A3A312DAEB
:10DA200050AA08AB09123D34E9FEEEF9740B02C2AC
:10DA300099EC25E0F8E433F92212DA3D2212D59868
:10DA4000F9E8FAE9FB22F583EAF0A3EBF07403228C
:10DA5000E50AF0A3E50BF02274F012251774F81212
:10DA60002BB68A088B0912DB13350912DC5CF874BB
:10DA70001F58F50A880BA3AE82AF83EEFCEFFDAA18
:10DA800018AB19123488EE2408FE50010FAC18AD03
:10DA9000197A8A7B1A123482E9607374E0550B702C
:10DAA00066AA0AEA2AFA7B001233808A0C8B0DEAF6
:10DAB000450D605A7C00801D8E828F8312C4F01247
:10DAC000DA31E50C28F582E50D3912E158EE240231
:10DAD000FE50010F0CECC3950A40DD780C122B268A
:10DAE000780A122B2A7403122B967900E508240B6E
:10DAF00012CC7512CC8912446C7403122AE8AA0C59
:10DB0000AB0D12338680077AD37B001237BE7408C0
:10DB100002D929EA241DF582E42274F01225178A1D
:10DB20000A8B0B890D8C088D0990190612CF88601D
:10DB3000757410122E00E0F50C12DA32E8240EFA99
:10DB4000E439FB1232DE8A0E8B0FAE0EAF0FEE4FB2
:10DB500060548E828F8374D4F012DBB7A3A3E50DDB
:10DB6000F0AC08AD09EE2405FAE43FFB123488124C
:10DB7000DBA9E50CF07411122E0012E2E378081212
:10DB80002B22AC0CEC2CFCE433FDEE240EFAE43F2B
:10DB9000FB1232BA7403122AE8EEFAEFFB90190670
:10DBA00012E2EE124A8902D92CEE12DBAE22240DCB
:10DBB000F582E43FF58322A3A3E50AF0A3E50B1267
:10DBC000DBC32212BF8DA322F58312DBD7FF8E8227
:10DBD0008F832288828983E0FEA3E022E08E828FF9
:10DBE00083F0A3AE82AF832274F612251774F81265
:10DBF0002BB6890812DB133B12DC5CF9741F59F851
:10DC00008909A3AE82AF837401687042EEFCEFFD18
:10DC1000AA18AB19123488EE2408FE50010FAC1874
:10DC2000AD197A8A7B1A123482E9602974E05509A9
:10DC3000701C8E828F83A3E0FA8E828F83A312C41E
:10DC4000F28E828F83E0F912449CA90880097AD36E
:10DC50007B001237BE7900740802C904F583E02402
:10DC600001FEA3E03400FF8E828F83E02274F01265
:10DC7000251774FD122BB68A0A8B0B8C088D098927
:10DC80000D750C017401122E00740312CFBF1243E4
:10DC9000F48A0E8B0FAE0EAF0FEE4F603F12CD81A8
:10DCA000740BF0A3E50D12DCFB7413122E0012DCD2
:10DCB000F512DE9512437012DCE312DD02EE241839
:10DCC000F582E43F12DD158E828F83A3A3E50AF06F
:10DCD000A3E50B12DE88123D34E9F50CA90C7403A0
:10DCE00002D92912DCEBEAF0A3EB22EE241AF5822A
:10DCF000E43FF58322E08882898322F0A3A882A9E9
:10DD00008322F0EE241612DD0A22F582E43FF58329
:10DD10007401F02239F58312DE81F02274EF1225AE
:10DD200017EAFEEBFF751000EE12DB143F12DF68FE
:10DD3000F508A3E0F50912D72A12CC89123CBCEAF7
:10DD40004B700302DDF58A828B83A3A3A3A3E0704B
:10DD50000302DDF5C39403400302DDF5E508C39437
:10DD60000F5004E50960057510018079EA2412F569
:10DD700082E43BF583E4F0E5087022904F2B7808AD
:10DD8000122CE512DDFA7808122D9D904F2B7808A1
:10DD9000122CE512E7517808122D9D803975090083
:10DDA00074027808122CBF742B2508F582744F1268
:10DDB000CC78780C122CE590812B7808122D7F7886
:10DDC0000C790812242812DDFA780C122D9D12E726
:10DDD00051780C122D9DEA241BF582E43BF58374E7
:10DDE00001F01237529019D4E0FCA91012CC631242
:10DDF000CC891244847F09022843EA2417F582E47F
:10DE00003BF5832274F012251774F5122BB68A089D
:10DE10008B09890B8C0C750A017401122E00740396
:10DE200012CFBF1243F48A0E8B0FAE0EAF0FEE4F20
:10DE3000604812CD81740C12DA52A3E50C12DE9503
:10DE4000124370EE241AF582E43F12DA46122B9642
:10DE5000AA08AB09123C3EE9600E12CF6C740312A3
:10DE60002B8612CD5A12CC988E828F83A3A312DEFA
:10DE70008112DE88123D34E9F50AA90A740B02D931
:10DE800029E508F0A3E5092212CDA67401F0EEFA07
:10DE9000EFFB227401F0EE241712DD0A2274F01257
:10DEA000251712DB133B12DF68F8A3E0FEE86003DE
:10DEB00002DF6574016E600874026E600302DF6544
:10DEC000EE9019D4F07508D47509197808122B262C
:10DED0007508017509007808122B267C007D007AF0
:10DEE000517B001234047404122AE874026E7075B7
:10DEF000901CCAE0700A904F2B7808122CE58028FD
:10DF0000F50874027808122CBF742B2508F582746A
:10DF10004F12CC787808122CE590812B780C122DBA
:10DF20007F7808790C12242890810B780C122D7FB1
:10DF30007808790C1224A8908117780C122D7F781C
:10DF400008790C1224289019D67808122D9D901962
:10DF5000D612294B7A007B40901AC3E0F91234465E
:10DF60007404122AE802D92CF583E02401F8A3E016
:10DF70003400F988828983E02274F612251774DA56
:10DF8000122BB6EAFEEBFF12CF8360508E828F8396
:10DF900012CC89AC18AD1912D1A5124358740912CC
:10DFA0002E0012E21D7003A3E069603012E2EA1253
:10DFB00029537508FE7509FF7808122B26741C1268
:10DFC0002E00E0F9740D122E0012B9A4740F122E57
:10DFD0000012CC89123F4A7404122AE8742602C93E
:10DFE0000474F7122517E9FD7A007B009019E6E02A
:10DFF0006004640170407C00800B12E08DE02AFA1E
:10E00000A3E03BFB0C90506E12EED05029EC75F063
:10E010001CA4F8AEF0EEF912EEF2F460E7740128F9
:10E02000F58274063912CF8660DAED60CD12E08D8C
:10E03000E4F0A3F080CE7C00800B12E07AE02AFAB4
:10E04000A3E03BFB0C12EECD502DEC75F017A4F8BD
:10E05000AEF0EEF912F0717003A3E0F460E674C65E
:10E0600028F58274073912CF8660D9ED60CC12E0B2
:10E070007AE4F0A3F080CD02B3EDEC75F017A4F8CC
:10E08000EEF974C628F582740739F58322EC75F031
:10E090001CA4F8EEF9740128F582740639F5832280
:10E0A00074EC122517890CEAFEEBFF901AC2E0C34C
:10E0B000950C503B1243C4901AF412E0F6901A5C8F
:10E0C000E0F508E4F509F50AF50B90816B7810127C
:10E0D0002D7F780879101224287808122B1E7A00D8
:10E0E0007B02901AC3E0F91234407404122AE80249
:10E0F00087268A828B83EEF0A3EFF02274F6122536
:10E1000017EAFEEBFF901AE0801388828983E06EA5
:10E110007003A3E06F603A88828983A3A312CF883B
:10E1200070E87A047B001233808A088B09A808A95A
:10E1300009E849601C8882898312E0F6901AE0128F
:10E14000CC8988828983A3A312E15A901AE012CC69
:10E150009802C907F582E43FF583EAF0A3EBF022C9
:10E1600074F41225177E00901AE080070E8A828BC5
:10E1700083A3A312B2F870F4EE25E0FAE433FB12A5
:10E1800033808A088B09EA4509607F7C00901AE099
:10E1900080228A828B83E0F50AA3E0F50B12DA3144
:10E1A000E50828F582E50939F58312DA500C8A82F0
:10E1B0008B83A3A312B2F870D9901ABE12E21D701D
:10E1C00003A3E0697808701C122B26EEF50A780A82
:10E1D000122B2A7C8A7D1A7900901ABE12CC8912E1
:10E1E000446C801A122B26EEF50A780A122B2A7C30
:10E1F0008A7D1A7900901ABE12CC89124460740389
:10E20000122AE8AA08AB09123386123D4C028FBECF
:10E210008E828F83A3A3A3A3A3A3A3A3A312D53BFF
:10E22000901A69E06822C082C08380128A828B8340
:10E23000A3A312BAD2901AE012CC98123386901A85
:10E24000E012B2F870E602C57574F5122517901A3F
:10E250007612BC60901AF412A02812CC987AF47B43
:10E260001A7950123B60901AF412E2E3801312EB19
:10E270009A7004A3E06509600612EBA71245080531
:10E280000A905061E493F8E50AC3985020E50A75B6
:10E29000F017A4F8A9F012EA486E7003A3E06F70BB
:10E2A000CD74BB28F582740712DD1480D2901AF465
:10E2B00012BC6090190812CF8860257A067B001284
:10E2C00032DEEA4B601A8A828B8374D5F0A3A3E412
:10E2D00012E6950412E2FA90190812E2EE124A8947
:10E2E00002B65D128735750A00228E828F8312E294
:10E2F000F22212D598F58388822212B198EEF0A30B
:10E30000EFF022C082C083901A69E064FE7003A31C
:10E31000E0F4600E901A63E0A2E15006124520126C
:10E3200044C602C57574F0122517901AB7E0605301
:10E33000F50CE4F50DF50EF50F9081177808122D08
:10E340007F780C79081224281232D88A088B09A801
:10E3500008A909905054E49358F508A3E49359F59B
:10E3600009E4F50AF50B780C7908122C99780C124F
:10E370002B1E7A007B01901AC3E0F9123446740414
:10E38000122AE802D92C74EE1225177E007F008E27
:10E390000A8E0B123CE6750D00803BAA0D7B001225
:10E3A0003CE08A088B09A808A909E8496026888208
:10E3B0008983A3A3A3A3E0600464047017888289FF
:10E3C00083A3A3A3A3A3A3A3A3A3A3E0F91245320A
:10E3D000E960010F050D90506EE493F8E50DC398C8
:10E3E00040B91244F68A0E8B0F750C008023AA0CDC
:10E3F0007B001245028A088B09A808A909E8496030
:10E400000EE8240F129AD3F9124532E960010E0585
:10E410000CC3E50C950EE4950F40D3EF2EFE700370
:10E4200002E51C8E0875090074027808122CBFAA38
:10E4300008AB091233808A0A8B0BEA450B70030282
:10E44000E51A750C008E0875090074027808122C04
:10E45000BFAC08AD0979FF1232C6750D00805EAA07
:10E460000D7B00123CE08A088B09EA4509604C8A62
:10E47000828B83A3A3A3A3E060046404703D8A821B
:10E480008B83A3A3A3A3A3A3A3A3A3A3E0F91245F0
:10E4900032E9F96026050C780A122B26EEFD850874
:10E4A00082850983A3A3A3A3A3A3A3A3A312E5AD7A
:10E4B00012CC891244CC7402122AE8050D90506ED9
:10E4C000E493F8E50DC3985006E50CC39F409075A2
:10E4D0000C00C3E50C950EE4950F5040AA0C7B0090
:10E4E0001245028A088B09EA4509602AEA240F12BC
:10E4F000AFF0F9124532E9F9601C780A122B26EECA
:10E50000FDE508240E12CC7512E5AD12CC8912443B
:10E51000CC7402122AE8050C80B87E007F62901A43
:10E5200061E0600BF91241F6E9F87454C398FF7585
:10E53000F003EF84F50D94204003750D1F850A0844
:10E54000850B09750C00EF6005750C207F00E50D4B
:10E55000C39E5005850D0F80088E0FE50CD2E6F5A1
:10E560000CAC08AD09AA0CA90F1244D2E9F50EE5CE
:10E570000CA2E6401D150F7800800BE5082404F579
:10E58000085002050908E8C3950F40EFE50FCEC318
:10E590009EFEE97006E50CA2E650A8E50A450B6070
:10E5A00007AA0AAB0B123386A90E02C29CE0FC85B7
:10E5B00008828509832274F2122517EAFEEBFF898F
:10E5C000088C098D0A7C007D00740E122E0012CC7E
:10E5D00089750B00800DEAFCEBFDEA2404FA50017A
:10E5E0000B050BE50BC3950A400302E6858A828B77
:10E5F00083E0F47003A3E0F4607AEC4D600C8C824D
:10E600008D83C3E09EA3E09F50CC8A828B8312E669
:10E6100088EE98EF9950BFEAF8EBF988828983E099
:10E62000F47003A3E0F46010E82404F85001090535
:10E630000BE50BC3950A40E3E8FCE9FDE824FCF890
:10E64000E934FFF98882898312E68D8C828D83E517
:10E650000CF0A3E50D12E6A48C828D83A3A312E631
:10E660009AA3A3A3E08C828D83A3A3A3F0C3EA980B
:10E67000EB9940C412E0F28A828B83A3A3E50912CE
:10E68000E695E508F0028B3012D53BC322E0F50C8D
:10E69000A3E0F50D2212B18CA32212E69E22F0888F
:10E6A0008289832212E6AAA3E02212E69EA32274A4
:10E6B000F212251774FD122BB689088A09ECFEEDBB
:10E6C000FF750A0175F003E9A42402C0E074011289
:10E6D0002E00D0E012CFBF1243F4EA4B607012D785
:10E6E000AB12CD867408F0741F55084509A3F0E8F5
:10E6F0002402F8500109750A0080338E828F83123C
:10E70000DCF512DCFB8E828F8312CD968E828F8396
:10E71000A3A3E05407C4FC8E828F83A3A3A3E05479
:10E72000074C12CD98EE2404FE50010F050AE50AAD
:10E73000C3950840C68A828B83A3A374FCF0A3749C
:10E74000FFF012E7517401F0123D34E9F50A028B33
:10E7500029EA2413F582E43BF5832274F11225178C
:10E760008A0A8B0B7508007AFE7BFF7CFE7DFFE535
:10E770000A12DB14350B12D918F509741F5509F567
:10E780000CE82402F8500109E509A2E74065E50A12
:10E790002417F582E412F594FE75F003E50CA42429
:10E7A000026E704FE50C600612DBD3FBEEFA750DBE
:10E7B00000801DE05407F50EA3A882A983EEFC900B
:10E7C0001A69E06E7003A3E06F7003850E08050DF3
:10E7D000E50DC3950C502612DBD3FCE4CCFDEE2CEA
:10E7E000E43DFFE82402F850010988828983E0545F
:10E7F0008860C07AD37B001237BE02E93EE508701C
:10E800000BA9091244DEE9700302E93E12E9431242
:10E81000CC89123CB68A0C8B0DAE0CAF0DEE4F605E
:10E820005A8E828F83A3A3A3A3A3A3A3E4F0905043
:10E830005993F88E828F83A3A3A3A3A3A3A3A3E0DA
:10E84000C398402412E94D5001097A027B0012233B
:10E8500031E88E828F83A3A3A3A3A3A3A3A3F0E590
:10E8600008C39407500205088E828F83A3A3A3A335
:10E87000A3A3A3A3A3E508F002E93E7CFF7DFF125A
:10E88000E94312CC891244EA8A0C8B0DAE0CAF0D11
:10E89000EE4F704F1244F08A0C8B0DAE0CAF0DEEA4
:10E8A0004F700302E93E7C177D0079001232C612D8
:10E8B000E94312CF791287838E828F83A3A3A3A308
:10E8C000A3A3A3A312B9D112B51C74AA12E96C5068
:10E8D00001097A027B0012233112DBA9E812E95800
:10E8E0007401F0905059E49312BF56C39840191226
:10E8F000E94D5001097A027B0012233112EFF8E54D
:10E9000008C394075002050812EFE4E50812E95D18
:10E91000E4F012A020123C32E97023850A82850BB4
:10E9200083A3A3A3A3A3A3A3A3E06012E50A2415D2
:10E93000F582E4350B12B9B212A0211234887F0798
:10E94000022843E50A12F462350BF58322905059F0
:10E95000E49379002401F822F012EFE822F012E9A2
:10E960006222EE240CF582E43FF58322F0905059A8
:10E97000E49379002401F82274F7122517E9FE7454
:10E98000FE6A700374FF6B603474605E6460602DB7
:10E99000EEA2E5401CA2E6901A69500DC3E09AA3CE
:10E9A000E09B5019790002B3EDC3E09AA3E09B40CD
:10E9B000F3901A6912E688EC98ED9940E7790180A6
:10E9C000E574F71225177E008008EE12EBA01245C1
:10E9D000080E12EA0240F37E00EE75F003A4F8A9D7
:10E9E000F074E228F8741A39F988828983A374FED6
:10E9F000F0A30412E69AE4F00EEEC3940340DA02A8
:10EA0000B3ED905061E493F8EEC3982274F71225A9
:10EA1000177E0080010E12EA025026EE12EA586AB2
:10EA20007003A3E06B70EE12EA486C7003A3E06D14
:10EA3000600A74FF6C700374FF6D70D912EBA780CD
:10EA4000047A007B0002B3ED12EA4C2274BB28F575
:10EA500082740739F583E02275F017A4F8A9F01243
:10EA6000EA632212EEC2E02274F61225177CFF7DC3
:10EA7000FF7AFE7BFF1244EAEA4B703C7508008087
:10EA800032E50875F017A4F8A9F074C028F582746F
:10EA900007129AD6600512EEE7701674B128FE745C
:10EAA0000739FF8E828F8312CC89123F50EEFAEF26
:10EAB000FB050812EABB40C902C907905061E49304
:10EAC000F8E508C39822C082C0837A007B007C00EE
:10EAD000801012F0697003A3E0F460050AEA700187
:10EAE0000B0C12EECD40EB02C57574F41225178A9B
:10EAF000088B09ECFEEDFF800B124508EEFCEFFDE4
:10EB0000AA08AB091244EAEA4B70EE028FBE74F712
:10EB10001225177D007C0080020D0C12EECD501CDA
:10EB200012F0697003A3E0F460F0EDF8EA684B704E
:10EB3000E8EC75F017A4F812EBA780047A007B00CC
:10EB400002B3ED74F7122517EAFEEBFFEE4F6018E3
:10EB50007C177D0079001232C68E828F8374FEF09E
:10EB6000A30412EFFFF0A3F002B3ED74F612251721
:10EB70008A088B097E00801AEE75F017A4F8A9F0B8
:10EB800012EB9A7004A3E06509600612EBA7124528
:10EB9000080E12EA0240E102C90712EA4C65082297
:10EBA00075F017A4F8A9F074B128FA740739FB229C
:10EBB00074F41225178A088B09ECFEEDFF9019E614
:10EBC000E0600464017020901A76E06E7003A3E0A8
:10EBD0006F7014123CB68A0A8B0BA80AA90BE8497D
:10EBE0006005E82408801AEEFCEFFDAA08AB0912C4
:10EBF00044EA8A088B09A808A909E8496009E824B9
:10EC00000DFAE439FB80047A007B00028FBE74F4B5
:10EC10001225178A088B09ECFEEDFF750A00750BAB
:10EC200000802FE50B12F059123C32E96022E50B0F
:10EC300012EA5865087004A3E065097003750A0AB2
:10EC4000EEFCEFFD12F060123482E96003430AA08B
:10EC5000050B905061E493F8E50BC3985004E50A66
:10EC600060C1A90A028FBE74F61225177E00805A71
:10EC7000EEFA7B00123CE08A088B09A808A909E893
:10EC800049604688828983A3A3A3A3E06401603915
:10EC900088828983A3A3A3A3E06402602CE82407ED
:10ECA000129AD3FA74012AF0901AB8E0C39A501954
:10ECB00088828983A3A3A3A3A3A3A3A3A3A3E412EA
:10ECC000ED4FA312ED5A123F500E90506E12EA050E
:10ECD000409E7E008059EE75F017A4F8AAF0EAF97C
:10ECE00012F0717003A3E0F4604474B128F8740763
:10ECF00039F9E8240C129AD3F8740128F0901AB864
:10ED0000E0C3985029EE75F017A4F8EAF974B12819
:10ED1000F8740739F9E812ED4939F583E4F0E8248D
:10ED20000EF582E439F583E412ED5A123F500E12CB
:10ED3000EA0240A27A00EA12D3C4600214F00AEA9E
:10ED4000C3940340F102C907EE240FF582E42212B6
:10ED5000E6AAA3A3A3A3A3A3A32212E69E12D1BD56
:10ED60002274F11225178A0A8B0BECFEEDFF750E4B
:10ED7000007A007B017508FE7509FF740F122E00E2
:10ED800012E68D80111232D8E50EF5F0EA84E5F036
:10ED9000FA750E007B007C00800712EEC2128731EC
:10EDA0000C12EECD505CEC75F017A4F8ADF0EDF957
:10EDB00012F0717003A3E0F460E612EA5F650A7076
:10EDC00004A3E0650B60D912F0547003A3E06F60F8
:10EDD000CF12EA5F650C7004A3E0650D60C212EE0D
:10EDE000E760BDC3940850B8E0640760ADEB050E62
:10EDF00070AEE50EC39A40A874B128F5827407027C
:10EE0000EE8C9019E6E060076401600302EE947CEA
:10EE100000800712EF021287310C90506E12EED074
:10EE20005072EC75F01CA4F8ADF0EDF912EEFD6433
:10EE3000FE7003A3E0F460E112EEFD650A7004A326
:10EE4000E0650B60D412EEFD6E7003A3E06F60C945
:10EE500012EEFD650C7004A3E0650D60BC12EED7E8
:10EE600060B7C3940850B212EEF2640160ABE06484
:10EE70000260A612EED764076099EB050E709AE562
:10EE80000EC39A409474F128F58274053DF58312FF
:10EE9000CC89802BE50E6011EA700E7401650E605E
:10EEA0000302ED857A0102ED9174FE650870047429
:10EEB000FF65096006AA08AB0980047AFE7BFF02A1
:10EEC000E93E74B128F582740739F58322905061C8
:10EED000E493F8ECC3982274FA28F582740512EED4
:10EEE000E22239F583E02274BF28F582740712EE1E
:10EEF000E22274F528F582740512EEE22212EF0286
:10EF0000E02274F128F582740539F5832274F51234
:10EF100025178A088B09ECFEEDFF750A00800205B3
:10EF20000A905061E493F8E50AC3985022EEFCEF92
:10EF3000FDE50A12F059123482E960E3E50A75F042
:10EF400017A4F8A9F074B128F582740712DD140231
:10EF5000B65DE9F87907C3940D400479018019E89A
:10EF6000C3940740047903800FE8C39403400479F5
:10EF7000058005E870027900022AD074F012251786
:10EF80008A088B098C0A8D0B890C1244F08A0E8B2F
:10EF90000FAE0EAF0FEE4F60487C177D0079001268
:10EFA00032C68E828F8312DE8112EFFF12DA50E5B5
:10EFB0000C600712B51BE50C800312EFF2F0901AFB
:10EFC000BDE06401700612EFE4E4800512EFE47422
:10EFD0000712E96C5001097A027B0012233112EF0B
:10EFE000F802D92C12EFE822EE240EF582E43FF568
:10EFF000832212CD73740122EE12DBAEE8F02212EE
:10F00000A9A1A32274F7122517EAFEEBFF750800E9
:10F01000803AE50875F017A4F8A9F012F0547003CF
:10F02000A3E06F601474FF6E700374FF6F701B12A7
:10F03000F0717003A3E0F4601112F060123C32E949
:10F040007008E50812EBA0124508050812EABB405B
:10F05000C102B3ED12EA636E2275F017A4F8A9F0AD
:10F0600074B328FA740739FB22EC75F017A4F8A9D9
:10F07000F012EA6364FE22C082C0837AFF7BFF1233
:10F08000453E02C575C082C083901AF67450F0A345
:10F090007445F0901AF87456F0A37445F0901AFA7B
:10F0A000745CF0A3744502AD7A74F7122517EAF880
:10F0B000EBF99019FF12F0F2CA2406F582E43AF552
:10F0C00083E0702B88828983A3A3A3A3A3A3A3A314
:10F0D000A31229539019FF12F0F7122DD1888289BB
:10F0E00083A3E0F9123E067402122AE8123D4C0294
:10F0F000B3EDE0FAA3E02212F0F2F5838A8222C097
:10F1000082C083901AC012F1C3F0901AC012CF8847
:10F110007005790112449602C57574F612251774AC
:10F12000FC122BB6E9FE90505BE493700874E16E1C
:10F13000600302F1BEEA2408F8E43BF9888289837F
:10F1400012F1C312F1CC700E901AC0E4F0A3F07962
:10F15000011244968068901CDEE06062F8901AC04C
:10F1600012CC89C3E89AE49B505479001244968AE1
:10F17000088B09AC08AD09ECF8EDF9E875F064A46A
:10F18000F8AAF075F064E9A42AF9901AC012CC89A3
:10F19000122339E8941AE99400402390190012CF01
:10F1A00088601B901AC012CC8D7402122E00ECF0F5
:10F1B000A3ED12CFBF90190012E2EE124A89740437
:10F1C00002C904E02401F0A3E034002212E69E12FA
:10F1D000D53BE84922C082C08374F8122BB69080D8
:10F1E000E2AC18AD197408122A4CAC18AD191234DF
:10F1F00082E964017004790080027901740802D503
:10F200007874F6122517740C122E0012BC60743A32
:10F210006E7001EF6006743B6E4F7023740A122EFD
:10F22000001229538C088D097808122B26EAFCEB72
:10F23000FDEEFAEFFB12340A7404122AE880027918
:10F240000A02C907C082C083901AFC74ECF0A37450
:10F250003CF0901AFE74F2F0A3743CF09019D4E0E4
:10F2600064017032901B00747AF0A37445F0901B17
:10F27000027480F0A37445F0901B047486F0A374AC
:10F2800045F0901B06748CF0A37445F0901B087435
:10F2900074F0A37445F0901B0012CF88600612C86A
:10F2A000AA124A8902C57574F412251774E6122B46
:10F2B000B68A088B097404122E007402F004122B13
:10F2C0008E1243F48A0A8B0BAE0AAF0BEE4F70031B
:10F2D00002F43112F481746012CDA212DE93124353
:10F2E0007012DCE312B9CD12DE8112BFAE70129043
:10F2F0001A55E0C0E012F436D0E0F0901A55E00460
:10F30000F012F4527016901CBEE0600D901A60E08E
:10F31000700A8E828F83E0700312CD64AC18AD1931
:10F32000EEFAEFFB12434C8A088B09EA4509700399
:10F3300002F42A7A217B001233807406122E001206
:10F34000E15A7406122E0012CF88700302F4237C57
:10F35000217D0079007406122E00E0FA1232C67484
:10F3600001122B8E7950123B5A7401122E0012BAE0
:10F37000D27406122E0012F0F2CA2409F582E43A81
:10F38000F58312CC98901A6912BAD27417122E0013
:10F3900012CC987406122E0012BC6512F458F07448
:10F3A00006122E0012B0DB740212F4A77406122E9D
:10F3B0000012F0F712CC987406122E0012F48C1280
:10F3C000F4B2C0E07406122E0012BC6512F468D0CC
:10F3D000E0F0EE240E12F440C0E07406122E00128B
:10F3E000F471D0E0F07406122E0012BC6512BC5607
:10F3F00012DD15EE240F12BACC740C122E0012CCB2
:10F40000988A828B83E0C0E0740E122E00D0E0F068
:10F410007406122B8E1242C27406122E0012CC8970
:10F42000123386AA08AB09123386EEFAEFFB1233C9
:10F4300086741A028FBBEE2414F582E43FF5832212
:10F4400012F445E022F8E43FF9E8FAE9FB8A828BFE
:10F45000832212BF4B64012212F46238F5837402D6
:10F4600022EA240BF582E422241EF582E438F58397
:10F470002212F4752212BC69240CF582E438F5835B
:10F480002212CC6712CD8C7404F0A322E012F49601
:10F490007401F0A3E422F8A3E0C812F49E22240D24
:10F4A000F582E438F5832212DBC312D53B22E8F063
:10F4B000A3E912A7F1E02274F61225177E00801846
:10F4C0007C047D0079FF8E088D0974027808122C67
:10F4D000BF12F6F21232C60E90505812EA0540E002
:10F4E00002C90774F412251774F7122BB6750800B9
:10F4F000802285080A750B007402780A122CBF74EA
:10F5000050250AF582740B12F59424FFF0A3E03421
:10F51000FFF0050890505812EABE506D85080A7534
:10F520000B007402780A122CBF12F58CF47003A33E
:10F53000E0F460DE85080A750B007402780A122C6C
:10F54000BF7450250AF582740B350B12CF8670A25A
:10F550007408122E007402F085080A750B00780AF0
:10F56000122CBF744E250AFE740B350BFF8E828F52
:10F570008312CC8D12F59A123BA27C047D0079FF98
:10F58000EEFAEFFB1232C6808902B0D6744E250A1D
:10F59000F582740B350BF583E02212F70B2274EE23
:10F5A00012251774F7122BB6EAFEEBFF750CFF74E9
:10F5B00008122E0012F6FD123B9CE9641A70030239
:10F5C000F670750E00741B122E007808122D7F80C5
:10F5D0000B74FF650C7003850E0C050E905058E4FB
:10F5E00093F8E50EC3985048850E1075110074020B
:10F5F0007810122CBF12F674F47003A3E0F460D1FB
:10F60000850E1075110074027810122CBF12F6745A
:10F610006E7003A3E06F70C2750F007402780E1253
:10F620002CBF7450250EF582740B350FF583803096
:10F63000E493650E702D74FF650C602E850C0E75BD
:10F640000F007402780E122CBF744E250EF8740B46
:10F65000350FF98882898312E0F688828983A3A313
:10F6600012DD177901740902C29912F59A123BA2B0
:10F67000790080F1744E2510F582740B3511F583F5
:10F68000E02274F412251774F7122BB6EAFEEBFF92
:10F690007408122E0012F6FD123BA27508008002BB
:10F6A000050890505812EABE504585080A750B00AF
:10F6B0007402780A122CBF12F58CF47003A3E0F4E4
:10F6C00060DE85080A750B007402780A122CBF12DE
:10F6D000F58C6E7003A3E06F70C67C047D0079FF2B
:10F6E0008D0974027808122CBF12F6F21232C6028B
:10F6F000B0D6744E2508FA740B3509FB2274021239
:10F70000A7F1EEF0A3EFF012F70B22901A7612B9E0
:10F71000ACAA18AB192274EE1225178A088B09ECD3
:10F72000FEEDFF750A00EE65087003EF6509600CD9
:10F730001233FE8A0C8B0DEA450D7006750A010224
:10F74000F7D2EEFAEFFB1233FE8A0E8B0FAC0EAD42
:10F750000FEC4D6007EEFAEFFB123410E4F50EF5F6
:10F760000F780E122B26AC0CAD0DEEFAEFFB123318
:10F77000F87402122AE8E96059AA0CAB0D12338022
:10F780008A0E8B0FEA450F6046780E122B26780CF6
:10F79000122B267C007D00AA08AB0912340A7404DF
:10F7A000122AE8E9701D780E122B26780C122B26EF
:10F7B0007C007D00EEFAEFFB1234047404122AE898
:10F7C000E96003750A01AA0EAB0F12338680037538
:10F7D0000A10A90A02C29C122392022AD0C082C037
:10F7E0008374FF122BB6AC18AD197A01798712FE1B
:10F7F00034C39403400F7402F07C007D00FA79E278
:10F800001234E8800CE4F0901CDDE0FA7B00123644
:10F810001A7401122AE8D083D082022AD074F0121E
:10F82000251774F5122BB6851882851983EAF0A383
:10F83000EBF0ECFEEDFF750820E9700302F9CE90C5
:10F840001864E0F47003A3E0F47057EC4F60687440
:10F850000A122E007403F07402122B8E1234889058
:10F86000185DE0F5087808122B2A7403122B9674A1
:10F8700001122E0012FF1F90185DE0F912407C74F7
:10F8800001122AE8E9F50870197D007C007900EE84
:10F89000FAEFFB12390E90813F12294B12FA9F1298
:10F8A0002AE8851882851983E0FCA3E0FDAA08797F
:10F8B000E11234E802F9EC750802740A122E0074A1
:10F8C00002F0122E0074FFF0A3F012F9FBA3A3A321
:10F8D00012295388828983A3A3A3A3A3A3A3A3A3C9
:10F8E000E0FC7402122B8E790112381E7402122A67
:10F8F000E8E9602F7508007808122B2AE4F50AF56C
:10F900000B780A122B267808122B2A7404122B86E5
:10F91000880A890B780A122B2612F9F612295379D4
:10F9200001805712F9FB12295388828983A3A3A36C
:10F93000A3A3A3E0FC7402122B8E790112381E746B
:10F9400002122AE8E9700302F8A27508007808128A
:10F950002B2A7401122B86880A890B780A122B260F
:10F960007508017808122B2AE4F50AF50B780A12BB
:10F970002B2612F9F612295379007CFF7DFF740AB9
:10F98000122B8E12391A7408122AE8E9F508E508D4
:10F99000600302F8A2901A15E0F50CA3E0F50DE45F
:10F9A000F50EF50F780C122B1E7A007B2090186351
:10F9B00012FAA6122AE8851882851983E0F8A3E0D6
:10F9C000F9901864E8F0A3E9F080211249E27C0084
:10F9D00085188285198312FF25124982EA4B70EB44
:10F9E00090813F12294B12FA9F122AE8740B122AB7
:10F9F000E87F0802284312FB6CA322901860E0F80D
:10FA0000A3E0F98882F583A3A3A3A3A3A3A32274ED
:10FA1000F712251774F7122BB67408122E00740211
:10FA2000F0851882851983EAF0A3EBF07D007C0055
:10FA3000AA18AB191239867409122AE802FC9474C8
:10FA4000F4122517E9FE7A007B40901863E0F91262
:10FA5000344CEE700512FF7480407A0112FF767408
:10FA6000FF6E6036EEC3944140027E40EEF50875AD
:10FA7000F0E8A4C508A8F075F003A428F8E428F578
:10FA8000093395E0F50AF50B7808122B1E7A007BF6
:10FA90004090186312FAA6122AE87F040228437ADB
:10FAA000007B019018CBE0F912344074042274F406
:10FAB00012251774F4122BB68C088D09E9FF741BFC
:10FAC000122E00E0FE74FE6A700374FF6B700974FE
:10FAD00008122E00E4F0801D851882851983EAF053
:10FAE000A3EBF07408122E007402F0124412E960C5
:10FAF00004EEC2E4FE740A122E00E4F0A3F012FB3E
:10FB00006CE0C0E07409122E00D0E0F0741C122EDC
:10FB100000E0F50A780A122B2A741B122B86880A39
:10FB2000890B780A122B26741B122E00122953EF10
:10FB3000F50A750B00780A122B267808122B26EE90
:10FB4000F97C5D7D187409122B8E124A4E740912CD
:10FB50002AE8E9FA600E741A122E00E0FC7D0079A2
:10FB6000E01234E8740C122AE802FA9A12FB7022AE
:10FB7000901860E0F8A3E0F58388822274F61225DD
:10FB800017E9FEEAFF8C088D09E9FA7B001233FEC3
:10FB9000EAF9EFC3995004790180207808122B26E6
:10FBA000EAF5087509007808122B267C007D00EE26
:10FBB000FA7B0012340A7404122AE8802974F612BF
:10FBC00025178C088D097808122B26EAF508750987
:10FBD000007808122B267C007D00E9FA7B001234A5
:10FBE000047404122AE87F0202284374F5122517D0
:10FBF000E9601714601C14602114602614602B1433
:10FC0000603014603F14604E80667508CE75091828
:10FC1000802675089A75090B804275086975091A5E
:10FC2000802875086C75091A802075086E75091A88
:10FC3000802A75086B75091A750A007808122B223C
:10FC40007C01802275087675091A750A00780812F9
:10FC50002B227C02801075088A75091A750A0078B3
:10FC600008122B227C087D001232BA7403122AE893
:10FC70007F0302284374F7122517E9FE74016E70A2
:10FC8000097D007C00790012390E800874F7122576
:10FC9000171231527F0102284374F71225171231CF
:10FCA0005880F174F212251774FF122BB6890A8A54
:10FCB000088B09EB5480700302FDBC800FA3E0F9B0
:10FCC00012314CEEFAEFFB1232E4A90A1232F68A34
:10FCD0000C8B0DAE0CAF0DEE4F700302FDB48E8297
:10FCE0008F83E024E6603D2449607414700302FDB4
:10FCF0009214601624F3700302FD9B14700302FD3E
:10FD0000A51460B924E5600B80B9EEFAEFFB12345C
:10FD1000DC80B0A3E0FA8E828F83A3A3A3E0F91264
:10FD200034CA809FEE2422F582E43FF583122953E2
:10FD3000EE2420F582E43FF5831229538E828F83CF
:10FD4000A3A3A3A3E0FCA3E0FD8E828F83A3A3A3C0
:10FD5000A312FF1D12316A7404122AE802FCC3A325
:10FD6000E0640660148E828F83A3E06407600A8ECD
:10FD7000828F83A3E064097005790002FCC08E8243
:10FD80008F83A3E060076401600302FCC379220251
:10FD9000FCC012FF1D12315E02FCC3A3E0FA8E828A
:10FDA0008F8302FD1BA3E0F98E828F83A3A312FE33
:10FDB0002B02FCC3AA08E50964808060EB54406014
:10FDC0000B12FF74AA08E50964408050EB542060D0
:10FDD00018792190186412FE2B90186474FFF0A318
:10FDE000F0AA08E50964208033EB54107A00602FF4
:10FDF00079081249ACAC18AD197A01790312FE34B6
:10FE0000A2E25005123494800D7CF47D017B327A9D
:10FE10000079021249A6AA08E5096410FB80027B5A
:10FE2000007401122AE87F06022843E0FAA3E0FBEF
:10FE30001234D0221234B2851882851983E02274DC
:10FE4000F612251774F7122BB6EA240CF582E43B60
:10FE5000F583E0F508A3E0F50978081227B1000062
:10FE6000020000806CFE068089FE18FF1238D88AD6
:10FE7000828B83E5822403FCE43583FDA3AA82AB55
:10FE800083790112316402FF181238DE8A088B0967
:10FE9000AE08AF09901864E0F47003A3E0F4607852
:10FEA0007408122E00740212FFB3E0F8A3E0F98583
:10FEB0001882851983E8F0A3E912FFB3A3A3A3E096
:10FEC000F5087808122B2A7401122B9690186412E8
:10FED000FF2512407C7401122AE8E9703B7A007B0E
:10FEE00020901863E0F912344C90813F12294B1294
:10FEF000FA9F122AE87D007C0079008E828F83129F
:10FF0000FF1E123914790090186412FF1F12315825
:10FF100090186474FFF0A3F0740902FBE3A3A3E05C
:10FF2000FAA3E0FB22E0FAA3E0FB12FF2E2212FB71
:10FF300070E0F92274F7122517E9901863F0901811
:10FF40006474FFF0A3F090185E7463F0A37418F06B
:10FF500090185DE4F0FA12FF767A007B80901863C7
:10FF6000E0F91239B67A067B80901863E0F912390D
:10FF7000B602FC947A0012FF2E124A2A2274F4125E
:10FF8000251789088A09ECFEEDFF7A047B001232FE
:10FF9000DEEA4B601B8A828B83E508F0A3E5091239
:10FFA000FFB3A3EEF0A3EFF0901863E0F91232EA8A
:10FFB00002FA9AF08A828B83A322C082C083901CAB
:10FFC0002AE060357480659E70FA439403E594A23C
:10FFD000E250FAE064027008122FF0122FFC801138
:10FFE000E06401600312491CE59DA2E6400312494A
:10FFF0001C901C2AE4F0123080D083D082022AD0D8
:020000040001F9
:10000000C082C083790012CFA2C082C0839019FB46
:1000100012C856D083D082C3E09CA3E09D500DEA65
:10002000240B12804F12802F60027901029E4BEA4E
:1000300075F00BA4FAA8F075F00BEBA428FB90194F
:10004000FDE02AF8A3E03B8882F583E0540F22F517
:1000500082E43B12B98B2274F7122517890812B07B
:10006000A41283B7ACF075F00BE9A42CF99019FD3C
:10007000E028F8A3E039F9E8FEE9FF7401650860BB
:10008000067402650870228A828B8312856D740261
:1000900065087021EA2403FA50010B123C32E97022
:1000A000148E828F83E4F0800CEA2403FCE43B127C
:1000B0008564123C2C8E828F83E0D2E7F012371CCD
:1000C00002AC5A74F412251712863E79008E828F84
:1000D00083E06078890A890B8063E50A75F00BA4D8
:1000E000FAA8F075F00BE50B12803B7048E50A7535
:1000F000F00BA4F8AAF075F00BE50B1285818E8247
:100100008F83E085088285098312A5321284E2EE8E
:100110002403FCE43F1281FA123C2C12AEA8E50A3B
:10012000F0A3E50B129B68D2E7F012371C7901901F
:1001300019FB12943B050AE50A7002050B9019FBA6
:1001400012C08EC3E50A9AE50B9B408E029B727427
:10015000F5122517EAFEEBFF750A01740B122E004B
:1001600012CCB3EC4D6015EC12BD583D12864C79A3
:1001700001123C14E508450960758023E50845092E
:10018000604412BD56350912864C1281FB123C3276
:10019000E96401701BEEFAEFFB123C1AE9F50A85DF
:1001A00008828509831284DA7902AA08AB098011D2
:1001B000128565123C32E9640170347903EEFAEF7E
:1001C000FB123C1480298E828F83A3E064FE7003AF
:1001D000A3E0F4700B128565123C32E96401700CE7
:1001E000EEFAEFFB123C1AE9F50A8003750A0002E9
:1001F0008CCBE50A2403FCE4350BFDE5082403FA67
:10020000E43509FB2274F71225179019FB12AFD8B9
:10021000EA4B602FEA75F00BA4FAA8F075F00BEB2F
:10022000A428FBEAFEEBFF1233809019FD12AFD831
:100230009019FD12ADED6012EEFCEFFD7900123267
:10024000C680079019FDE4F0A3F002AC5AC082C04A
:1002500083EC4D600512348880097C087D007900AC
:100260001232C6029E4BC082C0837900EA4B6016F0
:100270007800E8FCEA2C12B0B06004790178080834
:10028000E8C3940840EC029E4BC082C0837901EC25
:100290006A7002ED6B6011EA4B600BEC4D60071267
:1002A0003482E9F980027900029E4B74F712251717
:1002B00074F3122BB6ECFEEDFF851882851983E4EA
:1002C000F004122E00EAF0A3EB12C14E123C567459
:1002D00003122E00AC82AD83EEFAEFFB123C2CEE43
:1002E000FAEFFB123C3202AC5574F712251774F387
:1002F000122BB6ECFEEDFF851882851983E4F0EA37
:10030000FCEBFD7403122E00AA82AB83123C2CAAD4
:1003100018AB19123C5C7401122E0012A5438E8298
:100320008F8312AF9474FE68700374FF6960047960
:10033000018002790002AC5574F7122517EAFEEB32
:10034000FF123C0EE9F5087401650870111283A2D2
:10035000F4FA88828983E05A4480F012371CA90895
:1003600002AC5A74F7122517EAFEEBFF7508008EEF
:10037000828F83E0602A123C0EE9F508740165085B
:10038000701E1283A2FA88828983E05A70128E82CC
:100390008F83E04480FA88828983E04AF012371C18
:1003A00080BC12AD1CF81283B7128759F8A3E0394C
:1003B000F98E828F83E022A3E0F9E875F00BA4F8B0
:1003C0002274F41225178A088B097C007D00EA123A
:1003D00081FD123C2CE5081284FC79008508828599
:1003E0000983A3E064FE7003A3E0F460787E007FDD
:1003F000008065EEFAEFFB12802F6057EEFAEFFBFC
:10040000EA75F00BA4FAA8F075F00BEBA428FB90AA
:1004100019FDE02AF50AA3E03BF50B850882850962
:100420008312C08D850A82850B83A3E06A7003A3C3
:10043000E06B701FE50A2403FAE4350BFB123C3233
:10044000E9640170061281F2123C2C1284F17901E8
:1004500012C9BD0EEE70010F9019FB12C08EC3EED3
:100460009AEF9B408E029B7274F31225178A088BB9
:10047000098A828B831284DAEA1284FC750C00EA02
:100480001281FD123C32E9640170477E007F0080DA
:100490003C12874BFAA3E0398A82F583E0540F605F
:1004A0002712874BF50AA3E039F50B1281F21234BB
:1004B00082E964017012850A82850B831284E2123C
:1004C00084F1750C0112C9BD0EEE70010F12876820
:1004D00040BFA90C7F05022843A3A374FEF0A30428
:1004E000F022A312AC46850882850983A312A24B91
:1004F00022E508128506EEF0A3EFF02212850674BD
:10050000FEF0A304F022240BF582E43509F58322E2
:1005100074F5122517EAFEEBFF8E828F831284DAC0
:100520007C007D00128565123C2CEEFAEFFB123C3C
:100530000EE9F50A7401650A702712AC3F12857541
:10054000850882F58312856D1281FB123C32E964C5
:1005500001700EE5082403FCE43509128564123CA1
:100560002C028CCBFDEE2403FAE43FFB22A312C045
:100570009C12A24B22E875F00BA4F8AAF075F00BC0
:10058000E912875FF508A3E039F5092274F2122514
:100590001774E6122BB612863E750A0175080075AF
:1005A0000900750C00750D00851882851983E4F02B
:1005B000EE2403FCE43FFD7403122E00AA82AB83F9
:1005C000123C2CAA18AB19123C5CE96401701F7430
:1005D0000B122E0012864E7401122E0012C096705D
:1005E00003A3E069604AA818A91988088909740D4D
:1005F000122E0012A531A312A543740E122E001262
:10060000AF94740D122B8E123C56E964017009747C
:100610000D122B86880C890D780C122B26AC08AD98
:1006200009EEFAEFFB123C207402122AE8E9F50AFF
:10063000EEFAEFFB123C50A90A741A02AEBAEAFEB7
:10064000EBFF12AEAC74FEF0A304F022F58312C0EF
:100650007CF912AEAC12A24B22C082C08378007922
:1006600000800508E87001099019FB129850E99B79
:100670005029E8FAE9FBEA75F00BA4FAACF075F042
:100680000BEBA42CFB9019FDE02AFCA3E03B8C8231
:10069000F583E0540F70CC790080027901029E4B03
:1006A00074F61225177E007F008039EEF8EFF912FC
:1006B00085757808122B2675080B750900780812C5
:1006C0002B26EEFCEFFDEC75F00BA4FC75F00BEDAA
:1006D000A42AFD7A237B0012340A7404122AE80E3D
:1006E000EE70010F12876840C2028BE374F6122588
:1006F000177E007F00804C12874BF8A3E039F98801
:10070000828983E0A2E75036C2E7F08582088583BC
:10071000097808122B2675080B7509007808122B2A
:1007200026EEFCEFFDEC75F00BA4FC75F00BEDA4D0
:100730002AFD7A237B001234047404122AE80EEE98
:1007400070010F12876840AF028BE3EEF8EFF9E813
:1007500075F00BA4F812875922AAF075F00BE9A4E2
:100760002AF99019FDE028229019FB12AC46C3EE3D
:1007700098EF992274F6122517E4F508F509780820
:10078000122B269019FB12943675F00BA4FCA8F0DE
:1007900075F00BEDA428FD7A237B001233F8740268
:1007A000122AE8E9FE6003123C8602C6B274F61211
:1007B000251774FF122BB67E007F00803C851882BF
:1007C000851983E412919E122B2675080175090084
:1007D0007808122B26EEFCEFFDEC75F00BA4FCA8BC
:1007E000F075F00BEDA428FD7A237B00123404741D
:1007F00004122AE80EEE70010F12876840BF7401E0
:10080000028BE0C082C08390506EE49375F01CA40C
:10081000FCADF079FF7AF17B051232C6029E4B7473
:10082000F7122517E9FCEAFD7A007B008010EB1235
:100830008E799C4008E0F8EDC39840010A0B905077
:100840006EE493F8EBC39840E57B0002AC5A74EC7D
:1008500012251774F3122BB68A0C8B0D8C088D0998
:10086000890AEC45096016AA08AB09123CBC8A0E3D
:100870008B0FAE0EAF0FEE4F600302894C7A0080F3
:10088000010A90506E12BFD3500F128A4170F27459
:10089000F128FE740539FF80047E007F00EE4F7062
:1008A000030289F5905052128A1260257403650A7A
:1008B00060067404650A70197A047903123C928AFE
:1008C0000E8B0F90506EE493F8905052128A2B507A
:1008D0002D90504C128A12602C7401650A600674C7
:1008E00002650A70207A027901123C928A0E8B0FFF
:1008F00090506EE493F890504C128A2B40077A0087
:100900007B00028A0D8518828519837401F0122EEE
:1009100000E50CF0A3E50DF0AC08AD097403122E50
:1009200000AA82AB83123C2CAA18AB19123C687443
:100930000B122E0012A2448E828F83A3A3A3A3A323
:10094000A3E412C852AA0CAB0D1244FC7800E50ACD
:100950006007C39405500278048E828F83E50CF003
:10096000A3E50D128D3CA3A3E50AF0E88E828F83E8
:10097000A3A3A3A3A312C3635001097A027B0012AD
:10098000233112982BA3129CCA129857E50A605B78
:10099000C394035056901CC9E07018904F2B780CEC
:1009A000122CE5129802122D9D904F2B780C122CD0
:1009B000E58027F50875090074027808122CBF122B
:1009C0008A1C122CE590812B7810122D7F780C79DF
:1009D00010122428129802122D9DEE24131298054D
:1009E000122D9DEE241B12C35A800912980E1284F8
:1009F000DDA3F0A3F07A047900123C92128D2D4011
:100A000005901CE2E4F01243BEEEFAEFFB740D0217
:100A1000A051E493F8740193F9E84922742B250856
:100A2000F582744F3509F583780C22E493FA74014A
:100A300093FBE8C39AF8E49BF9C3E50E98E50F9998
:100A400022EA128A47F42275F01CA4F8A9F074F582
:100A500028F582740539F583E02274EE12251774A7
:100A6000F3122BB6EAFEEBFF8C108D11750800AA6D
:100A700010AB11123CBCEA4B7003028B758A828B5F
:100A800083E06E7003A3E06F7003028B758A828B24
:100A900083A3A3A3A3E0C394054003028B758A82BA
:100AA0008B8312C9ABE060728A828B83A3A3A3A35A
:100AB000E0C394035064901CC9E07021904F2B78E0
:100AC00008122CE5128B7C122D9D904F2B7808126A
:100AD0002CE5EA2413128B7F122D9D8030F50875CA
:100AE000090074027808122CBF128A1C122CE5909F
:100AF000812B7808122D7F780C7908122428129AFD
:100B00002C122D9DEA2413129A2F122D9DEA241BDC
:100B1000F582E43BF583E4F0801B7508FE7509FF60
:100B2000750AFF750BFF128B7C122D9DEA241312A0
:100B30008B7F122D9D750800750900750A00750BD5
:100B400000EA240C128B7F122D9D85188285198353
:100B50007401F0122E00EEF0A3EFF0AC10AD1174A2
:100B600003122E00AA82AB83123C2CAA18AB1912D6
:100B70003C68750801A908740D02C9A3EA2417F599
:100B800082E43BF58378082274F6122517123CB6EE
:100B90008A088B09A808A909E84960148882898312
:100BA000A3A3A3A3E06009C39405500479018002C4
:100BB0007900802F74F6122517123CB68A088B092B
:100BC000A808A909E849601488828983A3A3A3A37C
:100BD000E06009C394035004790180027900800326
:100BE000122AE87F0202284374F6122517123CB637
:100BF0008A828B83E5824583600BA3A3A3A3E07065
:100C00000479018002790080DAC082C083EAFCEBBB
:100C1000FD7A007B00029E48C082C0837C007D007C
:100C2000029E4874F512251774F3122BB6EAFEEBF8
:100C3000FF8C088D09C3EC94F8ED94FF4004EE4F4F
:100C40006065750A00801974FF6508700474FF659B
:100C500009600B12CF9C7004A3E06509603B050A94
:100C600090506EE493F8E50AC398503BE50A128A67
:100C70004260EBEE4F60D0128CB2122E0012C14ACD
:100C8000123C62E960D87403122E00AC82AD83EE90
:100C9000FAEFFB123482E960C5E50A75F01CA4F88E
:100CA000A9F0128E7080047A007B00740D122AE87D
:100CB000801B8518828519837401F074F328F582EE
:100CC000740539F58312AC46740B22A90A7F03021E
:100CD000284374F412251774F3122BB6750800120A
:100CE0003CBC8A0A8B0BAE0AAF0BEE4F6025851811
:100CF00082851983128D3A128CC5122E0012C14AB8
:100D0000123C4A7C1C7D0079FFEEFAEFFB1232C6E2
:100D10007508017A047900123C92128D2D500990C9
:100D20001CE27401F01243BEA908029B6D90506E44
:100D3000E493F8C3EA98EB940022740112A536A359
:100D4000A32274F7122517E9FE74FE6A700374FF7C
:100D50006B7C00700380240C128DA5501EEC128A4F
:100D60004260F4128F3F7003A3E06B70EA800BECDB
:100D7000128DBA6019E0640360140C128DA5501E28
:100D8000EE60ECEC128DAF60F1C3940550ECEC75A5
:100D9000F01CA4FCADF012D51212C08E80047AFEB5
:100DA0007BFF02AC5A90506EE493F8ECC398227526
:100DB000F01CA4F8A9F0128A4E2275F01CA4F8A920
:100DC000F0128A4E640122123CCE029E4BC082C0B9
:100DD00083790180F274F01225178A0A8B0B7A044A
:100DE0007901123C928A0C8B0DEA450D6040EA2A8B
:100DF000FAEB33FB1233808A088B09AE08AF09EE99
:100E00004F60267AFE7BFF123CD474FE6A70037436
:100E1000FF6B601E85088285098312AFD8E5082420
:100E200002F50850E2050980DE750C0080047E00A2
:100E30007F00850A82850B83E50CF0EEFAEFFB025A
:100E40009106C082C0837C008009EA24FF1AEB343B
:100E5000FFFB0C128DA55011EC128E79940550F207
:100E6000EA4B70E6128E7080047A007B00029E4B83
:100E700074F128FA740539FB22128A47C32274F7E9
:100E800012251774F3122BB67E00807DEF75F017D4
:100E9000A4F8A9F0128F3012C08EEE75F01CA4F8E1
:100EA000A9F0128F3F7003A3E06B603DEF75F01760
:100EB000A4F8AAF0EAF9128F3012A5437401122E99
:100EC00000E0687003A3E069601FEF75F017A4F8F5
:100ED000EAF974B328FC740739FD7403122E00AAD2
:100EE00082AB83123482E96013EF75F017A4F8A97E
:100EF000F074B128FA740739FB1245080F9050615D
:100F0000E493F8EFC39840840E12D4FF501FEE1202
:100F1000DA7DF47003A3E0F460EE128CB2122E00BE
:100F200012C14A123C62E960DF7F0080D002AC55FA
:100F3000128F342274B128F582740739F583221296
:100F4000DA886A2274F412251774F3122BB67E0025
:100F5000803890814B7808122D7FEE75F01CA4F834
:100F6000A9F0740428F582740639F5837808122CE8
:100F70000D60169081377808122D7FEE75F01CA455
:100F8000F812900C7808122C730E12D4FF507AEEDF
:100F9000128DAF60F4C3940350EF12900C122DDD4C
:100FA000E8494A4B70AC9019D4E06401702D901B55
:100FB0000412ADED6025EE75F01CA4F8A9F074F1F3
:100FC00028F8740539F912906212294B88828983B6
:100FD0001290F7124A897404122AE885188285193A
:100FE000837401F0EE75F01CA4F8A9F0128CBB120A
:100FF0002E0012C14A123C62E9608E7403122E0068
:10100000AA82AB83123CC88080029B6D740828F5CD
:1010100082740639F5832274F6122517123CB68ABB
:10102000088B09A808A909E849603288828983A346
:10103000A3A3A3E06023C39403501E129062122D59
:10104000C5E82417F582E439F583122DB9E8241B8D
:10105000F582E439F5837401F079018002790002A8
:101060008BE3E82413F582E439F5832274F012252A
:1010700017EAFEEBFF901AFE12ADED6072901B04B2
:1010800012ADED606A901B0812ADED606212D38B59
:10109000124A89E97059901CC9E0700A904F2B7868
:1010A00008122CE58028F5087509007402780812EA
:1010B0002CBF12D56D744F12D36C7808122CE590AA
:1010C000812B780C122D7F7808790C12242878084F
:1010D000122B1E1290F1124A897404122AE8E96454
:1010E00001700C8E828F83A3A312D379124A898058
:1010F000158E828F83A3A312B98D901B0412D38304
:1011000022740D122AE87F0802284374F61225176C
:10111000E4F508F5097808122B2690506EE493F553
:101120000874037808122CBF1294281233F8740242
:10113000122AE8E9FE740A6E6025E4F508F50978DC
:1011400008122B2690506EE49375F005A4FCADF0C8
:101150007A3F7B001233F87402122AE8EE60031221
:101160003D0402C6B274F612251774FE122BB68522
:101170001882851983E4F0A312919E122B2675081C
:10118000027509007808122B267C007D007A227BEC
:10119000001234047404122AE87402028BE0F0A8EE
:1011A00018A9198808890978082274EE122517747D
:1011B000DE122BB68A0E8B0F8C088D09750C007A07
:1011C000227B001233FE8A0A8B0B7A3F7B0012339C
:1011D000FE8A108B11AE10AF11E50A450B6017E5C2
:1011E00008650A7004E509650B600BAC0AAD0B7A63
:1011F000227B001234107436122E0012943BEE4FF4
:101200006015E50A6E7003E50B6F600BEEFCEFFDF9
:101210007A3F7B00123410E4F510F5117810122B90
:1012200026AC08AD097A227B001233F87402122A28
:10123000E8E9640A700302941EE4F508F5097808E9
:10124000122B26AC0AAD0B7A3F7B001233F87402E6
:10125000122AE8E9640A700302941E7404122B86B1
:10126000880889097808122B267508027509007804
:1012700008122B267C007D007A017B0312340A744D
:1012800004122AE8E9600302941E851882851983F6
:10129000E4F0A3F07E000293957406122B86880872
:1012A00089097808122B2675080875090078081234
:1012B0002B268E0874037808122CBFE5082402FC44
:1012C000E43509FD7A017B0312340A7404122AE81A
:1012D000E9600302941E7408122E00E0F47003A368
:1012E000E0F470030293947406122B86880889092F
:1012F0007808122B267508087509007808122B2625
:101300007404122E0012CCB374037808122CBF128E
:1013100094281234047404122AE8E9600302941E2B
:101320007402122B86880889097808122B26750802
:10133000057509007808122B26EE75F005A4FCADA2
:10134000F07A027B0312340A7404122AE8E970412D
:101350007402122B86880889097808122B267508D2
:10136000057509007808122B267404122E001294B9
:101370003675F005A4FCA8F075F005EDA428FD7AFB
:101380003F7B001234047404122AE8E960030294DB
:101390001E1299440E851882851983C082C08390DD
:1013A000506EE493F8D083D082C3E098A3E0940019
:1013B0005021851882851983C082C0837404122E3F
:1013C0000012A543D083D082C3E098A3E0995003D4
:1013D000029299A818A919880889097808122B2659
:1013E0007508027509007808122B267C007D007AAA
:1013F000227B001234047404122AE8E97020AC0E37
:10140000AD0F7A017B03123410E970127434122E7E
:101410000012C8567A027B03123410E96003750C7F
:1014200001A90C742202C9A3E5082402FCE43509D1
:10143000FD7A227B002212C85AEC22E0F50AA3E0D2
:10144000F50B2274EC12251774FE122BB6750A00E8
:10145000851882851983E4F0A3F090506E93F50E01
:10146000F50875090074037808122CBFE5082402FA
:10147000F50850020509E50E75F005A4F50EE5F036
:10148000F50F7A227B001233FE8A0C8B0DAE0CAF67
:101490000D7A3F7B001233FE8A108B11A818A91910
:1014A000880C890D780C122B26750C02750D0078AE
:1014B0000C122B267C007D007A227B0012340A74E9
:1014C00004122AE87A017B031233FE8A0C8B0D7A10
:1014D000027B031233FE8A128B13A812A913E50CA8
:1014E000450D700AE5086E7003E5096F7025E8493F
:1014F000700CE50E65107004E50F65117015E50CB4
:10150000450D607BEE4F604E85188285198312AFC2
:10151000DE60437C017D037A227B00124592E9F86C
:10152000880A705B7C027D037A3F7B00124592E95A
:10153000F8880A704AEEFCEFFD7A227B0012341024
:10154000E9700EAC10AD117A3F7B00123410E960E7
:1015500011750A018029AE0CAF0DE84960048810AE
:101560008911780E122B267810122B26AC08AD09A3
:10157000EEFAEFFB123D0A7404122AE8E9F50AA913
:101580000A740202A05174EC12251774D0122BB603
:10159000851882851983E4F0A3F0123D10E96003F9
:1015A0000297EAA818A919880889097808122B2631
:1015B0007508027509007808122B267C007D007AD8
:1015C000227B0012340A7404122AE8E960030297AD
:1015D000EA90506EE493F88518828519831298502A
:1015E000E49B50030297EA750A00750B007508002A
:1015F000803D7403122E00122DDD129821122DE968
:101600007403122E00122DDD12A868122DE9EE24AB
:101610001BF582E43FF583E4F07A047900123C92F2
:10162000128D2D4005901CE2E4F01243BE05081215
:1016300097F740030297EA12A53DC3E50A98E50B28
:101640009940030297EA7414122B86880C890D784E
:101650000C122B26750C08750D00780C122B2685A4
:10166000080C7403780C122CBFE50C2402FCE43542
:101670000DFD7A227B0012340A7404122AE8E97004
:10168000AC7416122E00E0F47003A3E0F4609E0523
:101690000AE50A7002050B7407122E007401F0743B
:1016A00016122E0012A5437412122E0012AF94745B
:1016B00007122B8E123C62E9700302962D12C8535A
:1016C0007414122E0012C08E1244FCE50875F01C32
:1016D000A4F8A9F074F128FE740539FF7414122BD4
:1016E00086880C890D750E00780C122B227C087DE3
:1016F00000EEFAEFFB1232BA7403122AE812C36842
:101700005001097A027B0012233112982B1298574C
:101710007402122B86880C890D780C122B26750CFE
:1017200005750D00780C122B26E50875F005A4FC54
:10173000ADF07A3F7B0012340A7404122AE8E960A3
:1017400003029619908137780C122D7F7403122EA4
:1017500000780C122C0D60030295F2E50875F01C60
:10176000A4F8AAF0EAF9128DB66071C39403506C24
:10177000901CC9E07018904F2B780C122CE5129831
:1017800002122D9D904F2B780C122CE58033F50C16
:10179000750D007402780C122CBF742B250CF58289
:1017A000744F12B95B780C122CE590812B781012D3
:1017B0002D7F780C7910122428EAF9129802122D44
:1017C0009DEE2413129805122D9DE50875F01CA4BA
:1017D000F8740C28F58274063902961512980E04D6
:1017E000141284DDA3F0A30296188518828519834C
:1017F000E0F9743002A05190506EE493F8E508C30C
:101800009822EE2417F582E43FF583780C22129893
:101810002174FEF0A304F0A3F0A3F012A86C74FEF0
:1018200022EE2417F582E43FF58322E88E828F832F
:10183000A3A3A3A3A3A3A3A312AC1A740112AC1A6B
:10184000A374AAF0EE2410F582E43FF583E4F022BD
:1018500012B98DC3E89A22A3F012AEACE4F0EE24E4
:101860000CF582E43FF583E4F0A3F0A3F0A3F022AB
:1018700074F212251774FE122BB68518828519830F
:10188000E4F0A3F075080002990FE50875F01CA4B8
:10189000F8A9F074F128F50C740539F50DAE087847
:1018A0000C122B26750A08750B00780A122B268E4F
:1018B0000A7403780A122CBFE50A2402FCE4350BF3
:1018C000FD7A227B001234047404122AE8E50C2409
:1018D00012F50AE4350DF50B780A122B26750A0568
:1018E000750B00780A122B26EE75F005A4FCADF0FE
:1018F0007A3F7B001234047404122AE8850C828536
:101900000D83A3A3A3A3E0F4600312994405081276
:1019100097F7500302988AA818A9198808890978A6
:1019200008122B267508027509007808122B267CF0
:10193000007D007A227B001234047404122AE874B9
:101940000202AEBA851882851983E02401F0A3E073
:101950003400F02274F012251774F3122BB6EAFE4D
:10196000EBFF7A027901123C92EA8E828F83F0704B
:1019700003029A1F75F00CA4FAABF01233808A08A8
:101980008B09EA45097003029A25AE08AF09750A6A
:1019900000801C90813712294BEEFAEFFB12333E88
:1019A0007404122AE88A0C8B0DAE0CAF0D050A9058
:1019B000506EE493F8E50AC398506AE50A128DBAAE
:1019C0006005E0640270E6128CB2122E0012C14A69
:1019D000123C62E960187403122E00AC82AD83EEF3
:1019E000FAEFFB1234888A0C8B0DAE0CAF0DE50AB2
:1019F00075F01CA4F8A9F0740C28F582740612D1B5
:101A0000EA6401708E128E70EA2413129A2F122D3E
:101A10007F129A2C122B9E780C122B1E029999750C
:101A20000800750900AA08AB09029101EA2417F51C
:101A300082E43BF583780C22C082C083901A06743E
:101A400074F0A37442F0901A08746EF0A37442F01C
:101A5000901A0C74C4F0A3743DF0029E4BC082C077
:101A600083901A0A7468F0A37442F0029E4B74F7D4
:101A7000122517EAFEEBFF901A78E06408601FE079
:101A80006404601A8E828F83E054036401704412F0
:101A9000AD18F8A3E0F5838882E0640670358E8285
:101AA0008F83A3A3E064FE7003A3E0F460258E821D
:101AB0008F83A3A312C8637003A3E0697008EE24A8
:101AC0001512C84A600512433A8003124340E9F5F3
:101AD0000880037508C2EEFAEFFB12338602835EBC
:101AE00074F41225178A088B098A828B83E0FAA383
:101AF000E0F8EA28FAE43400FB1233808A0A8B0B00
:101B0000AE0AAF0BEE4F605A850882850983E0FC70
:101B10007D0079001232C68E828F831284D91243DF
:101B2000768E828F83A3A3A3A3EAF0A3EB129B6814
:101B3000F8EE28F8E43F128651850882850983A3D0
:101B4000E0C0E012C34DD0E0F0124388EE240EF561
:101B500082E43FF583E912A4BEE0C0E012A216D0F1
:101B6000E0F0EEFAEFFB800A12A4B6E022740D1248
:101B70002AE87F0402284374F412251774E8122B14
:101B8000B68A088B098C0A8D0BE9FE901A78E064FE
:101B9000046005E06408700479C2804BA3780812E1
:101BA0002D9DEE901A7F129CCF1232C68518828529
:101BB00019837808122D9D7405122E00EEF074041E
:101BC000122E007401F07407122E00E4F0901A78BF
:101BD0007402F09019E6E0640270059019D4E4F004
:101BE000AA18AB19123B787418808474F412251764
